:1000000000800020BD010000EDDD0000A5DD000046
:10001000A5DD0000A5DD0000A5DD0000A5DD0000D8
:10002000A5DD0000A5DD0000A5DD0000EDDD000080
:10003000EDDD0000A5DD00006DD4000071D50000ED
:10004000EDDD0000EDDD0000EDDD0000EDDD000088
:10005000EDDD0000EDDD0000EDDD0000EDDD000078
:10006000EDDD0000EDDD0000EDDD0000EDDD000068
:10007000EDDD0000EDDD0000EDDD0000EDDD000058
:10008000EDDD0000EDDD0000EDDD0000EDDD000048
:10009000EDDD0000EDDD0000EDDD0000EDDD000038
:1000A000A9B90000B5B90000EDDD0000EDDD0000EC
:1000B000EDDD0000EDDD0000EDDD0000EDDD000018
:1000C000EDDD0000EDDD0000EDDD0000EDDD000008
:1000D000EDDD0000EDDD0000EDDD0000EDDD0000F8
:1000E000EDDD0000EDDD0000EDDD0000EDDD0000E8
:1000F000EDDD000009020100EDDD0000D9E800009F
:10010000EDDD000075EB0000EDDD0000EDDD000031
:10011000EDDD0000EDDD0000EDDD0000EDDD0000B7
:10012000EDDD0000EDDD0000EDDD0000EDDD0000A7
:10013000EDDD0000EDDD0000EDDD0000EDDD000097
:10014000EDDD0000EDDD0000EDDD0000EDDD000087
:100150005DD6000071D6000085D6000099D600005B
:10016000EDDD000091EE0000EDDD0000EDDD0000B2
:10017000EDDD0000EDDD0000EDDD0000EDDD000057
:10018000EDDD0000EDDD0000EDDD0000EDDD000047
:10019000EDDD0000EDDD0000EDDD0000EDDD000037
:1001A000EDDD0000EDDD0000EDDD0000EDDD000027
:1001B000EDDD0000EDDD0000EDDD0000564B4CF202
:1001C000205210B51A804DF628121A8000BF00BFC9
:1001D0000DF010FE514B4FF010621A60504A9A60B9
:1001E000504ADA60504A136813F4807304D14F49BF
:1001F0000B604FF4A85313604D4B1A78110703D5C9
:100200001A7842F008021A704A4B4B492A221A7097
:100210004A4A4B4B8B4204D252F8040F43F8040B6A
:10022000F8E7484B484900228B4202D243F8042B9E
:10023000FAE74649464A002352F8230041F82300D2
:1002400001336F2BF8D1434B434A802103F8011B44
:100250009342FBD1414B3D4A1A60414B8A221A70AE
:10026000A3F5805324225A70A0221A709A7992071B
:10027000FCD59A79D406FCD43A4A937903F00C035E
:10028000082B384BF9D103221A7140225A719A79FE
:100290009006FCD5334A9179324B4906FBD5324A58
:1002A000324911600221516020221A709A7902F0BD
:1002B0000C020C2AFAD12E4B2E4A1A602E4B2F4AD2
:1002C0001A6000225A60072243F8042C2C4AC3F813
:1002D0000C2D62B60EF03EF9144B1B68DA0705D5FB
:1002E00028480DF00BFF284B284A1A60284B1B7832
:1002F0005B0609D5244C254B22689A4204D121483B
:100300000DF0FCFE0023236011F036FA0DF078FDAD
:100310000DF0A6FCFEE700BF0E2005403080044033
:10032000823F04000100002B10D0034014D0034092
:1003300002D0074000E00740E49CFF1FA4530100E7
:100340004088FF1FE49CFF1F28A5FF1F0082FF1F9E
:100350000000000000E400E05FE400E008ED00E0E1
:100360000050064000400640448004400000030165
:1003700004800440C010050014E000E0FF76010096
:1003800000002020262831601CE00340A5C3945AB9
:1003900000F00740FFFFFFFFFFFFFFFFFFFFFFFF32
:1003A000FFFFFFFFFFFFFFFFFFFFFFFFFFFFFFFF5D
:1003B000FFFFFFFFFFFFFFFFFFFFFFFFFFFFFFFF4D
:1003C000FFFFFFFFFFFFFFFFFFFFFFFFFFFFFFFF3D
:1003D000FFFFFFFFFFFFFFFFFFFFFFFFFFFFFFFF2D
:1003E000FFFFFFFFFFFFFFFFFFFFFFFFFFFFFFFF1D
:1003F000FFFFFFFFFFFFFFFFFFFFFFFFFFFFFFFF0D
:10040000FFFFFFFFFFFFFFFFFFFFFFFFDEF9FFFF23
:1004100010B5054C237833B9044B13B10448AFF33E
:1004200000800123237010BDE49CFF1F000000002A
:10043000A8530100084B10B51BB108490848AFF399
:1004400000800848036803B910BD074B002BFBD0A0
:10045000BDE81040184700BF00000000E89CFF1FE7
:10046000A8530100E49CFF1F0000000038B50446BB
:10047000104621700A491D4610F060FF01464FF0FA
:100480007E5011F00FF8074910F058FFE5606060EA
:10049000256165610DF0EEFFE061204638BD00BFCB
:1004A000DB0FC9400024744938B50446104621705A
:1004B00009491D4610F042FF01464FF07E5010F0F2
:1004C000F1FF064910F03AFFE56060602561656163
:1004D0000DF0D0FFE06138BDDB0FC9400024744946
:1004E00038B503780446032B20D8DFE803F01A1848
:1004F0001002C168406910F017FE0D49054660689A
:1005000010F0D0FF0146284610F0CCFF38BD084956
:10051000406810F0C7FFE16810F010FF38BDC068F8
:1005200038BDC168406910F0FFFD38BD002038BDFE
:100530000024744970B504460E460DF09BFF054635
:10054000E069281A10F0A6FEE3682361E5616661A0
:10055000A0610146606810F0A5FF0146A060104848
:1005600010F0A0FF10F076FA0FF016FF10F088FDE3
:10057000054601464FF07E5010F0D6FD616910F03F
:10058000DDFE21690646284610F0D8FE01463046B9
:1005900010F0CCFDE0602046BDE87040FFF7A0BF42
:1005A000000080BF38B50E201C4C0DF033FA2188B6
:1005B0001B4B884205461A881DDA0023511AB1F5F3
:1005C000805FAABF1B03C3EB03330131142093FBED
:1005D000F1F10DF0A5FD134B1988F1B923889D4267
:1005E00010DAC3F57F630F33282091FBF3F1BDE8E8
:1005F00038400DF095BD9042D4BFC1EB0003C1EB74
:100600000203DBE740F6FF718D42D4BFC3EB050167
:10061000C3EB0101C1EB0131E3E738BDE89DFF1FEA
:10062000B29FFF1F509FFF1F10B504460CF0F4FF50
:10063000204610BD70B44C88A04220D9012301335C
:10064000DBB21CB2660031F8144084421D46F6D37A
:10065000A04211D005F10045013D965B31F815101F
:1006600032F81530401AF21A00FB02F0641A90FBBF
:10067000F4F4E01870BC7047905B70BC70470226C1
:100680000125E5E700280CDA064A434282FB0320F5
:10069000DA17C2EB600000EB4000A3EB8000C0F172
:1006A0000C007047ABAAAA2A38B5234B1B78002B45
:1006B0002CD015200DF0AEF9204B1860204B1B8874
:1006C000984203DA1F4C237863BB38BD1E4A148856
:1006D000A042A4EB0302A8BF20467F2A1CDDC01A5B
:1006E000C001541C90FBF4F4002CEBD0154B1A788D
:1006F0000AB901221A70154D2B689C4204D0144B84
:10070000E1B2187809F014FA2C6038BD11200EF00F
:100710009DFA0A4B1860D1E7C01AC0EBC01090FBDD
:10072000F2F4E1E70A4B0021187809F001FA0023FE
:10073000064A2370136038BD049FFF1F109DFF1FE2
:100740008E9DFF1FE49FFF1F7C9FFF1FDC9FFF1FED
:10075000689DFF1F38B50F200EF078FA1B4A1C4B1E
:1007600012881860C0F53B600830904220DB194BBE
:100770001B889842A3EB0204A8BF1846801A7F2C5E
:10078000C6BFC0010134C0EBC01090FBF4F47CB1D3
:10079000114B1A780AB901221A70104D2B689C422D
:1007A00004D00F4BE1B2187809F0C2F92C6038BDC3
:1007B000094C237803B938BD094B0021187809F09A
:1007C000B7F90023054A2370136038BDEC9DFF1F65
:1007D000289DFF1F689FFF1F8C9FFF1F9C9DFF1F71
:1007E000869DFF1FF0B40E8886420DD203F10043B0
:1007F000013B31F81350854202D9F0BCFFF71ABF14
:1008000032F81300F0BC70471088F0BC704700BF8E
:10081000094B1B880C2B09D8084A80B252F82320B8
:1008200028B143F6FE73984203D9108C70471088A4
:1008300070470349FFF7FEBE3E9DFF1FA42D010038
:10084000402F01004B4B4C4A2DE9F0471E8814689D
:100850004A4BB442B3F80080494B33DB4445A8BF50
:100860004446A6421C60C8BF00202DDDC6EB080729
:10087000B7F5804F33DB80037B1C90FBF3F0FFF771
:10088000C7FF404A404B15881B88C0F3C61909FBB7
:1008900005F57F2D8246A8BF7F252BB3A64253DCEA
:1008A0004445D4BFC6EB0404C6EB08049F42CCBF4A
:1008B00003FB04445C43354BC8BF013794FBF7F797
:1008C0001F6013E034461E60C6EB0807A045D4BF86
:1008D000C6EB0800C6EB0400B7F5804FCBDAC0EBDF
:1008E000803090FBF7F0CAE7284A1360284C236851
:1008F000994508D0274B1B88002B34D1264B1B88E9
:100900006BBBC4F80090254C23689A4506D0214B58
:100910001B885A1F032A19D9C4F800A0204C236849
:100920009D420FD01F4B188848B11A4B1E4A1B8896
:10093000D35C834203D0C0B2E9B209F0F9F8256074
:10094000BDE8F087BDE8F0870024AFE7164AD05C29
:100950002030C0B20AF07F0109F0EAF8DCE748462F
:1009600009F086F9CDE7104A4946D05C09F0E0F875
:10097000C4E700BFE89DFF1F4C9FFF1FB29FFF1FF2
:10098000089DFF1F189DFF1F1A9DFF1FB89FFF1F87
:10099000809DFF1F349FFF1FDA9DFF1F389DFF1FA3
:1009A000DC9DFF1F429FFF1F0C8AFF1F2DE9F04FA8
:1009B00001208BB00EF04AF9DFF870B3DFF870A3B6
:1009C000CBF8000000200EF041F9BA4BCAF8000045
:1009D0001B880C2B00F05E82B74EB84A3188B84BAA
:1009E00052F8214000221A70B64BB74A1B88B7490B
:1009F0001288013B012A31F91330059300F0AE81D2
:100A0000B34B0193B34B0293B34FDFF8288300231A
:100A10000093B24B1B88012B00F0F481DFF8189390
:100A2000AF4B0393D9F80050AE4B04930023AE4A6A
:100A30001288013A032A00F24982DFE812F0A50089
:100A4000ED000400C9002846059310F023FCA749D7
:100A500010F074FC059B0546184610F01BFCA449D9
:100A600010F06CFC0146284610F060FB10F02CFEE4
:100A70000546C9F80050386810F00CFC9B4910F08E
:100A80005DFC8146009810F005FC994910F056FC79
:100A90000146484610F04AFB10F016FE3860954AB1
:100AA000954B17881988954BDBF800201B88DFF8D9
:100AB0008CE2C7EB050C3D44039FC7F800C0471A02
:100AC000084404990D6001990F600299BEF8007006
:100AD00008609A4280F2E7800025C3EB070E744558
:100AE000DAF8000080F2D380611C984205FB01F522
:100AF0000EF1010E95FBFEF5C0F25F838742A8BFA1
:100B00000746FF1A01FB07F494FBFEF49A4200F338
:100B1000A780984200F3A480794C206810F0BAFBBB
:100B2000784910F00BFC784910F000FB10F0CCFD78
:100B3000A0F5FF531C3B082B98BF4FF40050D8F88A
:100B40000030184400282060C0F29F80B0F5804F2C
:100B500080F2F6806D4B1B781BB1B0F5005F40F062
:100B6000F7806B4D2B78002B40F0AB81694D2068EE
:100B70002B68634C984204D080B208F0A9FF236828
:100B80002B600BB0BDE8F08F2846059310F082FB78
:100B9000614910F0D3FB059B0546184610F07AFB1F
:100BA0005E4910F0CBFB0146284610F0BFFA10F06A
:100BB0008BFD0546C9F80050386810F06BFB5649AC
:100BC00010F0BCFB8146009810F064FB53495DE7D0
:100BD0002846059310F05EFB4A4910F0AFFB059BD9
:100BE0000546184610F056FB4D4910F0A7FB01468C
:100BF000284610F09BFA10F067FD0546C9F8005032
:100C0000386810F047FB3F4910F098FB8146009888
:100C100010F040FB424939E72846059310F03AFBB3
:100C2000404910F08BFB059B0546184610F032FB3F
:100C30003D4910F083FB0146284610F077FA10F08A
:100C400043FD0546C9F80050386810F023FB3549CC
:100C500010F074FB8146009810F01CFB324915E738
:100C60003388002B3FF458AF2B1B002BB8BF5B42DF
:100C7000092B00F32D81D8F80030214C4FF400509F
:100C8000184400282060BFF661AF00225AE0984265
:100C900005FB04F5B8BF002195FBFEF580F28482C8
:100CA00091FBFEF432E7BA42D4BFC3EB0205C3EBBB
:100CB000070512E77E9FFF1F769DFF1F8889FF1F94
:100CC0000E9DFF1F2089FF1F529FFF1FA4320100AE
:100CD000E09FFF1FAC9DFF1F009DFF1FE49EFF1FB5
:100CE000709FFF1FE89EFF1F5E89FF1FCDCC4C3F0A
:100CF000CDCC4C3E188AFF1F5C89FF1F489FFF1F09
:100D0000C089FF1F9A99193FCDCC4C4596A0FF1F73
:100D1000D89DFF1F2489FF1F3333733FCDCC4C3D3B
:100D2000CDCCCC3E6666663FCDCCCC3D709DFF1FE2
:100D3000349DFF1F889FFF1F6C9FFF1F549DFF1F47
:100D400043F6FF72C04B22601B78002B3FF409AFC3
:100D500005F094FFBD4B01221A7007E7BC4BBD4A5A
:100D60001B88BD491278013B31F91350002A40F02D
:100D7000C78011200DF06AFF0090B84B0193D3F8A3
:100D80000080009B984540F3C080B54BB54F1B8851
:100D9000B54A012B3B68B2F80090B44A0292204653
:100DA000A3EB050500F0E28010F074FA029A52F805
:100DB000291010F0C3FA0146002010F0B5F910F028
:100DC00083FC009BC8EB05029D42B8BF1D469042C4
:100DD000C8EB050580F2DE8000FB0555013295FB6E
:100DE000F2F5A34BDFF8B4820293D8F800302B441D
:100DF00003EBD3735B10C8F800309E4B1B88012BAC
:100E00007FF40CAE9C4B03931D460F200DF01EFF8C
:100E10002A6804929042034680F2CC80904A12885D
:100E2000012A00F03F81904A079012888F4D069268
:100E3000204610F02FFA069ADFF8649255F8221037
:100E4000D9F8005010F07AFA0146002010F06CF941
:100E5000059BEA1A059210F037FC059A079B049946
:100E60009A42C1EB020EB8BF1A46704580F2448127
:100E7000521A00FB02220EF1010192FBF1F2D8F8A6
:100E800000107E4804900A4402EBD2725210C8F857
:100E90000020CCE57A4B1B78002B3FF49DAD794EBA
:100EA000794A3188794B52F8210001221A7010F0EA
:100EB000F1F94FF07C5110F041FA10F005FC0446B6
:100EC00092E505F0D7FE00232B704FE63868E6E583
:100ED00005F500500130001B10F0DCF96C496D4C39
:100EE00010F02CFA0546206810F0D4F96A4910F089
:100EF00025FA0146284610F019F910F0E5FB1EE628
:100F000015200CF087FD009037E7594B0293D3F87A
:100F10000080009B984542DA514B524F1B88524A41
:100F2000012B3B68B2F80090504A039220461D44C2
:100F300000F0E98010F0AEF9039A52F8291010F091
:100F4000FDF910F0C1FB009B9D42C8EB0502A8BF54
:100F50001D46C8EB05059042BABF00FB055501329E
:100F6000454395FBF2F5DFF834813EE710F092F946
:100F7000029A52F8291010F0E1F910F0A5FB009B3D
:100F8000C8EB05029D42B8BF1D468242C8EB05056D
:100F90003FF722AF00FB05F595FBF2F521E7DFF8FF
:100FA000FC80304FD8F8003003EBD3735B10C8F8E7
:100FB00000302EE5314A049212680692904237DDE5
:100FC000274A1288012A00F0BC80274A099011881C
:100FD000264A08912046079210F05CF9079A089972
:100FE000DFF8BC9052F82110D9F8005010F0A6F9A3
:100FF000059B2B44059310F067FB0599099B069A06
:101000009942C2EB010EA8BF1946704580F2BE801E
:10101000891A00FB01110EF1010291FBF2F2D8F8DE
:1010200000100A4402EBD2725210C8F80020FEE40D
:10103000D8F80020DFF8689002EBD2725210D9F88D
:101040000050C8F80020F2E496A0FF1FD89DFF1FB3
:10105000648AFF1F049FFF1FF82E0100E09FFF1FFF
:10106000BE9DFF1F009DFF1F5C9DFF1FBC32010046
:10107000AC9DFF1FE49EFF1F709FFF1FE89EFF1F98
:10108000269DFF1F769DFF1F8889FF1F0E9DFF1F56
:10109000CDCCCC3EC089FF1F9A99193F889FFF1F76
:1010A0006C9FFF1F464A08901188464A07912046C8
:1010B000069210F0EFF8069A0799DFF80C9152F8B3
:1010C0002110D9F8005010F039F9059BE91A059163
:1010D00010F0FAFA0599089B049A9942C2EB010EA6
:1010E000B8BF1946704558DA891A00FB01110EF194
:1010F000010291FBF2F2C2E60499521A00FB02F2DD
:1011000092FBFEF2BBE610F0C5F8039A52F82910E4
:1011100010F014F90146002010F006F810F0D4FA8F
:10112000009A9542C8EB0503A8BF1546C8EB050514
:101130009842BABF00FB05550133454395FBF3F5D3
:1011400011E71F491F4A089020460D88079210F0AA
:10115000A1F8079ADFF8709052F82510D9F80050DE
:1011600010F0ECF8014600200FF0DEFF059B2B4449
:10117000059310F0A9FA0599089B069A9942C2EBCB
:10118000010EA8BF19467045FFF642AF069A891AAC
:1011900000FB01F191FBFEF241E7049A891A00FB82
:1011A00001F191FBFEF26AE6B842D4BFC3EB000145
:1011B000C3EB070104FB01F172E51F46A1E400BF88
:1011C0005C9DFF1FBC3201006C9FFF1F08B5244BC4
:1011D0001B88FBB1234B1B78FBB1234B1B78E3B17E
:1011E000224B1B78CBB1224B1B78B3B1214B224849
:1011F0001A78C2B9214A2249008812880968024433
:10120000B1EB620F09DD01221A706420BDE80840CD
:1012100005F048BD174A117801B908BD1370BDE843
:10122000084008F0F9BC154A164900881288096878
:101230000244B1EB620FF0DD00221A7008F0ECFC02
:10124000642005F02FFD642005F02CFD642005F0DE
:1012500029FD4FF41670BDE808400DF02DB900BF10
:10126000F69EFF1FAE9FFF1FAF9FFF1FB09FFF1F88
:10127000B19FFF1F3C9DFF1F549DFF1F489FFF1FF5
:10128000709DFF1F349DFF1F38B5114C232025781A
:101290000CF0C0FB0F4A42F82500131F02F1C400F6
:1012A000002253F8041F83420A44FAD123780A49E2
:1012B00007480A4C0133DBB2322B81FB025108BFD5
:1012C0000023D217C2EB21120370226038BD00BF89
:1012D0001C9DFF1FF89DFF1F1F85EB51449FFF1FA3
:1012E0002DE9F04FB84CB94D2068B94F83B00FF0DD
:1012F000D1FFB84910F022F8064610200DF0A6FCE8
:101300000FF0C8FFB44910F019F831460FF00EFF86
:1013100010F0DAF92988206088423B8843DA9E463B
:101320005B1A7F2B4FF0000247DDD2015E1C92FB5F
:10133000F6F2AA4EDFF8C882B6F800C0C8F800205E
:10134000BCF1190F00F0DF80BCF11A0F00F018811A
:10135000BCF11E0F00F021810126B146A04A12887F
:10136000002A00F09D808842C0F208817045D4BFF9
:10137000C1EB0000C1EB0E009A42BABF02FB0000B5
:101380000133504390FBF3F3964A1360964B188851
:10139000C0B9964A1288AAB9954B197801B11A704A
:1013A00003B0BDE8F08F9842D4BFC1EB0002C1EB9F
:1013B00003029E465B1A7F2BB7DCC2EBC21292FB84
:1013C000F3F2B6E72988D4F800E0DFF80082DFF80E
:1013D000F8A171456CDCDFF818C29CF80020002AE7
:1013E0002ED14FF0010B04288CF800B028D1002E2C
:1013F00040F095817D4B18880028D1D0B9F1000FBD
:10140000CED023682C883A88A34280F266810023DC
:10141000141B7E2C774DD5BFC3EB8313C3EBC313D3
:101420005B00013493FBF4F42B680134A34203D036
:10143000C0B2E1B208F07CFB2C6003B0BDE8F08FD5
:10144000012800F0F780022800F0EC800328D1D1B9
:10145000694B1B88092BCDD0002ECBD023682E885A
:101460003A88B34280F27C810023961B7E2EDFF8FF
:101470008CA1D5BFC3EB8313C3EBC3135B00013651
:1014800093FBF6F6DAF800300136B34203D0F1B23E
:101490004A2008F04DFBCAF80060ABE791460126F0
:1014A000BCF11E0F7FF472AF0022DFF858817FE09D
:1014B0004F4B1A78002A3FF473AF002401281C70A8
:1014C00000F0A480022840F00F81002E00F0A380DD
:1014D0004A4D2B68002B00F09E800420214608F026
:1014E00027FB424B2C60188800283FF459AFB9F114
:1014F000000F3FF455AFC0B2002108F019FB3D4B7F
:1015000000221A604CE7DFF8FC8098F80020C2B196
:10151000DFF8D890B9F800A0BAF1000F11D0DFF8C9
:10152000E89099F800B0934578D05FFA8AF07F216F
:1015300008F0FEFA98F80030B6F800C089F80030DC
:1015400010E0DFF8C49099F800A0924566D0274BD0
:101550000021187808F0ECFA98F80030B6F800C0CE
:1015600089F800301E4B1A88002A97D0BCF11E0F54
:1015700040F0078101264FF0000919E00020FBE64A
:10158000DFF8808098F80020002A0BBF0126002693
:101590004FF000094FF00109E0E6DFF86880104BDA
:1015A00098F800601A88B6FA86F676094FF00009B6
:1015B00098F80030002B3FF4E7AE2988B7F800E038
:1015C0002068C1EB0E03CEE6649DFF1FFC9EFF1F4B
:1015D000F89EFF1F9A99193FCDCCCC3E7E9FFF1FEE
:1015E000BC9FFF1FF09DFF1F6C9DFF1F909FFF1F63
:1015F000849FFF1F489DFF1F349FFF1FF49DFF1F07
:10160000649FFF1F269DFF1F229DFF1F1EB1624D7D
:101610002B68002B7CD1614B188865E701264FF0C1
:1016200000099BE6002E3FF4E5AEDFF86CA1DAF886
:1016300000202EE0002E3FF4DDAEB7F80080F0452C
:10164000D4BFC1EB0802C1EB0E02C1EB0808B8F130
:101650007E0FDFF844A1D5BFC2EB8212C2EBC212EB
:10166000520008F1010892FBF8F8DAF8002008F1BE
:101670000108424506D05FFA88F10120009308F086
:1016800057FA009B1888CAF8008002287FF4DEAE63
:1016900042462168B5F800803888414559DA002172
:1016A000C8EB0008B8F17E0FD3BFC1EB8111C1EBCD
:1016B000C11108F10108490091FBF8F808F101088F
:1016C000904506D05FFA88F10420009308F030FAC4
:1016D000009B1888CAF80080B8E69342D4BFC4EBD8
:1016E0000303C4EB020393E6032827D12C4B1B888A
:1016F000092B90D0002E8ED0274D2B68002B8AD03E
:101700004A20214608F014FA244B2C601888EBE696
:10171000214608F00DFA214B2C601888E4E64020A1
:101720007F218DE80C0008F003FA019B009A1888CD
:1017300058451CD002287FF489AE76E704287FF450
:101740006AAF002E3FF467AF2146402008F0F0F961
:1017500061E78142D4BFC8EB0101C8EB00019FE7FC
:101760009342D4BFC6EB0303C6EB02037DE6B8F891
:101770000010DAF800E0B7F800808E45FFF665AF9C
:101780005DE72988B7F800E02068C1EB0E03012669
:101790004FF00009E7E500BFF49DFF1F909FFF1F7A
:1017A000349FFF1F08B5114B1B88022B09D0052B56
:1017B00007D0032B15D0042B0BD00D4B01221A7030
:1017C00008BD7F21412008F0B3F9094B01221A70AE
:1017D00008BD7F21092008F0ABF9054B01221A70E2
:1017E00008BD4021092008F0A3F9E6E7EE9DFF1FA0
:1017F000929DFF1F38B5074B074D1B88052B0446EC
:1018000006D02B68834203D0C1B2052008F090F9BE
:101810002C6038BDEE9DFF1F989FFF1F38B5124DFD
:10182000124C2B88052B12D022684AB9022B0ED0FD
:10183000033B012B13D90E4A00231370236038BDDC
:101840000021052008F074F92B88022B04D1002117
:10185000412008F06DF9EEE7052BE9D1F7E700210B
:10186000092008F065F9E6E7EE9DFF1F989FFF1F2E
:10187000929DFF1F464B1B881D2B70B541D0454DD7
:101880000024454B1B88022B16D0444B1B88022B8F
:1018900054D02888424B002C1B780ADB8442A8BF16
:1018A000044634B1002B3AD02046BDE87040FFF723
:1018B000A1BF002B2FD170BD3A4B1B78002B37D026
:1018C00015200CF0A7F8384B1860384A1288002A07
:1018D000DBD0374A186811888142D6DC354B2A881C
:1018E0001B888342A3EB0106A8BF03465B1AB242E2
:1018F000BABF02FB03330136534393FBF6F31C4498
:10190000C3E72A4B1C888CB12B4B224D1C78002C32
:10191000B7D02C88B5E7BDE87040FFF77FBFFFF771
:1019200041FF2046BDE87040FFF764BF194DA8E7AE
:1019300011200DF08BF91C4B1860C6E70F200DF03D
:1019400085F91A4B1D4A1B881060002BA1D01C4A38
:10195000C0F53B63118808338B429ADB194A28880B
:1019600012889342A2EB0105A8BF1346A842A3EB3D
:10197000010306DA00FB0333013593FBF5F31C4446
:1019800088E700FB03F292FBF5F31C4482E700BFFB
:101990007E9FFF1F869FFF1F529FFF1FE49EFF1F1A
:1019A000929DFF1F049FFF1F109DFF1FEE9DFF1FB5
:1019B0008E9DFF1F7C9FFF1F269DFF1F289DFF1FE1
:1019C000EC9DFF1F689FFF1FF8B510200DF03EF93A
:1019D000C830B0F5FA7FC0F29680B0F57A6F014654
:1019E000A8BF4FF47A6101F51673B3F57A6FA8BFFB
:1019F0004FF47A639BB289B2914A924C11802220B3
:101A0000238008F0EFF921888F4D904C242008F0B6
:101A1000E9F90E200BF0FEFF40F6FF71C830884256
:101A2000A8BF084620EAE07000F2DC5283B28A4286
:101A3000A8BF0A460220194622802B8008F0D2F95E
:101A40002188042008F0CEF901200DF0FFF80446AB
:101A500000200DF0FBF8A042B8BF204600F1C801FD
:101A6000B1F5FA7FC0F2D180B1F57A6FA8BF4FF41B
:101A70007A6101F54873B3F57A6FA8BF4FF47A63C2
:101A80009BB289B2724A734C11800A20238008F0FD
:101A9000A9F921880C2008F0A5F90F200DF0D6F83F
:101AA000C0F53F610431B1F5AF6FC0F2AB80B1F565
:101AB000FA6FA8BF4FF4FA6189B2674BC0F5436073
:101AC000B0F5AF6F1980C0F29A80B0F5FA6FA8BF79
:101AD0004FF4FA6083B2614CA420238008F082F9AD
:101AE0002188A62008F07EF915200BF093FF00F561
:101AF0009671B1F52F7F0BDB41F25C23994240F3E5
:101B00008980194608E040F24C434FF4FA7173E7BC
:101B100040F214534FF42F71514A1180514C524DE1
:101B20002380062008F05EF92188504E082008F036
:101B300059F900274FF4AF74F9B24D4809F0A8FFE6
:101B400055F8043BC3F5967300FB03F086FB0023B6
:101B5000C017C0EB6310844207F10107A8BF044619
:101B6000062FE9D1434F414E0025E9B2424809F022
:101B70008FFF57F8043BC3F5967300FB03F086FB19
:101B80000023C017C0EB6310844205F10105A8BF14
:101B900004460C2DE9D1394F344E0025E9B23848BE
:101BA00009F076FF57F8043B304AC3F5967300FB03
:101BB00003F086FB0013C017C0EB6310844205F1ED
:101BC0000105A8BF04460C2DE8D1A4F11401312968
:101BD00031DD40F23A73A4F5B97403FB04F482FBDF
:101BE0000432E417A4EB621289B232322548264B44
:101BF00001801A602A20BDE8F84008F0F3B84FF4DD
:101C0000AF6368E74FF4AF6157E740F214534FF406
:101C1000FA7137E7124A00F5617089B2B0F52F7F8B
:101C20001180B8BF4FF42F73FFF678AF8342A8BF7F
:101C300003469BB272E740F26C723221D6E700BFD6
:101C4000FC9EFF1FF89EFF1FE89DFF1FB29FFF1F16
:101C5000489FFF1F549DFF1FEC9DFF1F689FFF1FA4
:101C60008E9DFF1F7C9FFF1F4C8AFF1FB5814E1B5F
:101C7000409DFF1F1C8AFF1F749DFF1F2C89FF1FA3
:101C8000E09DFF1FAC9FFF1F088AFF1F2DE9F84F43
:101C90000C200BF08BFE0C200CF040FBCB49DFF846
:101CA000B4A314200CF04AFBC949CA4809F082FBCE
:101CB000022103200CF0D8FB022104200CF0D4FBFD
:101CC000022105200CF0D0FB022106200CF0CCFBF9
:101CD00001210A200CF0C8FB012109200CF0C4FBF3
:101CE00001210D200CF0C0FB012128200CF0BCFBD1
:101CF000012114200CF0B8FB012116200CF0B4FBDC
:101D0000012117200CF0B0FB012121200CF0ACFBCD
:101D100002211C200CF0A8FB01211B200CF0A4FBCD
:101D200000211B200CF08CFB1C200CF08FFBB0FA68
:101D300080F35B091A208AF800300CF02BFD1F207D
:101D400000210CF0EDFC04200CF080FB002800F0DA
:101D5000318105200CF07AFB002800F0A6810023D9
:101D60009D4C062023700CF071FBB0FA80F35B09E8
:101D70004FF0000B994A137006F0BCFB2478002C3E
:101D800040F01481584608F057F8954B954A1B8847
:101D900015889549954840F23A72A3F5AF7302FB56
:101DA00003F381FB0312DB17A3EB621332330360EF
:101DB0008F4B01210D201D700CF042FB64200CF0B4
:101DC0007BFB4FF416710A200CF0AAF95D218948BB
:101DD00009F09AFE002800F0A58164200CF06CFB4D
:101DE00021460A200CF09CF94FF4967109200CF062
:101DF00097F95C21804809F087FE002800F07F8178
:101E000064200CF059FB214609200CF089F94FF4AD
:101E1000967116200CF084F95B21784809F074FE65
:101E2000002800F0498164200CF046FB2146162072
:101E30000CF076F94FF4967117200CF071F96420CC
:101E40000CF03AFB214617200CF06AF964200CF0E4
:101E500033FB21460D200CF0F3FA694A69481268F9
:101E6000DFF8F491684F694D694EDFF8F081002387
:101E70000121FEF719FB01233C602C60346089F8D6
:101E8000003004240F200CF0E1FE336803440E20E0
:101E900033600BF0BFFD3B6899F8002018443860B0
:101EA000002A7CD015200BF0B5FD2B681844286063
:101EB00004F0010080F0010004F0E4FEB8F8003006
:101EC000002B14BF4B20DC200CF0F6FA013CD9D1DA
:101ED000336839684C4A28684E4F002BB8BF03332B
:101EE0000029B8BF0331891011604B494B4A09885A
:101EF00014889B1000283360B8BF0330484E82100E
:101F0000581A19442A6031603860464D464847499E
:101F1000161B22442E6002600B60BBF1000F40F0E4
:101F2000AC80B8F80030002B00F09A80404B0124C0
:101F300004201C600CF08AFA18B93E4B2C4A1C7025
:101F400010703D4B1B881C2B00F09F803B4C04F114
:101F5000C80523200BF05EFD44F8040F01200CF0AF
:101F6000ABFAA542F5D19AF8003023B1344B1B7877
:101F7000002B40F09580002121200CF061FA314ABD
:101F8000314B1078187007F05FFD04F073FE45F6D2
:101F9000BF522E492E48BDE8F84F0BF0F3BA11207E
:101FA0000CF054FE2B681844286081E7BDE8F84F18
:101FB00009F010B906200CF049FA00287FF4C9AEE8
:101FC000054C034620704FF0010BD3E6001B37464B
:101FD00040420F00EC91FF1F449DFF1FEC9EFF1F2E
:101FE000AC9FFF1F809FFF1FB5814E1B088AFF1FFC
:101FF000A89DFF1F409DFF1FE09DFF1F749DFF1FB9
:102000002889FF1F109FFF1F149DFF1F009DFF1FAA
:102010006C9FFF1F709FFF1F188AFF1F5C89FF1FA7
:10202000E89EFF1FE09FFF1FAC9DFF1FC49FFF1F87
:10203000789FFF1F2C9DFF1F7E9FFF1FF49DFF1F9A
:10204000FE9EFF1F009FFF1FE39EFF1FA5050000D0
:10205000A09FFF1FE69EFF1F049FFF1F3E9FFF1FC5
:102060004FF4FA7004F01EFE04F008FE06F08CFD3A
:102070004FF4AF600CF020FA58E7FFF7A5FCB8F872
:102080000030002B7FF452AFEAE7294B1888002874
:102090003FF45CAF274BC0B2197807F049FD55E714
:1020A000012121200CF0CCF969E703200CF0CEF9D6
:1020B000B0FA80F35B0953E603200CF0C7F900285F
:1020C000FAD104200CF0C2F90028F5D105200CF05B
:1020D000BDF90028F0D106200CF0B8F90028EBD1AA
:1020E0000CF0D4FE04200CF0B1F940B905200CF03E
:1020F000ADF920B906200CF0A9F90028F0D0032092
:102100000CF0A4F90028FAD1ECE704200CF09EF9B9
:1021100040B905200CF09AF920B906200CF096F988
:102120000028DDD003200CF091F90028FAD1ECE76B
:10213000B09DFF1F609DFF1F2DE9F04FAD4C26782D
:10214000012E95B000F05582C0F00B82022E00F0F7
:10215000D880A949A94A91F800801178A84ADFF8E7
:102160003CE3A84DA84FA948A94B0292A94A009266
:10217000A94A9EF800B001922D78A84A3F7890F8BD
:1021800000E01B78DFF818A3DFF818C3DFF8189316
:102190000392012E84BF00222270A14AA14813702D
:1021A000A14A80F800B01570A048A14A077082F8D3
:1021B0000080A048A04A03709CBF013626701170B1
:1021C000BEF1000F40F074819C4A10880D2800F089
:1021D000B9819B4C00202070024604462DB19748DF
:1021E0000088002840F0BA810546964806882544B4
:1021F000002E40F067819448944C019E0078367818
:1022000024780130A0EB4600002C40F05682039C5D
:1022100094F800E0CEEB0004BEF1000F40F07682AF
:102220000026DFF874E202989EF800E00078A41B14
:10223000A4EB4E043C44CBEB040410B1B7FA87F096
:1022400040099CF800602718BC1B1EB11EF1000657
:1022500018BF0126009F99F8000097F800909AF89F
:1022600000C07B4FC6EB040EC0EB0E00A0EB490094
:102270008044C3EB0803A3EB41010C2313FB0C11B7
:102280003960744B744F754C75481B880088D7F8BB
:1022900000C0744E2788744C3688D4F800E0033BA5
:1022A000C0EBC00403EB4303C7EBC70001EB8303A0
:1022B00064446E4F334470446D4E57F8244056F8D2
:1022C00020000C3B1D44254405440AB1694B1960AC
:1022D000694A13689D4200F03181684B684819686B
:1022E0000791079901601B6808936648089B00885E
:1022F00015605B1A834284BF634B1D6015B0BDE857
:10230000F08FDFF8A881614E08AF0025E9B2604880
:1023100009F0BEFB58F8043BC3F5967300FB03F0CD
:1023200086FB00230135C017C0EB63100C2D47F866
:10233000040BEBD1574B384D0195384DB3F800C025
:102340000395109D09980F99404EDFF8C0A0DFF863
:10235000B490DFF8BC80654511AA8CCAAE46ACBF0C
:102360004FF0000E4FF0010E8445D4BF0020012035
:1023700030708C4528480B9D1F4E8AF800E0D4BF72
:1023800000210121017094452449DFF814A1D4BF34
:10239000002201220A709C453F4AD4BF002301233A
:1023A000BC45AB46D4BF002701271370AC45164B84
:1023B0000C9D1F70D4BF4FF0000B4FF0010B374B3B
:1023C0000F4A0292AC45DFF834C0124A83F800B0DD
:1023D000D4BF0025012589F8005098F800309CF8FA
:1023E000001096F80080DFF8BCC02678DFF8B890BF
:1023F0000092CEE6E29EFF1F309FFF1F329FFF1F1D
:10240000C09DFF1F379FFF1F909DFF1FEC9FFF1F69
:10241000319FFF1F829FFF1F959FFF1F969FFF1FEA
:10242000E69FFF1FE79FFF1FE89FFF1FE99FFF1F1A
:10243000EA9FFF1FEB9FFF1F839FFF1FEE9FFF1F62
:10244000269DFF1F0C9DFF1F1A8AFF1FD09FFF1F95
:10245000389FFF1F569FFF1FF09DFF1F949DFF1F7A
:10246000749FFF1F1E9DFF1FB89FFF1FB830010004
:10247000402A0100C89FFF1F889DFF1FD4A0FF1F97
:10248000789DFF1F8E9FFF1FD49FFF1FB5814E1B9E
:10249000E09DFF1FAC9FFF1F979FFF1F919DFF1F98
:1024A000ED9EFF1FE59FFF1FAA9FFF1F2C89FF1FA7
:1024B000AF4AB04814880122182C027040F20581FE
:1024C00000248BE6012E00F08F81022E00F0EE81B9
:1024D000032EA94B00F01F811E78009B9CF800E0A2
:1024E0001C78019B99F800C01878029B93F8008033
:1024F000039B1F78A6EB4E03A4EB8404CCEB030CE8
:10250000C0EB80760CEB0403C0EB8600034403EBC6
:10251000480303EB810327B198490978002940F06B
:10252000608201269AF800109548C1F1060101EB7E
:102530004101334403EB81010160A2E69149924BD2
:102540000968D0E6002D3FF444AE894A894E1488CC
:102550000122182C327040F2B8807446A0F10D05AB
:1025600043E6DFF87092894F0DF120080025E9B2AB
:10257000874809F08DFA59F8043BC3F5967300FBC0
:1025800003F087FB00230135C017C0EB6310062D55
:1025900048F8040BEBD17F4BDFF83CA219880D9B68
:1025A00000228B428AF8002080F2A2807A4B8AF8BF
:1025B00000507A497A4A7B4891F8008011787A4A2B
:1025C0001D7002920378794ADFF810C2DFF810928A
:1025D0000092774A774E784D784892F800E0784A32
:1025E0000192784A96F800B02D7807782678039201
:1025F000CFE5DFF8F081654E08AF0025E9B27248FB
:1026000009F046FA58F8043BC3F5967300FB03F053
:1026100086FB00230135C017C0EB63100C2D47F873
:10262000040BEBD15B4B0C9D1F885F4B02935F4B00
:1026300000930B9B0A98099ADFF8A0C1089EDFF867
:10264000A0910F99BB429E46ACBF4FF0000E4FF0D9
:10265000010EAF42D4BF002501258742109B8CF8A4
:102660000050D4BF00200120504D89F8000097424F
:10267000D4BF00220122B742D4BF4FF000084FF070
:1026800001082A709F42474A4448474E80F800801C
:10269000D4BF002301231370129A414886F800E04A
:1026A0008F42D4BF00210121974201701ADC002221
:1026B0004648DFF824A102708BE7039C46B12678D8
:1026C000002E40F06081441EABE50C3C012285E504
:1026D00094F800E00138CEEB0004BEF1000F7FF467
:1026E000A0AD9DE5119A9742D4BF00220122DFE7F9
:1026F0000C9A374B9142CCBF012200221A7040F352
:10270000458105258AF80050234B52E7002E3FF4FF
:1027100087AD012685E51C78009B029893F8008020
:10272000019B9CF800601B7890F800C099F800703D
:102730000398A4EB4604E71B90F800E0C3EB837416
:10274000A8EB88003844C3EB8403034403EB4C0339
:1027500003EB8103BEF1000F40F0488101269AF897
:102760000010074833440C2414FB0131016088E554
:102770007E9FFF1F269DFF1F1A8AFF1F979FFF1F27
:10278000389FFF1F789DFF1FD4A0FF1FB5814E1BF0
:10279000409DFF1FAC9FFF1FFA9EFF1F309FFF1F32
:1027A000329FFF1F319FFF1FC09DFF1F829FFF1F92
:1027B000EC9FFF1F919DFF1F379FFF1F909DFF1FE5
:1027C000959FFF1F969FFF1F749DFF1F5A9DFF1F20
:1027D000B19FFF1F4C8AFF1FED9EFF1FE59FFF1F4C
:1027E000AA9FFF1F1C8AFF1FA34CDFF89CE22078E2
:1027F00005909EF8004001980494059C0078019093
:102800000134A4EB40040498002840F0AF80039802
:1028100090F800E00498261ACEEB06000390BEF173
:10282000000F40F09E8074460298944E007802900B
:10283000039836780496041BA4EB460402983C44A3
:10284000CBEB0404002800F08780B7FA87F040093A
:102850009CF800602044871B1EB10498061C18BF1A
:102860000126009C99F800002478BE1B301AA0EBCA
:10287000440080440198C3EB0803A3EB4103002804
:1028800067D1BEF1000F40F0BB807344002C5ED1D5
:1028900000290CBF00206FF009009AF80010784C56
:1028A00003440C2010FB01312160EAE4039E019CEB
:1028B00036780396009E2478019434786F4E7148E0
:1028C00099F800E0009496F800906F4C9DF80C6029
:1028D00086709DF80460067080F806E09DF8006040
:1028E00080F803909CF800C02478DFF8B491DDF8FC
:1028F00004E080F80880077180F805C0C671417255
:1029000044704FF000080120009500215D4C0D46F9
:102910005FFA88FC4F46764607E0022809D00A296C
:102920000BD014F8016F17F8010F864201F1010175
:10293000F3D101350A29EDB2F3D1092D72D808F18E
:102940000108B8F1100F36D019F80A0FDDE70020A2
:10295000A3E74FF0000E98E7029879E7CEEB04006A
:1029600003900198041C18BF01245DE7019800281A
:102970004ED0039890F800E0BEF1000FEED1601E3B
:102980000390744650E7841B01264AE40B9A3F4BA0
:102990009142CCBF012200221A703EDC0A9A3C4BC5
:1029A0009142CCBF012200221A7052DD03258AF821
:1029B0000050384BFDE5304837490478C86B029920
:1029C000009D097801342044CBEB0000084400212D
:1029D0009AF800402A4B401A0C2111FB040119609F
:1029E0004FE41BF1000618BF01269BE52349097837
:1029F00000293FF4B3AE1BF1000618BF0126AEE676
:102A0000049800280CBF4FF0000E4FF0090E3CE771
:102A1000039890F800E03046FDE604258AF800505F
:102A20001C4BC6E514481C49047851F8280002994B
:102A3000009D097801342044CBEB00006646084431
:102A4000002BC4D0002EC2D1BBF1000FBFD001219A
:102A5000BEE7099A114B9142CCBF012200221A70A5
:102A600004DD02258AF800500A4BA2E5089B994232
:102A700018DD01259AE500BF1A8AFF1F979FFF1FE7
:102A8000389FFF1FB49DFF1FD09FFF1FB09FFF1FE8
:102A9000AF9FFF1FFA9EFF1FC889FF1FAE9FFF1F3A
:102AA000882F0100154B1D78012D25D9144A8AF86D
:102AB00000501288D2B1134A1288013A92B2062A03
:102AC00014D8114A12788AB1104A1268012A7FF488
:102AD00070AD0F4A0F4E10680C2290FBF2F102FB12
:102AE000110232800C4A0321117062E5074A126814
:102AF000012A7FF45EADF5E735465AE5FA9EFF1FE1
:102B0000609FFF1F029FFF1FEA9DFF1F789FFF1F0F
:102B1000D49FFF1F3C9FFF1FBC89FF1F2DE9F04F73
:102B20003A4B1B788BB0002B6BD10E200AF072FF52
:102B30000EF0B0FB01463648364E374DFDF7FAFC35
:102B40003348FDF7CDFC0EF0BFFD80F30C00306084
:102B5000FFF7F2FA2C68012C7AD0022C00F00683E1
:102B6000032C00F02C842D4E2D4C33682D4A2E4E14
:102B70000993099B316812882360591A013A9142DE
:102B8000274F00F2EE82294E32689A1A0D2A00F27F
:102B9000D782274E32689A1A132A00F2CC82254E29
:102BA00032689A1A252A1AD9234B1B88002B40F029
:102BB0005B81224B1B78002B40F05681FEF764FBB3
:102BC0001F4B1B881B3B9BB2022B04D81D4B1B7851
:102BD000002B40F04C8104F077F8236833601A4DE5
:102BE0002A689B1A502B00F20D82184B1B88012B70
:102BF00000F0258206F020FF06F004FE0BB0BDE8D1
:102C0000F08F08F06FF90BB0BDE8F08F449DFF1F07
:102C1000109FFF1F4C9FFF1F789FFF1FD4A0FF1F17
:102C20000C9FFF1FC489FF1FE49DFF1FCC9DFF1F4A
:102C3000A09DFF1FA49DFF1FF69EFF1F3C9DFF1F31
:102C40007E9FFF1F269DFF1FF09EFF1F509FFF1FAF
:102C5000DFF820939F4AB9F800001378834204D02C
:102C6000C3B21846137006F0D9FEDFF804839A4AFF
:102C7000B8F800301178994204D0984F397800297B
:102C800040F04087964A33681288964E9A42C0F2C6
:102C9000F880954A1278002A40F0F380DFF8D8A235
:102CA000BAF8003023B9914B1B88002B00F05885EF
:102CB0008F4A904B11881B888F4A0B4412685B1017
:102CC00093428E4A126880F2FA8400219342B4BF84
:102CD00001230B4604910093ACBF4FF0010B8B46D0
:102CE00005910E200AF096FE854B864A1B681768F0
:102CF00003930133A7F25232002B8446029240F331
:102D00001287802BA8BF80237F4A804912780191C7
:102D1000002A00F0C0800978914200F0BC80B8F829
:102D20000010DFF84CE2994201F0FC806B49AEF8EC
:102D30000030774B4FF0010E81F800E01978DFF892
:102D40003CE2019B8EF800101A70009B002B00F0F3
:102D50001781BAF80030002B00F012816D4B1B6810
:102D60005A1C002A40F3E386802A00F3DF866A4C6F
:102D70006A496B482488098800682144B0EB610FD8
:102D8000C1F24283A3F148020F2A02D8473BA9F8B7
:102D900000300E200AF03EFE6FF454731F44874249
:102DA00002DC604B00221A705F4B1B88002B00F086
:102DB0007D845E4B5E4A1B781178994243D0002B8C
:102DC00041D05C490C78002C00F075875A4991F885
:102DD00000C0BCF1000F40F06C87584F0097584F6F
:102DE00058480297554F007887F800C0544F4FF06D
:102DF000010E87F800C081F800E0002841F0E28071
:102E000051490978002901F03680504903910C4658
:102E10000978002941F02C804D48494F00783970DD
:102E200001210297217070B14448434900904948FC
:102E300003270770002008700099029F087003990B
:102E400001243C7008701370434B1B88A3F11B02D4
:102E5000012A40F21D861D2B7FF486AE3C4A3F4B73
:102E600012781A703E4C80E6FEF7B0F9A6E63D4BAC
:102E70001B78002B3FF4AFAE2B68012B7FF4ABAE79
:102E8000ABE63168384A069106983849106002224C
:102E90000B602A6002E71E49DFF8E0E009780029AC
:102EA0003FF44FAF9EF8000081423FF44AAF0398D1
:102EB0004B2840F3FE871833802BB8F80000A8BFDA
:102EC000802398423FF43DAF294803800348012303
:102ED000037036E7E39EFF1FA89DFF1F2C9DFF1F79
:102EE000E89DFF1FD4A0FF1F3C9DFF1FD29DFF1F29
:102EF000549DFF1F489FFF1F709DFF1F349DFF1FA4
:102F0000C89FFF1F149DFF1FBE9FFF1F849DFF1FB3
:102F1000BF9FFF1F389FFF1FFC9EFF1FF89EFF1FD4
:102F2000649DFF1F4C9DFF1F029FFF1F5A9DFF1FA7
:102F3000049DFF1FE99FFF1F409FFF1F949FFF1FDE
:102F4000EA9DFF1FEA9FFF1FE69FFF1F059DFF1FD2
:102F5000269DFF1FBC89FF1F7E9FFF1F229DFF1F15
:102F60000C9FFF1F839FFF1F989DFF1F089FFF1F40
:102F7000809FFF1F009FFF1F8C9DFF1F859DFF1FD0
:102F8000029B9C45BFF605AFA54B1B88002B3FF469
:102F900000AFBBF1000F7FF4E1AEA24B1B881BB169
:102FA000059B002B7FF4DAAE049B002B3FF4F1AEBF
:102FB0009D4B1A78002A7FF4ECAEDFF8109399F855
:102FC000004001221A70002C40F09783974B1B7829
:102FD000002B02F0B980964B1B78002B02F08E83F9
:102FE000944B1B78002B7FF4D4AE934B1B78002BB3
:102FF0003FF4CFAEB8F8003090490A3BA8F8003053
:103000000A70C6E605F0BEFA8D4B1B7873B98D4B7E
:103010001B785BB98C4B1B7843B98C4B1B782BB955
:103020008B4B1B7813B903F025FE01E003F02EFE55
:1030300023682B60874B1B88012B7FF4DBAD864B0D
:10304000864A1B6886481178183B2A2202FB03F344
:1030500003608448A9B10268934200F3C38310DA85
:10306000814D2978002940F09A8780490D68D5F173
:103070007F0548BF0335AD100135521B9342B8BFE1
:1030800013467B4A1268A92101FB02F2002ABCBF49
:1030900002F57F523F3277499213543A098813441C
:1030A000036051B3744A246852F82110B4FBF1F262
:1030B000782901FB124200F35783C2EB0212D200BF
:1030C00092FBF1F26D4C6E4954F8222009686D4C68
:1030D000A2F2FF7201FB02F202F57D3202F560728C
:1030E00002EB4201C2EBC10284FB02411144D21740
:1030F000C2EBA1420B3A134403606349634A0C8854
:10310000118804F65C72B2F57C6FA1F16400BABF5D
:1031100004F65D725E495F4903FB02F281FB0231F6
:103120001144D317C3EBE123C11881F30C0128200C
:103130000AF0F6FF5EE5FEF79DFB236833602EE59F
:10314000FDF734FCFEF7CCF8534B1B88032B00F043
:103150000E85524B1B88032B00F0058523683360D6
:1031600017E5FDF76FFB3B6833600CE54C4A3468AC
:103170001288A24204DB364B1B78002B00F05E83E2
:10318000484E494833680793484B079900681B88A5
:10319000091A994200F2C180002B00F0BE80444B16
:1031A000198800293FF4E0AC424B43481B68008873
:1031B000A342B8BF23469A4241F31F813F4B1A6096
:1031C000DFF80C8188F80010234FFDF73BFB3868CF
:1031D0007F2840F360853A4B7F3883FB0032C3176A
:1031E000C3EB620303EB4303A0EB83007330354B67
:1031F00001931B883860002B40F07B86124B0093B4
:103200001B78002B00F0C5832F4C2378002B00F097
:10321000C083DFF8C090DFF8A8A04FF0000B68E093
:10322000D29DFF1F069FFF1F4C9DFF1FE69FFF1FA4
:10323000E79FFF1FE89FFF1FE99FFF1F2C9DFF1FB8
:10324000EA9DFF1F409FFF1F949FFF1F059DFF1FCB
:103250003C9DFF1F509FFF1FD49FFF1F929DFF1F8C
:10326000C49DFF1FD49DFF1F9C9FFF1F989FFF1FA2
:10327000C089FF1F209DFF1F642F01003C28010013
:10328000649FFF1F4D261281D89FFF1FA89FFF1F1D
:1032900081DFFF8183200882529FFF1FE49EFF1F72
:1032A000E89DFF1FD4A0FF1F989DFF1FD09DFF1F0B
:1032B000249DFF1F089FFF1FB29FFF1F089DFF1F38
:1032C000ABAAAA2A6A9DFF1F8489FF1FED9EFF1FDC
:1032D000C19DFF1F5C89FF1F03F17300C0B298F806
:1032E000001006F055FC23780BF1010B5B4540F311
:1032F00050833B6859F8040F1844A0F17F038AFB00
:103300000321DA17C2EB610202EB42027F28A3EB32
:103310008203E1DCFDF7B6F9E0E7554B55491B6840
:1033200008885549A342B8BF23469A4200F36D82EC
:10333000524C09888342A8BF0346236000297FF4CA
:103340003FAF9A42C8BF0B4640F36682801AB0F581
:10335000804FAABF9B03C3EB8333013093FBF0F094
:10336000FDF756FAC0F3C6100DF094FF444B044627
:1033700018880DF08FFF4349074620460DF0DEFF09
:10338000014638460DF0DAFF21460DF0CFFE4FF032
:103390007E5104460EF070F9002841F023803A492E
:1033A00020460EF087F9002840F0068620460EF0F1
:1033B000B1F9C0B2DFF8F08088F8000004E7334BC1
:1033C00034681988A14273DD314B1B78002B6FD113
:1033D000DFF8D89099F800007F2840F3DC85A3F14E
:1033E00055337F3803F1004383FB0032C317C3EB2F
:1033F000620303EB4303A0EB83007330254B01937F
:103400001B88C0B289F80000002B40F0D687224B01
:1034100000931B78002B00F07B84204C2378002B3A
:1034200000F076841E4FDFF87C804FF0000A0AE03F
:1034300003F17300C0B206F0CFFB23780AF1010A52
:10344000534540F3658457F8043F99F80000184449
:10345000A0F17F0388FB0321DA17C2EB610202EBC4
:1034600042027F28A3EB8203E2DCFDF70BF9E1E7E0
:10347000089FFF1FB29FFF1F249DFF1F089DFF1F76
:10348000C09FFF1FCDCCCC3D0000FE42E89DFF1F3A
:103490003C9DFF1F6A9DFF1F949FFF1F8489FF1F94
:1034A0005C89FF1FABAAAA2AC19DFF1F369FFF1F81
:1034B000B14F38687F2840F3B681B04B7F3883FB2B
:1034C0000032C317C3EB620303EB4303A0EB83009B
:1034D0007330DFF8009399F800A0824500F0FF8177
:1034E000A74B1B88002B43D1A64AA7481268008827
:1034F000914205DC8242D4BFC1EB0203C1EB000361
:10350000411AB1F5804FA6BF9B030131C3EB833352
:1035100093FBF1F0FDF77CF9C0F3C6100DF0BAFE95
:103520009A4B044618880DF0B5FE9949804620460E
:103530000DF004FF014640460DF000FF21460DF05E
:10354000F5FD4FF07E5104460EF096F8002840F04D
:10355000A486904920460EF0ADF8002840F0298559
:1035600020460EF0D7F8C0B2DFF86C8288F8000071
:10357000BAF17F0F40F38B838048AAF17F0A80FB6A
:103580000A304FEAEA73C3EB600000EB4000AAEB9D
:1035900080007330804B00931B78C0B289F8000024
:1035A000002B40F0EB827D4B03931B78002B40F007
:1035B000D5847B4B02931B78002B40F01687794B08
:1035C0000193029B1B78FBB1774B1B88012B00F00A
:1035D000E285022B00F06E87032B01F08881042B1B
:1035E00001F00F83052B01F02B84062B01F0808561
:1035F000072B01F03387082B02F03980092B02F0EA
:103600007D810A2B02F09282009B1B78002B00F038
:103610004284019B634C1988002900F09884386823
:103620007F2840F3A882554B7F3883FB0032C317B5
:10363000C3EB620303EB4303A0EB830073303860FA
:10364000002940F04D84009B1B78002B00F0538133
:10365000564C2378002B00F04E81DFF880A1DFF874
:1036600078814FF0000B0CE003F17300C0B298F8C2
:10367000001006F08DFA23780BF1010B5B4540F347
:103680003A813B685AF8040F3C4A1844A0F17F0382
:1036900082FB0321DA17C2EB610202EB42027F28B0
:1036A000A3EB8203E0DCFCF7EDFFDFE73C4C404896
:1036B00039493A4A237003700B70FFF7C4BB934239
:1036C0004FF0000B80F2B2800123CDF800B0CDF8AE
:1036D00014B00493FFF705BB364B1B78002B7FF427
:1036E00058AB039B344A243B83F34703D9B25B2096
:1036F000136006F01DFA99F80040032C30D1DFF872
:10370000E08098F80030002B42F040812B4F3B784E
:10371000002B42F02E81274C2378002B42F01C8195
:10372000274B1B78002B42F00A81264A1380264B38
:103730001B78002B42F0D081114B7F221A8098F821
:1037400000306BB93B785BB923784BB91F4A7F21B6
:103750000720138006F0ECF97F210B2006F0E8F932
:103760001B4B1F68FFF715BBC2EB0214013102EBC4
:10377000C40292FBF1F2A5E4D49FFF1FABAAAA2AD0
:10378000249DFF1F089DFF1FB29FFF1FC09FFF1FAB
:10379000CDCCCC3D0000FE42949FFF1F059DFF1F36
:1037A000EA9DFF1F6A9DFF1F029FFF1F8489FF1F65
:1037B000409FFF1FE99FFF1F509DFF1FE89FFF1FB6
:1037C000E79FFF1FDA9DFF1FEA9FFF1F349FFF1F28
:1037D000149DFF1F369FFF1FC19DFF1F5C89FF1FA8
:1037E000E69FFF1FB3490D78002D40F03783B249A3
:1037F0000968D1F17F0148BF033102EBA1014A1CE6
:1038000093420260A8BF13463BE4AC4B09881A60A0
:1038100000297FF4D5AC13469842D4BFC2EB000315
:10382000C2EB030392E5FCF72DFF52E60123CDF82E
:1038300010B0CDF800B00593FFF753BA01232B6009
:10384000FFF791B9029B1B78FBB19D4B1B88012BA5
:1038500000F01A84022B00F0AB86032B00F0CE8719
:10386000042B01F0F381052B01F06E82062B01F091
:103870003784072B01F03F85082B01F0AF86092B19
:1038800002F005800A2B02F07681019B1B88002B39
:1038900000F02083009B1B783BB9039B1B7823B966
:1038A000029B1B78002B00F08987864B1B78002B2E
:1038B00000F0FE8084490B78082B00F2F9808348E1
:1038C0003A680068824C0133DBB25F1E101A44F87C
:1038D00027000B707F4B3468198889F80020A142BB
:1038E0007D4EBFF641A932687C4B0892089A7C4C09
:1038F0001A60FFF73AB9039B1B78002BA2D03B68F4
:10390000A3F10C007F2840F3408376488B3B80FB7B
:103910000320DA17C2EB600000EB4000A3EB80034A
:1039200003F17300DFF8D081C0B298F8001006F000
:103930002FF9009B1B78002B84D0634C2378002B3D
:1039400080D0DFF8B8A14FF0000B0CE003F173005A
:10395000C0B298F8001006F01BF923780BF1010BA8
:103960005B457FF76FAF3B685AF8040F5D4A184418
:10397000A0F18B0382FB0321DA17C2EB61020C3842
:1039800002EB42027F28A3EB8203DFDCFCF77AFE26
:10399000DEE74C4B1B78002B40F0B2823B68524A6A
:1039A0001278002A45D0A3F10C007F2840F3F08262
:1039B0004C4A8B3B82FB0321DA17C2EB610202EB1C
:1039C0004202A3EB820303F17300C0B298F8001027
:1039D00006F0DEF8009B1B7853B33B4C23783BB3D7
:1039E000DFF81891DFF8FCA04FF0000B0BE003F1BB
:1039F0007300C0B298F8001006F0CAF823780BF1F3
:103A0000010B5B4514DD3B6859F8040F1844A0F125
:103A10008B038AFB0321DA17C2EB61020C3802EB3D
:103A200042027F28A3EB8203E1DCFCF72BFEE0E7F8
:103A30003B682E4A1278FAB1214A1288012A00F016
:103A40002F84022A00F03586032A00F0CA87042A50
:103A500001F02081052A01F05582062A01F06D83CC
:103A6000072A01F0A383082A01F05B86092A01F0E6
:103A7000D1860A2A02F0BD80019A1288002A00F03D
:103A80004A821B4A164C137003232B60FFF76DB854
:103A9000DFF86C8098F80030002B40F00081154F63
:103AA0003B78002B40F0B3840D4C3B70FFF75DB8C2
:103AB0003A680FE79C9FFF1F989FFF1F089DFF1FFD
:103AC000029FFF1F409FFF1F8489FF1F309DFF1F24
:103AD0006089FF1FE89DFF1FD4A0FF1F80A0FF1F6C
:103AE0000C9FFF1FABAAAA2A059DFF1FEA9DFF1F7F
:103AF000369FFF1F229DFF1FC19DFF1F5C89FF1F77
:103B0000269DFF1FDBB21846137006F0CFF8A54BB9
:103B1000A5491A46A54B184600230B703B7013703D
:103B20000370FFF7AFB80123FFF7EEB88024A04978
:103B3000A04BA14A09881B8812680B44B2EB630FA3
:103B4000BFF627A99D4B1B78002B40F0F181B8F8F8
:103B500000309B4AA3423FF41CA99A4B14800122D7
:103B60001A70FFF716B9FCF7F5FDFFF7F7BAFCF787
:103B70009BFDFFF7EEBAFCF785FD60E5924B0193E4
:103B80001B8863BB894B0393904B0293904C237823
:103B90007BB3DFF85882DFF83CA24FF0000B09E05E
:103BA00003F17300C0B206F017F823780BF1010B94
:103BB0005B451EDD58F8043F99F800001844A0F159
:103BC0007F038AFB0321DA17C2EB610202EB420298
:103BD0007F28A3EB8203E3DCFCF754FDE2E7734BA1
:103BE00003937A4B029305F0F7FF009B1B78002BA1
:103BF000CCD1039B1B78002B3FF4E3AC99F8003049
:103C0000A3F10C007F2840F3BD8172488B3B80FB01
:103C10000320DA17C2EB600000EB4000A3EB800347
:103C200003F17300C0B205F0D7FF009B1B78002B97
:103C300000F09D81664C2378002B01F06282DFF852
:103C4000AC81DFF890A14FF0000B0AE003F17300A4
:103C5000C0B205F0C1FF23780BF1010B5B457FF784
:103C6000B0AC58F8043F99F800001844A0F18B0359
:103C70008AFB0321DA17C2EB61020C3802EB420225
:103C80007F28A3EB8203E1DCFCF7FCFCE0E7504675
:103C9000FCF7F8FC7EE4FCF7F5FCFFF7A8BA4E4A07
:103CA0001278002A40F09B814C4F4D4C3B70FEF740
:103CB0005CBF002008704B49087840B13949009139
:103CC0000978002900F07B81009F00213970464966
:103CD000097800297FF499A8002C40F0CC800028B6
:103CE00040F0C980354C2F4F94F800E02F4C0394DE
:103CF000364C02942D4C2C492070344C009708709F
:103D000038702070BEF1000F7FF491A8FFF79BB8C8
:103D1000264B1B78002B6BD099F80030A3F10C00D8
:103D20007F2840F399832B4A8B3B82FB0321DA17D0
:103D3000C2EB610202EB4202A3EB820303F17300C8
:103D4000C0B205F049FF009B1B78002B50D0204CDF
:103D50002378002B4CD0254FDFF878804FF0000AF5
:103D600009E003F17300C0B205F036FF23780AF1D1
:103D7000010A53453CDD57F8043F99F80000184408
:103D8000A0F18B0388FB0321DA17C2EB61020C3828
:103D900002EB42027F28A3EB8203E2DCFCF772FC19
:103DA000E1E700BF949FFF1F409FFF1F059DFF1F7E
:103DB000FC9EFF1FF89EFF1F649DFF1F269DFF1F97
:103DC000809FFF1F2C9DFF1F6A9DFF1FEA9DFF1F05
:103DD0008489FF1FABAAAA2A839FFF1F229DFF1F72
:103DE0000C9FFF1FEA9FFF1FE69FFF1F5C89FF1FBD
:103DF000914B1B78FBB1914B1B88012B00F07A860D
:103E0000022B00F07487032B01F0ED80042B01F0EE
:103E10008381052B01F0C183062B01F0E584072B7C
:103E200001F0C085082B01F01887092B01F091875C
:103E30000A2B01F06F87019B1B88002B00F0B882D2
:103E40007F4B1B78002B40F0AE827E4B7E4A198858
:103E500034680020012310602B6040E50135EDB28D
:103E6000022D86BF00230B700D701346FFF709B9B2
:103E70000398002101707549097800293EF4E3AFE9
:103E80006D4902910978002900F0578702980021B6
:103E90000170FEF7D8BF039B1B78002B7FF4B9ABF2
:103EA000029B1B78002B7FF4B4AB019B1988FFF7B2
:103EB000B6BB243B002BB8F8000040F3798498424D
:103EC0003EF43FAF9BB26248A8F800300123037074
:103ED000FEF737BF5F4B3878197805F059FED9E403
:103EE000DFF87081C0B298F8001005F051FEFFF7BE
:103EF000AABBC0B298F8001005F04AFEFFF77EB9E1
:103F00007F21402005F014FE5349544A3B680B6062
:103F10000021117043E5D8B298F8001005F038FE82
:103F20003B68AEE54E4BDFF858E11978FEF709BF64
:103F30004B2C40F346821834802CB8F80030494AA4
:103F4000A8BF8024A3427FF408AEFEF722BF99F8F1
:103F5000000005F041FE2188FFF761BB424B019351
:103F60001B88002B41F03687334B029346E6029BB9
:103F70001B78002B7FF428AB039B1B78002B7FF46E
:103F800048AB92E7FCF77EFB4CE6FCF77BFBC9E411
:103F9000FCF778FB19E5FCF775FBFFF72FBA4B1C14
:103FA000DBB2022B40F25B8200232B701346FFF73B
:103FB00068B87F20FFF7D8BA7F20FFF7FBB91E4F04
:103FC0001F4902974FF0000C81F800C0009F029932
:103FD0004FF0010E87F800E081F800C077E6234F2C
:103FE000387802F0DBFE224B1B78002B00F0458274
:103FF0003B887E2B00F241821E4CDFF888902268BD
:10400000D9F80010521A0F2A40F22E821A4A0133B0
:10401000108899B23980002800F04882C9B2C0B235
:1040200005F086FD154F226898F80030C9F8002089
:104030003B70FEF79ABD00BFEA9DFF1F029FFF1F66
:10404000409FFF1FE89DFF1F089DFF1F269DFF1F2C
:104050002C9DFF1FC19DFF1F309DFF1F8489FF1FE7
:10406000BF9FFF1F809FFF1F6A9DFF1F609DFF1F57
:10407000EB9FFF1F0C9FFF1FB09DFF1F229DFF1F87
:10408000859DFF1FCC9FFF1FDFF8B4A33868BAF8E7
:104090000030E44AE44CC31A82FB031ED917C1EB7B
:1040A0006E0101EB4101A3EB810303EB430354F8E1
:1040B000233018447F2840F390847F3882FB0032FD
:1040C000C317C3EB620303EB4303A0EB830073301E
:1040D000DFF87083DFF870B398F80010C0B205F015
:1040E00057FDBBF80030022B7FF6CFAB3968BAF82A
:1040F0000030CC4ACB1A82FB030ED817C0EB6E00FF
:1041000000EB4000A3EB800303EB430304EB8303CA
:10411000586808447F2840F358877F3882FB003274
:10412000C317C3EB620202EB4202A0EB82007330C2
:10413000C0B298F8001005F02BFDBBF80030032B3F
:104140007FF6A3AB3968BAF80030B64ACB1A82FBC7
:10415000030ED817C0EB6E0000EB4000A3EB80030A
:1041600003EB430304EB8304A06808447F2840F377
:1041700081817F3882FB0032C317C3EB620202EBFE
:104180004202A0EB8200733098F80010C0B205F034
:10419000FFFCFFF77ABBDFF8A8A299F80000BAF895
:1041A0000030A04AA04CC31A82FB031ED917C1EBF2
:1041B0006E0101EB4101A3EB810303EB430354F8D0
:1041C000233018447F2840F383847F3882FB0032F9
:1041D000C317C3EB620303EB4303A0EB830073300D
:1041E000DFF864B2C0B205F0F7FCBBF80030022B78
:1041F0007FF60AAA99F80010BAF80030894ACB1A5B
:1042000082FB030ED817C0EB6E0000EB4000A3EB5F
:10421000800303EB430304EB8303586808447F28BF
:1042200040F3D7867F3882FB0032C317C3EB6202AC
:1042300002EB4202A0EB82007330C0B205F0CCFC6E
:10424000BBF80030032B7FF6DFA999F80010BAF80D
:104250000030744ACB1A82FB030ED817C0EB6E00F5
:1042600000EB4000A3EB800303EB430304EB830468
:10427000A06808447F2840F3E9807F3882FB003241
:10428000C317C3EB620202EB4202A0EB8200733061
:10429000C0B205F0A1FCFFF7B7B90120FFF764B980
:1042A000DFF89CA15F49BAF800205F4C9A1A81FBA5
:1042B000020ED017C0EB6E0000EB4000A2EB8002B4
:1042C00002EB420254F8220018447F2840F3048491
:1042D000A0F17F0381FB0321DA17C2EB610000EB41
:1042E0004000A3EB80007330DFF85CB198F8001059
:1042F000C0B205F04DFCBBF80030022B50D9396834
:10430000BAF80030474ACB1A82FB030ED817C0EB2D
:104310006E0000EB4000A3EB800303EB430304EBD0
:104320008303586808447F2840F3C0867F3882FBA7
:104330000032C317C3EB620202EB4202A0EB820021
:104340007330C0B298F8001005F022FCBBF80030C2
:10435000032B25D93868BAF80030324AC31A82FBD9
:10436000031ED917C1EB6E0101EB4101A3EB8103E1
:1043700003EB430304EB8304A36818447F2868DD40
:104380007F3882FB0032C317C3EB620202EB4202AA
:10439000A0EB82007330C0B298F8001005F0F8FB73
:1043A0003B68FFF769BB0021402005F0C1FB4CE5ED
:1043B00099F8000005F010FC42E505F00DFCFFF750
:1043C00026B8243C002CB8F8003040F30686A342FF
:1043D0003EF4DFACA4B2154BA8F8004001221A70DD
:1043E000FEF7D7BC0120FEF7E5BF114B01931B88F8
:1043F000002B3FF4E6A8FFF7F6BB0E4A8342A8BFA6
:1044000003461360FEF7DCBE1446FFF79BBB0A4B66
:104410000A4C19886A2005F0E5FC98F800303B70DA
:10442000FEF7A3BBABAAAA2A682E01002C9DFF1F92
:104430006A9DFF1F089DFF1F609DFF1F0C9FFF1FB0
:104440003C9FFF1FC19DFF1F429DFF1FFCF71AF9F4
:104450001EE7FCF717F99EE7FCF714F970E42B70E0
:104460001346FEF70EBEDA4CDA4F98F800303B7078
:10447000FEF77BBBFCF706F986E6D74B1B78002BD3
:10448000F1D03B88D54F002BEDD0D14CDFF85C93B9
:104490002268D9F80010521A0F2AE5D9D04A013BF8
:1044A000108899B2398000287FF4B8ADC8B205F001
:1044B000DFFBB7E5DFF838A399F80000BAF8003061
:1044C000C84AC94CC31A82FB031ED917C1EB6E013F
:1044D00001EB4101A3EB810303EB430354F82330C9
:1044E00018447F2840F3FA837F3882FB0032C317D9
:1044F000C3EB620303EB4303A0EB83007330DFF8ED
:10450000F4B2C0B205F068FBBBF80030022B7FF6B6
:104510007BA899F80010BAF80030B24ACB1A82FB97
:10452000030ED817C0EB6E0000EB4000A3EB800336
:1045300003EB430304EB8303586808447F2840F3EC
:10454000E7857F3882FB0032C317C3EB620303EBBE
:104550004303A0EB83007330C0B205F03DFBBBF812
:104560000030032B7FF650A899F80010BAF80030FD
:104570009C4ACB1A82FB030ED817C0EB6E0000EBEF
:104580004000A3EB800303EB430304EB8304A06828
:1045900008447F287FF75AAF7F3882FB0032C31769
:1045A000C3EB620303EB4303A0EB830073306FE6BE
:1045B000DFF83CA23868BAF800308A4A8A4CC31A3D
:1045C00082FB031ED917C1EB6E0101EB4101A3EB86
:1045D000810303EB430354F8233018447F2840F34E
:1045E00080837F3882FB0032C317C3EB620303EB87
:1045F0004303A0EB83007330DFF8FC81DFF8F4B1F4
:1046000098F80010C0B205F0C3FABBF80030022BD6
:104610007FF63BA93968BAF80030724ACB1A82FBA0
:10462000030ED817C0EB6E0000EB4000A3EB800335
:1046300003EB430304EB8303586808447F2840F3EB
:1046400074857F3882FB0032C317C3EB620303EB30
:104650004303A0EB83007330C0B298F8001005F05C
:1046600097FABBF80030032B7FF60FA93868BAF829
:1046700000305C4AC31A82FB031ED917C1EB6E01DE
:1046800001EB4101A3EB810303EB430304EB830440
:10469000A36818447F287FF7EDAE7F3882FB003295
:1046A000C317C3EB620303EB4303A0EB8300733038
:1046B0006AE5DFF83CA14B49BAF800204A4C9A1A47
:1046C00081FB020ED017C0EB6E0000EB4000A2EBA6
:1046D000800202EB420254F8220018447F2840F383
:1046E0000383A0F17F0381FB0321DA17C2EB610092
:1046F00000EB4000A3EB80007330DFF8F8B098F8CF
:104700000010C0B205F044FABBF80030022B7FF66F
:1047100047AE3968BAF80030324ACB1A82FB030E32
:10472000D817C0EB6E0000EB4000A3EB800303EB57
:10473000430304EB8303586808447F2840F3F9845B
:104740007F3882FB0032C317C3EB620303EB4303E2
:10475000A0EB83007330C0B298F8001005F018FA8F
:10476000BBF80030032B7FF61BAE3868BAF8003078
:104770001C4AC31A82FB031ED917C1EB6E0101EB61
:104780004101A3EB810303EB430304EB8304A36820
:1047900018447F287FF75DAE7F3882FB0032C31755
:1047A000C3EB620303EB4303A0EB83007330F2E53A
:1047B00001283EF4C6AA0123FFF785BB4FF47A43D4
:1047C000013BFDD199F8000005F006FAFFF76DB83E
:1047D0000C9FFF1F229DFF1FEA9FFF1F609DFF1F71
:1047E000B09DFF1FABAAAA2A60310100CC9FFF1F1A
:1047F0003C9FFF1F429DFF1FC19DFF1FDFF8E8A2E6
:104800003868BAF80030B64AB64CC31A82FB031EA9
:10481000D917C1EB6E0101EB4101A3EB810303EB5F
:10482000430354F8233018447F2840F3DB817F385A
:1048300082FB0032C317C3EB620202EB4202A0EB21
:1048400082007330DFF8A482DFF8A4B298F8001079
:10485000C0B205F09DF9BBF80030022B7FF615A819
:104860003868BAF800309E4AC31A82FB0321DA176F
:10487000C2EB610202EB4202A3EB820303EB4303B0
:1048800004EB83035B6818447F2840F31C847F3863
:104890000C2290FBF2F302FB13007330C0B298F8C5
:1048A000001005F075F9BBF80030032B7EF6EDAF74
:1048B0003868BAF800308A4AC31A82FB0321DA1733
:1048C000C2EB610202EB4202A3EB820303EB430360
:1048D00004EB8304A36818447F287FF7CBAD7F38AF
:1048E0000C2290FBF2F302FB130073304CE4DFF870
:1048F000F8A199F80000BAF80030794A794CC31A47
:1049000082FB031ED917C1EB6E0101EB4101A3EB42
:10491000810303EB430354F8233018447F2840F30A
:1049200064817F3882FB0032C317C3EB620202EB63
:104930004202A0EB82007330DFF8B4B1C0B205F0E0
:104940004BF9BBF80030022B7EF65EAE99F8000002
:10495000BAF80030624AC31A82FB0321DA17C2EBAD
:10496000610202EB4202A3EB820303EB430304EB7D
:1049700083035B6818447F2840F39C837F380C22B4
:1049800090FBF2F302FB13007330C0B205F024F980
:10499000BBF80030032B7EF637AE99F80000BAF86A
:1049A00000304F4AC31A82FB0321DA17C2EB6102BF
:1049B00002EB4202A3EB820303EB430304EB830409
:1049C000A36818447F287FF741AD7F380C2290FB05
:1049D000F2F302FB130073305AE4FBF753FEFFF7C8
:1049E00077BBDFF804A13E49BAF800203D4C9A1A83
:1049F00081FB020ED017C0EB6E0000EB4000A2EB73
:104A0000800202EB420254F8220018447F2840F34F
:104A1000EF80A0F17F0381FB0321DA17C2EB610174
:104A200001EB4101A3EB81007330DFF8C4B098F8CB
:104A30000010C0B205F0ACF8BBF80030022B7FF6D6
:104A4000AFAC3868BAF80030254AC31A82FB03219C
:104A5000DA17C2EB610202EB4202A3EB820303EB23
:104A6000430304EB83035B6818447F2840F33283DD
:104A70007F380C2290FBF2F302FB13007330C0B2BC
:104A800098F8001005F084F8BBF80030032B7FF68F
:104A900087AC3868BAF80030114AC31A82FB032188
:104AA000DA17C2EB610202EB4202A3EB820303EBD3
:104AB000430304EB8304A36818447F287FF7C9AC41
:104AC0007F380C2290FBF2F302FB1300733062E498
:104AD000FBF7D8FDFFF784BBFBF7D4FD04E400BF70
:104AE000ABAAAA2AF03101003C9FFF1FC19DFF1F06
:104AF000429DFF1FDFF83CA399F80000BAF8003090
:104B0000C44AC54CC31A82FB0317D917C1EB67010E
:104B100001EB4101A3EB810303EB430354F8233082
:104B200018447F286ADD7F3882FB0032C317C3EB4D
:104B3000620202EB4202A0EB82007330DFF8F8B2AF
:104B4000C0B205F049F8BBF80030022B7FF673A91C
:104B500099F80000BAF80030AE4AC31A82FB03216C
:104B6000DA17C2EB610202EB4202A3EB820303EB12
:104B7000430304EB83035B6818447F2840F3AD8252
:104B80007F380C2290FBF2F302FB13007330C0B2AB
:104B900005F022F8BBF80030032B7FF64CA999F8FA
:104BA0000000BAF800309B4AC31A82FB0321DA17CF
:104BB000C2EB610202EB4202A3EB820303EB43036D
:104BC00004EB8304A36818447F2814DD7F380C228B
:104BD00090FBF2F302FB13007330C0B204F0FCFF51
:104BE000FFF729B9FBF74EFD2CE6FBF74BFDA3E6DB
:104BF000FBF748FD19E7FBF745FDEEE7FBF742FD44
:104C00009CE7DFF830A299F80000BAF80030814A3A
:104C1000824CC31A82FB031ED917C1EB6E0101EB54
:104C20004101A3EB810303EB430354F82330184401
:104C30007F28DADD7F3882FB0032C317C3EB6203C3
:104C400003EB4303A0EB8300733075E6DFF8E4A1C8
:104C50003868BAF800306F4A704CC31A82FB031EE2
:104C6000D917C1EB6E0101EB4101A3EB810303EB0B
:104C7000430354F8233018447F28B3DD7F3882FB88
:104C80000032C317C3EB620303EB4303A0EB8300C3
:104C90007330D7E5DFF89CA15E49BAF800205F4C7D
:104CA0009A1A81FB020ED017C0EB6E0000EB400099
:104CB000A2EB800202EB420254F8220018447F2843
:104CC00096DDA0F17F0381FB0321DA17C2EB6100BF
:104CD00000EB4000A3EB80007330A6E6FBF7D2FCAC
:104CE0000DE4FBF7CFFC87E4FBF7CCFC05E5DFF830
:104CF00044A199F80000BAF80030464A484CC31A5B
:104D000082FB0317D917C1EB670101EB4101A3EB4C
:104D1000810303EB430354F8233018447F287FF7C3
:104D20006DAF7F3882FB0032C317C3EB620303EB26
:104D30004303A0EB8300733000E73A4800903A4801
:104D40003A490390FEF773B8DFF8E8A03868BAF87C
:104D50000030304A364CC31A82FB0321DA17C2EB0B
:104D6000610202EB4202A3EB820303EB430354F81C
:104D7000233018447F2840F3A0817F380C2290FB19
:104D8000F2F302FB13007330DFF8B080DFF8A8B055
:104D900098F80010C0B204F0FBFEBBF80030022B04
:104DA0001AD93868BAF800300C22C11A91FBF2F314
:104DB00002FB131302FB03435B6818447F2840F394
:104DC00052847F3890FBF2F302FB13007330C0B2C1
:104DD00098F8001004F0DCFEBBF80030032B7EF6E0
:104DE00054ADBAF8003038680C22C11A91FBF2F3C6
:104DF00002FB131302FB0344A36818447F287FF7C8
:104E000039AB7F3890FBF2F302FB13007330FFF7EE
:104E1000BBB900BFABAAAA2A682E0100D42A0100A0
:104E200060310100949FFF1F059DFF1F409FFF1FE2
:104E3000283001003C9FFF1F429DFF1FC19DFF1FA7
:104E4000DFF860A399F80000BAF80030CC4ACD4CE6
:104E5000C31A82FB0321DA17C2EB610202EB4202A2
:104E6000A3EB820303EB430354F8233018447F2859
:104E700040F32D817F380C2290FBF2F302FB1300EC
:104E80007330DFF824B3C0B204F0A6FEBBF80030E4
:104E9000022B19D999F80000BAF800300C22C11A77
:104EA00091FBF2F302FB131302FB03435B6818440C
:104EB0007F2840F390837F3890FBF2F302FB1300CE
:104EC0007330C0B204F088FEBBF80030032B7EF6CE
:104ED0009BABBAF8003099F800000C22C11A91FB84
:104EE000F2F302FB131302FB0344A36818447F2868
:104EF0007FF7ACAA7F3890FBF2F302FB130073300C
:104F0000FFF7C6B9DFF89CA29D49BAF800209D4C76
:104F10009A1A81FB0210D117C1EB600101EB41012C
:104F2000A2EB810202EB420254F8220018447F28CF
:104F300040F3C680A0F17F030C2093FBF0F200FB4E
:104F400012307330DFF860B298F80010C0B204F08D
:104F50001FFEBBF80030022B1AD93868BAF80030AF
:104F60000C22C11A91FBF2F302FB131302FB034361
:104F70005B6818447F2840F32B837F3890FBF2F363
:104F800002FB13007330C0B298F8001004F000FE6A
:104F9000BBF80030032B7FF603AABAF8003038685C
:104FA0000C22C11A91FBF2F302FB131302FB034420
:104FB000A36818447F287FF74CAA7F3890FBF2F350
:104FC00002FB13007330FFF7E6B9FBF75BFBFFF75B
:104FD000AFB8FBF757FBFFF730B9012B3DF4D9AE63
:104FE0000124FFF7F8B9DFF8BCA199F80000BAF87E
:104FF0000030634A644CC31A82FB0321DA17C2EB08
:10500000610202EB4202A3EB820303EB430354F879
:10501000233018447F2846DD7F380C2290FBF2F3C2
:1050200002FB13007330DFF880B1C0B204F0D4FD8E
:10503000BBF80030022B19D999F80000BAF80030FB
:105040000C22C11A91FBF2F302FB131302FB034380
:105050005B6818447F2840F38F807F3890FBF2F321
:1050600002FB13007330C0B204F0B6FDBBF8003091
:10507000032B7EF6E0AEBAF8003099F800000C225F
:10508000C11A91FBF2F302FB131302FB0344A36862
:1050900018447F287FF7AFAD7F3890FBF2F302FB17
:1050A0001300733099E5FBF7EDFABCE7FBF7EAFA7A
:1050B000FFF747B9FBF7E6FA67E4FBF7E3FA63E6C5
:1050C000FBF7E0FA3EE7FBF7DDFAFFF7E7BBFBF79C
:1050D000D9FAD6E6FBF7D6FAD1E4FBF7D3FA56E5D0
:1050E000DFF8C0A03868BAF80030254A274C32E60D
:1050F000DFF8B0A099F80000BAF80030204A234C3D
:10510000A6E6029B1B78002B7EF45EAAFEF781BA0E
:10511000FBF7B8FAFFF720BADFF888A099F800008B
:10512000BAF80030164A1A4C65E7FBF7ABFAFFF7FE
:1051300093BAFBF7A7FAFFF70EBBDFF868A0104998
:10514000BAF80020114CE3E6124B1B78002B00F05C
:10515000C282114B1B78002B7DF41BAE0F4B1B78CA
:10516000002B3DF416AEB8F800300D490A33A8F80C
:1051700000300A70FDF70DBEFBF784FA73E700BF3D
:10518000ABAAAA2A28300100F0310100E432010064
:10519000D42A0100E79FFF1FE89FFF1FE99FFF1F21
:1051A0002C9DFF1F3C9FFF1F429DFF1FA44C228888
:1051B000002A00F02183A349DFF89CB20988BBF8DC
:1051C00000000331884227DD9F48A0490088B1F8DC
:1051D00000E0DFF87CC2181A0C2190FBF1F901FB0A
:1051E00019004FF0900909FB0EFE01FB00E06FF083
:1051F0000B0E5CF8000003440EFB02307F2840F3E6
:10520000F1847F3890FBF1F301FB13007330C0B2DF
:1052100098F8001004F0BCFCBBF80020238813446D
:10522000022B23DD884B894A38681B88B2F800C0FE
:10523000DFF81CE2C31A0C2193FBF1F201FB1232DE
:10524000902303FB0CF301FB023373445B681844A7
:105250007F2840F351857F3890FBF1F301FB130069
:105260007330C0B298F8001004F092FCBBF8002034
:1052700023881344032B23DD734B744A38681B883F
:10528000B2F800C0DFF8C8E1C31A0C2193FBF1F2B9
:1052900001FB1232902303FB0CF301FB0233734436
:1052A0009B6818447F2840F32B857F3890FBF1F3EF
:1052B00001FB13007330C0B298F8001004F068FCD2
:1052C000BBF8002023881344042B7FF769A85D4BAB
:1052D0001B88012B7FF464A83A68A2F10C007F2898
:1052E0007FF7B7A88B3A0C2092FBF0F300FB13205A
:1052F0007330FFF750B8524C2388002B40F0BC822B
:10530000DFF854B15049514A0988D7F80080B2F803
:1053100000E04F48C1EB080C0C229CFBF2F102FBB1
:1053200011C14FF0900C0CFB0EFE02FB01E16FF07F
:105330000B0E405880440EFB03807F2840F31784F7
:10534000A0F17F0393FBF2F002FB10307330414B6E
:10535000C0B2197804F01CFCBBF800202388134469
:10536000022B23DD384A394B11883868B3F800C066
:10537000DFF8DCE0411A0C2291FBF2F302FB13117F
:10538000902303FB0CF302FB013373445B68184466
:105390007F2840F3FD847F3890FBF2F302FB13007B
:1053A00073302C4BC0B2197804F0F2FBBBF800202C
:1053B00023881344032B23DD234A244B11883868A8
:1053C000B3F800C0DFF888E0411A0C2291FBF2F339
:1053D00002FB1311902303FB0CF302FB0133734414
:1053E0009B6818447F2840F377847F3890FBF2F362
:1053F00002FB13007330174BC0B2197804F0C8FBDE
:10540000BBF8002023881344042B7EF73EAA0D4BE3
:105410001B88012B7EF439AA3A68A2F10C007F2880
:1054200040F356818B3A0C2092FBF0F300FB1320E3
:105430007330084BC0B2197804F0AAFBFEF725BA06
:10544000C89DFF1F5E9DFF1F3C9FFF1FEE9EFF1F1D
:10545000642B0100C19DFF1F429DFF1FCB4C238881
:10546000002B40F0CC81DFF854B3C949C94A098800
:1054700099F80000B2F800E0DFF84483C1EB000CBB
:105480000C229CFBF2F102FB11C14FF0900C0CFBC3
:105490000EFE02FB01E16FF00B0E58F801100844FC
:1054A0000EFB03007F2840F3A183A0F17F0393FB51
:1054B000F2F002FB10307330C0B204F08DFBBBF889
:1054C000002023881344022B22DDB14AB14B1188FE
:1054D00099F80000B3F800C0DFF8E4E2411A0C22AA
:1054E00091FBF2F302FB1311902303FB0CF302FB7D
:1054F000013373445B6818447F2840F3F1837F389D
:1055000090FBF2F302FB13007330C0B204F064FBB3
:10551000BBF8002023881344032B22DD9C4A9D4BBB
:10552000118899F80000B3F800C0DFF894E2411A3E
:105530000C2291FBF2F302FB1311902303FB0CF3FB
:1055400002FB013373449B6818447F2840F3CE83E9
:105550007F3890FBF2F302FB13007330C0B204F00B
:105560003BFBBBF8002023881344042B7EF74CA898
:10557000894B1B88012B7EF447A899F80020A2F1E3
:105580000C007F287EF762AF8B3A0C2092FBF0F381
:1055900000FB13207330FEF77BBEDFF8F4A199F80F
:1055A0000000BAF800307D4CC11A0C2291FBF2F3D6
:1055B00002FB131302FB03F3E35818447F287FF721
:1055C00072AD7F3890FBF2F302FB130073302AE5D3
:1055D000FBF758F8D7E4FBF755F872E4704B1A88DC
:1055E000182A13D03B681344A3F118007F2840F316
:1055F000D3830C20973B93FBF0F200FB123303F1B3
:105600007300684BC0B2197804F0C2FA664B674960
:105610001A78022A94BF013200221A701A7831F8DF
:105620001200182810D10424022A02F10100C2B28B
:1056300088BF002231F81200182804D1013CF3D1B0
:105640001A70FEF722B91A703B680344A3F11800E0
:105650007F283DDD0C20973B93FBF0F200FB1233DB
:1056600003F17300E5E6FBF70DF8FFF7B0BB4C4B19
:105670001B88182B12D099F800201344A3F11800AE
:105680007F2840F341830C20973B93FBF0F200FB13
:10569000123303F17300C0B204F09EFA424A434B46
:1056A000127833F81230182B3DF4AEAF99F8002081
:1056B0001344A3F118007F287EF7C8AE0C20973B57
:1056C00093FBF0F200FB123303F17300FEF7E0BD31
:1056D000FAF7D8FFADE6364B1B78002B7DF4FCAF14
:1056E000344B1B78002B3DF454ABB8F800303249F2
:1056F0000133A8F800300A70FDF74BBB2C4B1B7828
:10570000002B7DF446AB2B4B1B78002B3DF441ABBB
:10571000B8F800302849013BA8F800300A70FDF7BE
:1057200038BB1F4A1288182A12D01344A3F118005C
:105730007F2840F3DE820C20973B93FBF0F200FBC6
:10574000123303F17300C0B298F8001004F020FA8D
:10575000154B16491A78022A94BF013200221A709A
:105760001A7831F8120018282DD10424022A02F1E7
:105770000100C2B288BF002231F81200182821D1DE
:10578000013CF3D11A703B68FEF776B9C89DFF1F44
:105790003C9FFF1FEE9EFF1F5E9DFF1F28300100F4
:1057A000929FFF1FC19DFF1FBC89FF1F589FFF1FB6
:1057B000E89FFF1FE99FFF1F2C9DFF1F429DFF1FBA
:1057C000642B01001A703B680344A3F118007F2882
:1057D0007EF73FAE0C20973B93FBF0F200FB1233B9
:1057E00003F17300FEF7D7BDDFF82CA399F8000092
:1057F000BAF80030BF4CD7E6DFF82CB3E4E4BE4A79
:10580000DFF824B31288BBF80010033291427FF70F
:1058100056AE2AE6B94A1288182A12D01344A3F1C8
:1058200018007F2840F373820C20973B93FBF0F223
:1058300000FB123303F17300C0B298F8001004F0BB
:10584000A7F9AF4BAF491A78022A94BF0132002260
:105850001A701A7831F812001828B4D10424022AD8
:1058600002F1010294BFD2B2002231F812001828CE
:10587000A8D1013CF3D185E79F4ADFF8ACB212888A
:10588000BBF80010033291427FF766AD3AE59B4BBF
:105890001A88182A13D03B681344A3F118007F28F4
:1058A00040F30C820C20973B93FBF0F200FB123389
:1058B00003F17300944BC0B2197804F069F9904B6E
:1058C00090491A78022A94BF013200221A701A787D
:1058D00031F8120018287FF4B7AE0424022A02F12E
:1058E000010294BFD2B2002231F8120018287FF4CE
:1058F000AAAE013CF2D11A70FDF7C7BF7F4B1B88DF
:10590000182B12D099F800201344A3F118007F2817
:1059100040F3E9810C20973B93FBF0F200FB12333C
:1059200003F17300C0B204F057F9754A754B127851
:1059300033F81230182B7FF4B9AEFDF765BE734B08
:1059400001227F2107201A8004F0F2F87F210B202A
:1059500004F0EEF8FDF7EBBE6D4B04227F2107202B
:105960001A8004F0E5F800210B2004F0E1F8FDF7BF
:10597000D7BE674B02227F2107201A8004F0D8F897
:105980007F210B2004F0D4F8FDF7C5BE604B002149
:1059900007201C8004F0CCF87F210B2004F0C8F80D
:1059A000FDF7B4BE5B4C2388002B40F08A81DFF802
:1059B00078B1594999F80000584A09881788DFF8E2
:1059C00060E1411A0C2291FBF2FC02FB1C114FF02A
:1059D000900C0CFB07F702FB01716FF00B075EF8F0
:1059E0000110014407FB03107F2840F3D8817F3862
:1059F00090FBF2F302FB13007330C0B204F0ECF83A
:105A0000BBF8002023881344022B21DD424B434A7C
:105A100099F800001B88B2F800E0414FC31A0C212E
:105A200093FBF1F201FB1232902303FB0EF301FB17
:105A300002333B445B6818447F2840F3C8817F38B9
:105A400090FBF1F301FB13007330C0B204F0C4F813
:105A5000BBF8002023881344032B21DD2E4B2F4A53
:105A600099F800001B88B2F800E02D4FC31A0C21F2
:105A700093FBF1F201FB1232902303FB0EF301FBC7
:105A800002333B449B6818447F2840F38B817F3866
:105A900090FBF1F301FB13007330C0B204F09CF8EB
:105AA000BBF8002023881344042B7EF7C4A9124BB3
:105AB0001B88012B7EF4BFA999F80020A2F10C00ED
:105AC0007F287FF798A88B3A0C2092FBF0F300FB1D
:105AD00013207330FFF781B8124B00227F2107207B
:105AE0001A8004F025F87F210B2004F021F8FDF73F
:105AF00026BE00BFE43201005E9DFF1F569DFF1FC2
:105B0000BC89FF1FD09EFF1FC19DFF1FDA9DFF1F95
:105B1000349FFF1FC89DFF1F3C9FFF1FEE9EFF1F6E
:105B2000642B0100249DFF1F429DFF1FAB4B1B8870
:105B3000182B12D099F800201344A3F118007F28E5
:105B400040F33C810C20973B93FBF0F200FB1233B7
:105B500003F17300C0B204F03FF8A14AA14B1278E0
:105B600033F81230182B7FF4A1ADFDF74DBDFAF7D5
:105B700089FDFFF7ECBB994B1A88182A13D03B68B4
:105B80001344A3F118007F2840F31B810C20973B9E
:105B900093FBF0F200FB123303F17300924BC0B29F
:105BA000197803F0F5FF8E4B8E491A78022A94BFBC
:105BB000013200221A701A7831F8120018287FF486
:105BC00043AD0424022A02F1010294BFD2B20022A2
:105BD00031F8120018287FF436AD013CF2D11A706A
:105BE000FDF753BEFAF74EFDFFF711BBFAF74AFD7A
:105BF00062E47A4A1288182A12D01344A3F11800DA
:105C00007F2840F3D2800C20973B93FBF0F200FBFF
:105C1000123303F17300C0B298F8001003F0B8FF1C
:105C20006F4B70491A78022A94BF013200221A7011
:105C30001A7831F8120018287FF4C5AD0424022A1E
:105C400002F1010294BFD2B2002231F812001828EA
:105C50007FF4B8AD013CF2D194E5644B1B88182B5E
:105C600012D099F800201344A3F118007F2840F3C4
:105C7000AB800C20973B93FBF0F200FB123303F157
:105C80007300C0B203F0A8FF554A594B127833F89D
:105C90001230182B3EF4CFA899F800201344A3F13A
:105CA00018007F287EF7A7AF0C20973B93FBF0F2FC
:105CB00000FB123303F17300FEF78FBFFAF7E2FC2B
:105CC000F8E54C4ADFF83CB11288BBF8001003320B
:105CD00091427FF795AE6CE6FAF7D4FCFFF78BBBE9
:105CE000FAF7D0FC11E4FAF7CDFC1BE6FAF7CAFC90
:105CF00034E4FAF7C7FC26E5FAF7C4FCFFF7B1BABB
:105D0000FAF7C0FCFFF7D7BAFAF7BCFCC3E4FAF71E
:105D1000B9FC91E5314B1B88182B11D099F8002064
:105D20001344A3F118007F2842DD0C20973B93FB1E
:105D3000F0F200FB123303F17300C0B203F04CFF2A
:105D4000274A284B127833F81230182BA4D1FEF7CB
:105D500072B8294B1B88182B11D099F800201344D6
:105D6000A3F118007F2826DD0C20973B93FBF0F26F
:105D700000FB123303F17300C0B203F02DFF184A89
:105D80001E4B127833F81230182B85D1FEF753B81A
:105D9000FAF778FCFFF705BBFAF774FC31E4FAF781
:105DA00071FC2AE6FAF76EFC77E6FAF76BFC32E74D
:105DB000FAF768FCC1E7FAF765FCDDE7FAF762FC81
:105DC000C8E6FAF75FFCE9E6FAF75CFC59E7FAF790
:105DD00059FC3AE60A4B0293FDF705BF589DFF1F99
:105DE000BC89FF1FD89EFF1FC19DFF1F929FFF1FF1
:105DF000589FFF1F5E9DFF1F569DFF1FD09EFF1FD8
:105E0000EA9DFF1F429DFF1F38B507F09FFE0E4819
:105E100005F0D6FD0D4805F0D3FD0D4805F0D0FD89
:105E200000234FF07E5201210A48FAF71FFB0A4B6C
:105E30000A4A0B49802400251C7118461D60BDE8E4
:105E400038400BF087BC00BF409DFF1F749DFF1FB3
:105E5000E09DFF1F109FFF1FA09FFF1F1C89FF1FBA
:105E60002906000010B50446A4206368198803F0D1
:105E7000B9FFE368A6201988BDE8104003F0B2BF5F
:105E800043682A20198803F0ADBF00BF10B504464F
:105E900022206368198803F0A5FFE368242019888D
:105EA000BDE8104003F09EBF10B504460A206368A9
:105EB000198803F097FFE3680C201988BDE81040AB
:105EC00003F090BF10B5044606206368198803F0FC
:105ED00089FFE36808201988BDE8104003F082BFFD
:105EE00010B5044602206368198803F07BFFE3685D
:105EF00004201988BDE8104003F074BF70B50E4C43
:105F000084B0122504220123064603900293204602
:105F10008DE824001423102106F056FF06220923E1
:105F2000029303960195204600921423102106F057
:105F30004BFF04B070BD00BF1CA0FF1FF8B5B04CF4
:105F4000B4F90030032B00F01281002B6AD0022B31
:105F500000F08A80052B00F0B580012B00F0DD8079
:105F6000042B00D0F8BDA74FA74E00254FF4AF7407
:105F7000E9B2A64805F08CFD57F8043BC3F59673CB
:105F800000FB03F086FB0023C017C0EB63108442C4
:105F900005F10105A8BF0446062DE9D19C4F9A4E94
:105FA0000025E9B29B4805F073FD57F8043BC3F5A3
:105FB000967300FB03F086FB0023C017C0EB631051
:105FC000844205F10105A8BF04460C2DE9D1924F8A
:105FD0008D4E0025E9B2914805F05AFD57F8043B73
:105FE000894AC3F5967300FB03F086FB0013C017C4
:105FF000C0EB6310844205F10105A8BF04460C2DD7
:10600000E8D1A4F11401312900F3A38040F26C72AD
:1060100032218348834B01801A602A20BDE8F84072
:1060200003F0E0BE0E2007F0F5FC40F6FF71C8302B
:106030008842A8BF084620EAE07000F2DC5283B232
:106040008A42794D794EA8BF0A460220194633800C
:106050002A8003F0C7FE2988042003F0C3FEB4F9A8
:106060000030022B7FF476AF012008F0EFFD0546EB
:10607000002008F0EBFDA842B8BF284600F1C80197
:10608000B1F5FA7FC0F2B480B1F57A6FA8BF4FF4D2
:106090007A6101F54873B3F57A6FA8BF4FF47A635C
:1060A0009BB289B2624A634D11800A202B8003F0B3
:1060B00099FE29880C2003F095FEB4F90030052BD9
:1060C0007FF44BAF0F2008F0C1FDC0F53F630433F0
:1060D000B3F5AF6FC0F28980B3F5FA6FA8BF4FF484
:1060E000FA6399B2544BC0F54360B0F5AF6F1980B5
:1060F00061DBB0F5FA6FA8BF4FF4FA6083B24F4D81
:10610000A4202B8003F06EFE2988A62003F06AFEEF
:10611000B4F90030012B7FF423AF152007F07AFC8F
:1061200000F59671B1F52F7F4DDB41F25C2399426A
:1061300063DC434A00F5617089B2B0F52F7F1180AE
:10614000B8BF4FF42F7344DB8342A8BF03469BB212
:106150003FE040F23A73A4F5B97403FB04F482FB08
:106160000432E417A4EB621289B2323251E71020F4
:1061700008F06CFDC830B0F5FA7F1FDBB0F57A6F20
:106180000146A8BF4FF47A6101F51673B3F57A6F33
:10619000A8BF4FF47A639BB289B22A4A2A4D118074
:1061A00022202B8003F01EFE2988242003F01AFEF3
:1061B000B4F90030C9E64FF4AF63A0E740F24C43B6
:1061C0004FF4FA71E9E740F214534FF42F711C4A6F
:1061D00011801E4D06202B8003F004FE2988082024
:1061E00003F000FEB4F90030BAE64FF4AF6179E78E
:1061F00040F214534FF4FA7154E71946E7E700BF31
:10620000F69FFF1F4C8AFF1FB5814E1B409DFF1F4D
:106210001C8AFF1F749DFF1F2C89FF1FE09DFF1F1D
:10622000AC9FFF1F088AFF1FB29FFF1FE89DFF1F43
:10623000489FFF1F549DFF1FEC9DFF1F689FFF1F7E
:106240008E9DFF1FFC9EFF1FF89EFF1F7C9FFF1F60
:106250002DE9F041224D82B0012602B284B20092B3
:10626000284601967823192106F0F4FC04F10C026B
:1062700012B28DE844002846A7197823192104F1A9
:10628000020806F0E7FC3FB20FFA88F819233A46F5
:10629000284619460196CDF8008006F0DBFC7823ED
:1062A0003A4628461946CDF80080019604F10A07BF
:1062B0000B3406F0CFFC3FB224B278233A4628468E
:1062C00019468DE8500006F0C5FC192300943A46A3
:1062D00001962846194606F0BDFC02B0BDE8F081E3
:1062E0001CA0FF1F30B583B000230C4605B20093FD
:1062F00026225B231C210C4806F0FCF929460123C9
:106300002622094805F006FD002C24B205DB2146B3
:1063100001232622044805F0FDFC044A044B1580A5
:106320001C8003B030BD00BF1CA0FF1F668AFF1F8A
:10633000688AFF1F2DE9F041BB4C237882B01BB166
:10634000BA4B4FF6FF721A80B94BB3F90030CBB994
:10635000B84AB64B1068B3F9002080F30C005B23F9
:1063600003FB00F000131C3082424BD04FF0FF3192
:10637000FFF7B8FFB04806F021FA0023237002B0FF
:10638000BDE8F081012B1BD0022B5AD0032B3FD04C
:10639000042B00F09980052BEFD10F2008F056FC5C
:1063A000C0F53B600830B0F5AF6F48DBB0F5FA6F71
:1063B000A8BF4FF4FA60A0F5AF625B239F4835E0B9
:1063C0009F4B1B78002B75D0152007F023FB9D4BAE
:1063D0001860B0F52F7F32DB41F25C239842A8BFF2
:1063E0001846A0F52F735B22974802FB03F380FB4E
:1063F0000320DB17C3EBA0201C308C4BB3F900301B
:106400008342B3D1914BB3F900300133AED1B4E73D
:106410008F4B1B68B3F5FA7F11DBB3F57A6FA8BF1A
:106420004FF47A638B48A3F5FA725B2303FB02F304
:1064300080FB0320DB17C3EB20201C30DDE71C2092
:10644000DBE7854B1B68B3F5FA7F3BDBB3F57A6F6F
:10645000A8BF4FF47A63A3F5FA727E485B2303FB6F
:1064600002F380FB0320DB17C3EB20201C307B4BA7
:106470001B68B3F5FA7F23DBB3F57A6FA8BF4FF43F
:106480007A63A3F5FA7273495B2303FB02F381FB82
:106490000321DB17C3EB21211C31644BB3F900301E
:1064A00083427FF465AF694BB3F900308B427FF4D0
:1064B0005FAF62E7112008F0C9FB624B186088E704
:1064C0001C21EAE71C20D2E7252200258DE82400C4
:1064D00076231C215848624E624FDFF8A08106F0F7
:1064E000B9FB16E0B0F5AF7FA8BF4FF4AF703238FC
:1064F00002FB00F088FB0031C017C0EB61111C31BA
:1065000009B201231D4425224B4805F003FC0C2D44
:1065100014D0E9B2544805F0BBFA56F8043BC3F571
:10652000967300FB03F087FB0013C017C0EB6310EA
:1065300031284FF05B02D5DC1C21E2E72622002542
:106540008DE8240076231C213B48484E454FDFF858
:106550002C8106F07FFB16E0B0F5AF7FA8BF4FF4AB
:10656000AF70323802FB00F088FB0031C017C0EB7F
:1065700061111C3109B201231D4426222E4805F069
:10658000C9FB0C2D14D0E9B2394805F081FA56F850
:10659000043BC3F5967300FB03F087FB0013C017A1
:1065A000C0EB631031284FF05B02D5DC1C21E2E721
:1065B000272200258DE8240076231C211E482D4E1D
:1065C000284FDFF8B88006F045FB17E0B0F5AF7F45
:1065D000A8BF4FF4AF70323802FB00F088FB0031E7
:1065E000C017C0EB61111C3109B201231D442722E1
:1065F000114805F08FFB062D3FF4BCAEE9B21E48F2
:1066000005F046FA56F8043BC3F5967300FB03F019
:1066100087FB0013C017C0EB631031284FF05B02FB
:10662000D4DC1C21E1E700BFF09FFF1F668AFF1F3B
:10663000F69FFF1F4C9FFF1F1CA0FF1F37800B6D95
:10664000049FFF1F109DFF1FD3058541688AFF1F10
:10665000649DFF1F011FB812709DFF1F349DFF1F17
:106660001C8AFF1FB5814E1B749DFF1F2C89FF1FC5
:10667000E09DFF1F4C8AFF1F409DFF1F4B48371BAB
:106680002DE9F041044682B071482768E56805F0BD
:1066900089FF1120FFF7DCFD012619234FF02808A0
:1066A000194624226A480196CDF8008006F0D2FAF5
:1066B00078231946242266480196CDF8008006F01A
:1066C000C9FA3146624806F05BFE02221921604891
:1066D00006F052FE38460BF013FE394602465C487F
:1066E00006F0E4FF5A4806F0F7FF1422002158484C
:1066F00006F042FE03225749554806F0D7FF54489A
:1067000006F0EAFF23220021514806F035FE03225D
:1067100051494F4806F0CAFF4D4806F0DDFF7DB1F4
:106720002F20FFF795FD32220021494806F024FE74
:1067300003224A49464806F0B9FF454806F0CCFF17
:106740000123474A18461370FFF7D8FB2189638954
:1067500062685B1A5C2B128854DD521A02EB42020B
:10676000C2EB4212013392FBF3F31B333D4A38482C
:10677000138001261A221BB28DE844001946142208
:1067800006F068FA002D4FD0218A638AE2685B1A0E
:106790005C2B12883EDC511A5C2202FB01F292FB58
:1067A000F3F31B33304A2A48138001251BB23822E9
:1067B00019468DE82400322206F04CFA40230022CC
:1067C00009218DE806002248194606F011FA2946EB
:1067D0001F4806F0D5FD022244211D4806F0CCFDDD
:1067E00063681B48198806F0C7FF2A461F491848E6
:1067F00006F05CFFE3681648198802B0BDE8F04176
:1068000006F0BABF511A5C2202FB01F292FBF3F3CD
:106810001B33ABE7521A02EB4202C2EB4212334483
:1068200092FBF3F31B33BDE7402309212A46009175
:1068300007480195194606F0DBF93146044806F091
:106840009FFD02226821024806F096FD6368D2E7A8
:106850001CA0FF1F4C3401005034010054340100CF
:1068600095A0FF1FF29FFF1FF49FFF1F58340100E8
:106870002DE9F0471F4682B01446002A4ED0052A63
:106880000646D0F80C8000F0AB800B9B894A00EBE9
:10689000C305012CB5F80AE029896868C1EB0E032D
:1068A00082FB03C21A444FEAE373C3EBA2130288CC
:1068B00051D0042C00F08D800022402309218DE866
:1068C00006007D48194606F093F901217A4806F042
:1068D00057FD0222B8F1000F00F0E1804421764814
:1068E00006F04AFD73687448198806F045FF73493D
:1068F0007148012206F0DAFEF3686F48198806F045
:106900003BFF6F4B022CB3F9001000F0A680082C5F
:1069100000F0C280012002B0BDE8F087694E6A4AEB
:1069200033681268CB1A93420D4655D9674A3B88A3
:1069300011786148012918BF012414700A9A06329F
:106940001BB212B28DE814001946BDF9282006F0DA
:1069500081F93560DEE79BB2D31A994203DC9E458C
:106960007146A8BF19460A9A0180B7F90030BDF9EF
:1069700028A0514802F106094FF0000E0FFA89F9DC
:1069800019465246CDF80090CDF804E006F062F9C1
:1069900029896A896868521A03885C2AA3EB010373
:1069A00073DD03EB43030132C3EB431393FBF2F3B9
:1069B00003F11B0213B201203A801946524601909E
:1069C000CDF800903C4806F045F9404B00221A7083
:1069D00072E712FA83F3C0E7204602B0BDE8F08701
:1069E00007254FF000095A2323228DE820021A219F
:1069F000314806F0FDF801212F4806F0C1FC0121C5
:106A00002D4806F0C3FC232235212B4806F0B4FCA8
:106A10002A462F49284806F049FE274806F05CFE22
:106A2000254805F0CBFE4FF4FA6007F045FDFFF76F
:106A300085FA5A2323221A218DE820021E4806F0E7
:106A4000D7F81D4805F0BAFE3046FFF719FE214B76
:106A500001221A70FFF76EFC2EE74A1C12B21A8050
:106A600091423FF457AF0A9AB7F900301248063204
:106A7000012412B2009219460194BDF9282006F0B3
:106A8000E9F8204602B0BDE8F0875C2101FB03F382
:106A900093FBF2F21B328DE700221A80E0E76821B7
:106AA000054806F069FC73680348198806F064FE1F
:106AB00027E700BFC94216B21CA0FF1F58340100CF
:106AC000FA9FFF1F80A0FF1F5044010095A0FF1FE9
:106AD0005C340100F09FFF1F2DE9F04F5A4E5B4DD3
:106AE000B6F900704C7855F8277085B08146984605
:106AF00004B10C78DFF874A11AB99AF80030002BB1
:106B000039D0534D002338462B808AF80030FFF7E8
:106B1000B7FD504A504BB5F90000012111704FF6F6
:106B2000FF721A8060B301285ED001203223224612
:106B3000019000934946494B3846FFF799FE0024DF
:106B40000346B5F90020022A39DD00222A80B6F971
:106B500000203D49002A3BDB052AC4BF00220A80F1
:106B6000B8F1000F39D1002C0CBF18464FF0FF30A0
:106B700005B0BDE8F08F364DB5F900000028D2D140
:106B8000DFF8ECB0364ADBF800301268C3EB0903DB
:106B9000934227D9334B1A78012A18BF0120187065
:106BA000FFF7ACF90123CBF80090012C2AD0042C7C
:106BB00035D0022C3AD0082C3ED00024C1E7C6D1F3
:106BC000FA68002AC1D0B6F900201F49002AC3DAAA
:106BD00005220A80B8F1000FC5D00393FFF7AAFB86
:106BE000039BC0E70346E0E74FF0000E1423224664
:106BF0008DE8084049461C4B38467446FFF738FE7E
:106C000003469EE732888AF80040013232807A6972
:106C100082B10024384603939047039B91E7328862
:106C20000121013A32808AF80010F0E701222A801F
:106C300000248CE7144684E77A69002129804FF00C
:106C4000FF34002AE6D182E7F69FFF1F6C8AFF1F00
:106C5000FA9FFF1FF09FFF1F668AFF1FF49FFF1F11
:106C60005044010095A0FF1FF29FFF1FF89FFF1FD8
:106C700080A0FF1F01210D2007F0E2BB00210D20A5
:106C800007F0DEBB01460D2007F0DABB08B50D208A
:106C900007F0DCFBB0FA80F149090D20BDE808409F
:106CA00007F0CEBB10B5002144080D2007F0C8FB4B
:106CB000204607F001FC0D20012107F0C1FB204612
:106CC000BDE8104007F0F8BB2D4A2E4B10881B681A
:106CD000984210B549DA2C4A1288141A9A42A8BF71
:106CE0001A46B4F5157F36DA121A40F2532303FB25
:106CF00002F393FBF4F105310A2007F011FA234B5C
:106D00001978C9B3224B23491B6840F2271283F339
:106D1000070302FB03F381FB03211944DB17C3EBD9
:106D2000A1110531092007F0FBF91B4B1968F1B1DE
:106D300081F3070140F22712164802FB01F380FBA2
:106D400003211944DB17C3EBA11105311620BDE85F
:106D5000104007F0E5B9131A4FF41572611C02FBDD
:106D600003F393FBF1F10531C6E70021C4E71620D8
:106D7000BDE8104007F0D4B9092007F0D1F9D4E7F5
:106D8000E89DFF1F089DFF1FB29FFF1F929DFF1FE1
:106D9000989FFF1F09040281649FFF1F7F2838B559
:106DA000A8BF7F200F4C4FF4167202FB00F284FB49
:106DB00002311144D2170546C2EBA1110A2007F097
:106DC000AFF97F3D4FF4967303FB05F384FB03217A
:106DD0001944DB17A3EBA1110920BDE8384007F0E7
:106DE0009FB900BF09040281C368B3F9003030B510
:106DF00083EAE374A4EBE374002BA0B218DB012355
:106E000000E0134603EB830252009442F9DA0A4D84
:106E100090FBF3F285FB03E403FB1200DB17303237
:106E2000D3EBA40380B201F8012BF1D10B7030BD7C
:106E30002D230B700131E2E76766666638B5094DB0
:106E40008224204602F0E8FF35F8021B00B2884297
:106E5000204601D002F0C6FF0234A4B28A2CF0D141
:106E600038BD00BFD89EFF1F024B8020198802F05A
:106E7000B9BF00BF589DFF1F38B5094D7824204683
:106E800002F0CAFF35F8021B00B28842204601D04A
:106E900002F0A8FF0234A4B2802CF0D138BD00BFAC
:106EA000D09EFF1F024B7620198802F09BBF00BFC7
:106EB000569DFF1F38B5094D4624204602F0ACFF11
:106EC00035F8021B00B28842204601D002F08AFF4A
:106ED0000234A4B24E2CF0D138BD00BF589FFF1F22
:106EE000024B4420198802F07DBF00BF929FFF1F14
:106EF000024B4E20198802F075BF00BF6A9DFF1F2C
:106F0000024B9A20198802F06DBF00BFC89DFF1F79
:106F1000024B9820198802F065BF00BF5E9DFF1FDD
:106F2000024B8C20198802F05DBF00BFEE9EFF1F50
:106F3000024B9C20198802F055BF00BF429DFF1FE5
:106F4000024BA020198802F04DBF00BF609FFF1FB9
:106F5000024B9620198802F045BF00BF3C9FFF1FDF
:106F6000024B8A20198802F03DBF00BF029FFF1F1D
:106F7000024B1020198802F035BF00BF009FFF1F91
:106F8000024B2C20198802F02DBF00BF3E9DFF1F31
:106F9000024B1E20198802F025BF00BF5C9DFF1F19
:106FA000C3680E20198802F01DBF00BF024B2820C5
:106FB000198802F017BF00BF569FFF1F024B6420C5
:106FC000198802F00FBF00BF509FFF1F024BB42073
:106FD000198802F007BF00BFA89FFF1F024BB62011
:106FE000198802F0FFBE00BFD89FFF1F024B5A2036
:106FF000198802F0F7BE00BF189DFF1F024B162034
:10700000198802F0EFBE00BF249DFF1F024B2E2007
:10701000198802F0E7BE00BFD09DFF1F024B302051
:10702000198802F0DFBE00BFC09FFF1F024B9E20E9
:10703000198802F0D7BE00BFC489FF1F024BAC20E5
:10704000198802F0CFBE00BF529FFF1F024BAE2037
:10705000198802F0C7BE00BF689DFF1F024BB02019
:10706000198802F0BFBE00BFE49EFF1F024BB22092
:10707000198802F0B7BE00BF869DFF1F024B182083
:10708000198802F0AFBE00BFEE9DFF1F024BA22089
:10709000198802F0A7BE00BF869FFF1F024B1A206F
:1070A000198802F09FBE00BF769DFF1F024B1C2077
:1070B000198802F097BE00BF6C9DFF1F024B66202F
:1070C000198802F08FBE00BF909FFF1F024B7220F5
:1070D000198802F087BE00BFBC9FFF1F024B202013
:1070E000198802F07FBE00BF8E9FFF1F024B322027
:1070F000198802F077BE00BF7E9FFF1F024B6820F9
:10710000198802F06FBE00BFB09DFF1F024B6C20BC
:10711000198802F067BE00BF0C9DFF1F024B6E2056
:10712000198802F05FBE00BFEE9FFF1F024B522086
:10713000198802F057BE00BF5E89FF1F024B502026
:10714000198802F04FBE00BF2089FF1F024B542058
:10715000198802F047BE00BF188AFF1F024B5C204F
:10716000198802F03FBE00BF648AFF1F024B5E20F9
:10717000198802F037BE00BF5C89FF1F024B562002
:10718000198802F02FBE00BFBE9DFF1F244B1B8835
:107190000B2B43D8DFE803F00B10151A1F24292E00
:1071A00033383D06084604221E490BF067B90846ED
:1071B00004221D490BF062B9084604221B490BF05A
:1071C0005DB9084604221A490BF058B90846042252
:1071D00018490BF053B90846042217490BF04EB971
:1071E0000846042215490BF049B9084604221449FF
:1071F0000BF044B90846042212490BF03FB9084687
:10720000042211490BF03AB9084604220F490BF049
:1072100035B9084604220E490BF030B9704700BF5B
:107220003C9FFF1FF0400100443E0100AC3C0100C8
:10723000E03D0100B03C010034420100B43C0100DB
:10724000B83C0100883F0100BC3C0100FC4001004B
:10725000C03C0100064B074A10B41C88064B084688
:10726000002C14BF11461946042210BC0BF006B9BD
:107270008C9DFF1FC43C0100C83C0100064B074A1F
:1072800010B41C88064B0846002C14BF1146194642
:10729000042210BC0BF0F2B8D29DFF1FC43C0100C9
:1072A000C83C0100064B074A10B41C88064B084630
:1072B000002C14BF11461946042210BC0BF0DEB896
:1072C000F69EFF1FC43C0100C83C0100064B074A64
:1072D00010B41C88064B0846002C14BF11461946F2
:1072E000042210BC0BF0CAB83E9FFF1FC43C010033
:1072F000C83C0100064B074A10B41C88064B0846E0
:10730000002C14BF11461946042210BC0BF0B6B86D
:10731000DA9DFF1FC43C0100C83C01001B4B1B88C9
:107320000A2B0AD8DFE803F00A0E12161A1E2226CC
:107330002A2E0600164B186808607047154B18680F
:1073400008607047144B186808607047134B186842
:1073500008607047124B186808607047114B186836
:1073600008607047104B1868086070470F4B18682A
:10737000086070470E4B1868086070470D4B18681E
:10738000086070470C4B186808607047029FFF1F29
:10739000F03C0100C83C0100CC3C0100D03C0100A5
:1073A000D43C0100D83C0100DC3C0100E03C010081
:1073B000E43C0100E83C0100EC3C0100F0B52B4E40
:1073C0002B4FDFF8C4E005460FCE87B06C460FC4E4
:1073D00096E803003B68274A274F44F8040B40F621
:1073E000CC308342C8BF3A46BEF800602180012EEF
:1073F00011889278ADF80D108DF80F202AD032D375
:1074000040F6CA02022E18BF00229A4226DAA3F6DC
:1074100098031A491A4AC3EB031381FB0301194469
:10742000DB17C3EB6123243382FB0321DA17C2EBA2
:10743000A10202EB8201A3EB4103303330328DF81D
:1074400013308DF811206946284616220BF016F8E5
:1074500007B0F0BD40F698029A42D8DB094B186895
:10746000CDF81100EFE740F6FC02CEE7043D010045
:10747000449FFF1FF83C0100F43C01003B773B9820
:1074800067666666FC3C0100E09EFF1FF8B5174C7E
:10749000174E2278174D33782F888E46003218BF4A
:1074A000012201467046FFF717FB00239842337014
:1074B000237015DB14BF012000202B889F420ED0C3
:1074C00040F23A72A3F5AF730B490C4C02FB03F385
:1074D00081FB0312DB17A3EB621332332360F8BD89
:1074E0000749012218460A702270E6E7148BFF1F35
:1074F00009A0FF1FAC9FFF1FB5814E1B088AFF1F0D
:1075000094A0FF1F014B187802F004BC7CA0FF1F61
:10751000014B187802F018BCD091FF1F134BB3F940
:10752000003030B583EAE374A4EBE374002BA0B21F
:1075300018DB012300E0134603EB83025200944260
:10754000F9DA0B4D90FBF3F285FB03E403FB120029
:10755000DB173032D3EBA40380B201F8012BF1D159
:107560000B7030BD2D230B700131E2E7D091FF1F6E
:1075700067666666144BB3F9003070B583EAE3754D
:10758000A5EBE375002BACB21ADB012300E0034648
:1075900003EB830040008542F9DA0C4E94FBF3F0D4
:1075A00086FB03E503FB1044DB173030D3EBA50368
:1075B000A4B201F8010BF1D105480B70106070BD49
:1075C0002D230B700131E0E7189DFF1F676666668B
:1075D0001C3D0100134BB3F9003030B583EAE3746E
:1075E000A4EBE374002BA0B218DB012300E01346E8
:1075F00003EB830252009442F9DA0B4D90FBF3F255
:1076000085FB03E403FB1200DB173032D3EBA4034A
:1076100080B201F8012BF1D10B7030BD2D230B701E
:107620000131E2E7C489FF1F67666666134BB3F951
:10763000003030B583EAE374A4EBE374002BA0B20E
:1076400018DB012300E0134603EB8302520094424F
:10765000F9DA0B4D90FBF3F285FB03E403FB120018
:10766000DB173032D3EBA40380B201F8012BF1D148
:107670000B7030BD2D230B700131E2E7689DFF1FB9
:1076800067666666134BB3F9003030B583EAE3747E
:10769000A4EBE374002BA0B218DB012300E0134637
:1076A00003EB830252009442F9DA0B4D90FBF3F2A4
:1076B00085FB03E403FB1200DB173032D3EBA4039A
:1076C00080B201F8012BF1D10B7030BD2D230B706E
:1076D0000131E2E7869DFF1F67666666134BB3F9CB
:1076E000003030B583EAE374A4EBE374002BA0B25E
:1076F00018DB012300E0134603EB8302520094429F
:10770000F9DA0B4D90FBF3F285FB03E403FB120067
:10771000DB173032D3EBA40380B201F8012BF1D197
:107720000B7030BD2D230B700131E2E7869FFF1FE8
:1077300067666666134BB3F9003030B583EAE374CD
:10774000A4EBE374002BA0B218DB012300E0134686
:1077500003EB830252009442F9DA0B4D90FBF3F2F3
:1077600085FB03E403FB1200DB173032D3EBA403E9
:1077700080B201F8012BF1D10B7030BD2D230B70BD
:107780000131E2E75E89FF1F67666666134BB3F956
:10779000003030B583EAE374A4EBE374002BA0B2AD
:1077A00018DB012300E0134603EB830252009442EE
:1077B000F9DA0B4D90FBF3F285FB03E403FB1200B7
:1077C000DB173032D3EBA40380B201F8012BF1D1E7
:1077D0000B7030BD2D230B700131E2E72089FF1FB4
:1077E00067666666134BB3F9003030B583EAE3741D
:1077F000A4EBE374002BA0B218DB012300E01346D6
:1078000003EB830252009442F9DA0B4D90FBF3F242
:1078100085FB03E403FB1200DB173032D3EBA40338
:1078200080B201F8012BF1D10B7030BD2D230B700C
:107830000131E2E7188AFF1F67666666134BB3F9EA
:10784000003030B583EAE374A4EBE374002BA0B2FC
:1078500018DB012300E0134603EB8302520094423D
:10786000F9DA0B4D90FBF3F285FB03E403FB120006
:10787000DB173032D3EBA40380B201F8012BF1D136
:107880000B7030BD2D230B700131E2E7648AFF1FBE
:1078900067666666134BB3F9003030B583EAE3746C
:1078A000A4EBE374002BA0B218DB012300E0134625
:1078B00003EB830252009442F9DA0B4D90FBF3F292
:1078C00085FB03E403FB1200DB173032D3EBA40388
:1078D00080B201F8012BF1D10B7030BD2D230B705C
:1078E0000131E2E75C89FF1F6766666608B5B8206C
:1078F00002F092FA044B1988884204D0B820BDE8FF
:10790000084002F06FBA08BD209DFF1F08B5702027
:1079100002F082FA044B1988884204D07020BDE836
:10792000084002F05FBA08BDE09EFF1F08B5742052
:1079300002F072FA044B1988884204D07420BDE822
:10794000084002F04FBA08BD749FFF1F054B1B880B
:107950000846042213B904490AF090BD03490AF00D
:107960008DBD00BF6A9DFF1F243D0100203D010029
:107970000E4B1B88032B17D8DFE803F0110C07020E
:10798000084604220A490AF079BD0846042209493A
:107990000AF074BD0846042207490AF06FBD084684
:1079A000042206490AF06ABD704700BFEE9EFF1F21
:1079B000303D0100C83D01002C3D0100283D010083
:1079C00010B40A4B0A4C0A4693E8030083B023889C
:1079D00002AC04E9030004EB8303104653F8081CCF
:1079E000052203B010BC0AF049BD00BFDC34010021
:1079F000509FFF1F30B40A4B0A4D0C4693E8070016
:107A000084B02B8804AD05E9070005EB830320460D
:107A100053F80C1C042204B030BC0AF02FBD00BF88
:107A2000E4340100E09EFF1FF0B40C4D0C4F0E46F5
:107A30000FCD8CB001AC0FC40FCD0FC495E807007B
:107A40003B8884E807000CAA02EB8303304653F816
:107A50002C1C04220CB0F0BC0AF010BDF034010064
:107A6000349FFF1F30B50A4B0A4D0C460FCB85B033
:107A70000DF1100E0EE90F002B880EEB830320464C
:107A800053F8101C042205B0BDE830400AF0F6BCE3
:107A90002C350100529FFF1F30B50A4B0A4D0C4692
:107AA0000FCB85B00DF1100E0EE90F002B880EEBF9
:107AB0008303204653F8101C042205B0BDE8304073
:107AC0000AF0DCBC2C350100E49EFF1FF0B40B4D26
:107AD0000B4F0E460FCD86B06C460FC495E80300E1
:107AE0003B8884E8030006AA02EB8303304653F880
:107AF000181C042206B0F0BC0AF0C0BC3C350100E2
:107B0000EE9DFF1FF0B40A4D0A4F0E460FCD86B012
:107B100001AC0FC42A683B88226006AA02EB8303EB
:107B2000304653F8141C0C2206B0F0BC0AF0A6BC78
:107B3000543501006C9DFF1FF0B40B4D0B4F0E46EA
:107B40000FCD86B06C460FC495E803003B8884E8EF
:107B5000030006AA02EB8303304653F8181C0422E4
:107B600006B0F0BC0AF08ABC68350100749FFF1FA4
:107B7000164B1B880BB31BB283EAE370A0EBE370D8
:107B8000002B30B584B21DDB012300E0134603EB6C
:107B9000830252009042F9DA0D4894FBF3F280FB25
:107BA00003E503FB1244DB173032D3EBA503A4B289
:107BB00001F8012BF1D10B7030BD084604220549B4
:107BC0000AF05CBC2D230B700131DDE7B09DFF1F77
:107BD00067666666343D0100F0B40A4D0A4F0E46F2
:107BE0000FCD86B001AC0FC42A683B88226006AA7C
:107BF00002EB8303304653F8141C042206B0F0BC99
:107C00000AF03CBC803501000C9DFF1F054B1B8812
:107C10001BB9054B186808607047084604220349E1
:107C20000AF02CBCC89DFF1FC83C0100C43C0100E9
:107C3000164B1B880BB31BB230B583EAE374A4EB7D
:107C4000E374002BA0B21CDB012300E0134603EB1E
:107C5000830252009442F9DA0D4D90FBF3F285FB5A
:107C600003E403FB1200DB173032D3EBA40380B232
:107C700001F8012BF1D10B7030BD064B186808607C
:107C800070472D230B700131DEE700BF5C9DFF1FA5
:107C900067666666C83C0100164B1B880BB31BB2B7
:107CA00030B583EAE374A4EBE374002BA0B21CDBD1
:107CB000012300E0134603EB830252009442F9DAF9
:107CC0000D4D90FBF3F285FB03E403FB1200DB1781
:107CD0003032D3EBA40380B201F8012BF1D10B7049
:107CE00030BD064B1868086070472D230B700131BA
:107CF000DEE700BF209DFF1F67666666C83C010087
:107D0000164B1B880BB31BB230B583EAE374A4EBAC
:107D1000E374002BA0B21CDB012300E0134603EB4D
:107D2000830252009442F9DA0D4D90FBF3F285FB89
:107D300003E403FB1200DB173032D3EBA40380B261
:107D400001F8012BF1D10B7030BD064B18680860AB
:107D500070472D230B700131DEE700BF429FFF1FEC
:107D600067666666C83C0100164B1B880BB31BB2E6
:107D700030B583EAE374A4EBE374002BA0B21CDB00
:107D8000012300E0134603EB830252009442F9DA28
:107D90000D4D90FBF3F285FB03E403FB1200DB17B0
:107DA0003032D3EBA40380B201F8012BF1D10B7078
:107DB00030BD064B1868086070472D230B700131E9
:107DC000DEE700BF249DFF1F67666666383D010041
:107DD000174B1B881BB31BB270B583EAE375A5EB89
:107DE000E375002BACB21EDB012300E0034603EB7E
:107DF000830040008542F9DA0E4E94FBF3F086FBD7
:107E000003E503FB1044DB173030D3EBA503A4B22A
:107E100001F8010BF1D108480B70106070BD074BE1
:107E20001868086070472D230B700131DCE700BF34
:107E3000D09DFF1F676666663C3D0100C83C01009F
:107E4000164B1B880BB31BB230B583EAE374A4EB6B
:107E5000E374002BA0B21CDB012300E0134603EB0C
:107E6000830252009442F9DA0D4D90FBF3F285FB48
:107E700003E403FB1200DB173032D3EBA40380B220
:107E800001F8012BF1D10B7030BD064B186808606A
:107E900070472D230B700131DEE700BFC09FFF1F2D
:107EA00067666666C83C0100164B1B880BB31BB2A5
:107EB00030B583EAE374A4EBE374002BA0B21CDBBF
:107EC000012300E0134603EB830252009442F9DAE7
:107ED0000D4D90FBF3F285FB03E403FB1200DB176F
:107EE0003032D3EBA40380B201F8012BF1D10B7037
:107EF00030BD064B1868086070472D230B700131A8
:107F0000DEE700BF909FFF1F67666666C83C010002
:107F1000164B1B880BB31BB230B583EAE374A4EB9A
:107F2000E374002BA0B21CDB012300E0134603EB3B
:107F3000830252009442F9DA0D4D90FBF3F285FB77
:107F400003E403FB1200DB173032D3EBA40380B24F
:107F500001F8012BF1D10B7030BD064B1868086099
:107F600070472D230B700131DEE700BFBC9FFF1F60
:107F700067666666C83C0100174B1B881BB31BB2C3
:107F800070B583EAE375A5EBE375002BACB21EDB9D
:107F9000012300E0034603EB830040008542F9DA49
:107FA0000E4E94FBF3F086FB03E503FB1044DB1756
:107FB0003030D3EBA503A4B201F8010BF1D108488E
:107FC0000B70106070BD074B1868086070472D2358
:107FD0000B700131DCE700BF8E9FFF1F676666668E
:107FE0003C3D0100C83C0100054B1B881BB1054B03
:107FF000186808607047044B18680860704700BF35
:10800000BE9DFF1F503D01004C3D010070B5FAF7C9
:1080100093F8164B1B7813B1154C237833B9154BD5
:108020001020198801F0DEFE012070BD124D134EA4
:108030002B783288B3FA83F382F008025B09114689
:1080400042202B70328001F0CDFE23780BB12B78CB
:108050002BB90021212006F0F3F9002070BD012189
:10806000212006F0EDF9002070BD00BF269DFF1F06
:10807000E69EFF1F009FFF1FFE9EFF1FB49FFF1F76
:10808000184B1A8852B3184A128830B50A80B3F9CF
:108090000030002B83EAE374A4EBE374BCBF2D2310
:1080A0008B70A0B2ACBF02310331012300E0134654
:1080B00003EB830252009442F9DA0C4D90FBF3F289
:1080C00085FB03E403FB1200DB173032D3EBA40380
:1080D00080B201F8012BF1D10B7030BD044B186850
:1080E00008607047769DFF1F543D01006766666615
:1080F000C83C010070B53C4D2B780646002B35D1AD
:108100001C4673780BB9204670BDFAF715F8374A4C
:10811000374B3848127831781B78007802EB4303EC
:108120004A1E03EB80030E2AEDD801A050F822F07E
:1081300099810000BB810000078100009981000047
:10814000078100000781000007810000878100008F
:1081500007810000078100000781000007810000FF
:10816000078100000781000083810000AE212248C2
:1081700003F0C8FF204804F015FA00232B700124F7
:10818000BFE706F083FEAF211B4803F0BBFF1B4A8D
:10819000012313702B70B6E783B9194803880429AB
:1081A0004FF6FF7103F1FF320CBF01230B4613445E
:1081B00003F07F03013303800FE073B1013B114AE9
:1081C00032F813304BB10E4E0F481049104A33802D
:1081D0000123002606700B701370084A0221012348
:1081E00011702B70204670BD148BFF1F959FFF1FD1
:1081F000969FFF1F979FFF1F1CA0FF1F94A0FF1FAC
:10820000809FFF1FC09EFF1FA89DFF1F2C9DFF1F6B
:1082100097A0FF1F10B5064B064C1A882046012177
:1082200001F0CEFD21884220BDE8104001F0DABD0A
:108230008C9DFF1FB49FFF1F10B5064B064C1A887C
:108240002046022101F0BCFD21884220BDE81040FB
:1082500001F0C8BDD29DFF1FB49FFF1F10B5064B94
:10826000064C1A882046042101F0AAFD21884220EC
:10827000BDE8104001F0B6BDF69EFF1FB49FFF1F82
:1082800010B5064B064C1A882046002101F098FDD7
:1082900021884220BDE8104001F0A4BD3E9FFF1F91
:1082A000B49FFF1F08B5122001F0B6FD054B1988D9
:1082B000884206D0122001F095FDBDE8084001F08B
:1082C0005BBC08BD349FFF1F08B5582001F0A4FD1A
:1082D000054B1988884206D0582001F083FDBDE87F
:1082E000084001F049BC08BD429FFF1F08B514209B
:1082F00001F092FD054B1988884206D0142001F048
:1083000071FDBDE8084001F037BC08BDDA9DFF1FD4
:10831000F0B480EAE075A5EBE0750028ACB21FDB95
:108320001DBF2B230B704E1C0E46012300E013468D
:1083300003EB830252009542F9DA0B4F94FBF3F200
:1083400087FB030503FB1244DB173032D3EBA50395
:10835000A4B206F8012BF1D133700846F0BC704787
:108360002D230B704E1CE0E767666666084B188885
:1083700028B10D2807D00D3800B2FFF7C9BF054A54
:10838000106808607047044A10680860704700BFB2
:10839000EE9FFF1FC83C0100583D0100174B188895
:1083A0000C2813D0192815D01A2817D01B2819D03B
:1083B0001C281BD01D281DD01E2803D00C3800B24D
:1083C000FFF7A6BF0E4A1068086070470D4A106894
:1083D000086070470C4A1068086070470B4A1068C4
:1083E000086070470A4A106808607047094A1068B8
:1083F00008607047084A1068086070477E9FFF1F3A
:10840000743D01005C3D0100603D0100643D0100E0
:10841000683D01006C3D0100703D0100034B188870
:10842000A0EB8000400000B2FFF772BF7CA0FF1FEE
:10843000024B1888643800B2FFF76ABFD89FFF1F4D
:10844000024B1888643800B2FFF762BFA89FFF1F75
:10845000024B1888033800B2FFF75ABF569FFF1F20
:10846000024B18880C3800B2FFF752BF1E9DFF1F49
:10847000024B1888183800B2FFF74ABF589DFF1FFB
:10848000024B1888183800B2FFF742BF569DFF1FF5
:10849000024B1888183800B2FFF73ABF929FFF1FAF
:1084A000C3681888183800B2FFF732BF054B1B8825
:1084B0001BB9054B18680860704708460422034939
:1084C00009F0DCBF609FFF1FC83C0100C43C0100F5
:1084D000054B1B881BB9054B186808607047084698
:1084E0000422034909F0CABF5E9DFF1FC83C01007A
:1084F000C43C010030B5134C85B001252B463C220D
:1085000002212046009503F073FE204604F04AF84D
:1085100000224021802320460191009311460A4BFE
:10852000029504F0EDFC204604F048F9074808499C
:10853000084A0023036083800B608B801360938064
:1085400005B030BD1CA0FF1F30380100FC9FFF1F8D
:1085500014A0FF1F84A0FF1F10B500EBC00000F1A6
:108560000F02D2B293B284B09C1E981C3D2303919B
:108570008DE819003921024804F026FC04B010BD32
:108580001CA0FF1F014B01221A70704709A0FF1F9A
:10859000F0B5784B784C794F794E7A4D85B00422FE
:1085A0008DE80C0002932046774B4022802103F097
:1085B00027FC2046754A7649764C09F0CBF8764B75
:1085C00076489F61764FDF61764FB761764FF761EE
:1085D000764FAF61764FEF61764FA761764FE761D7
:1085E000764F87617649774FC761774F8F61774ABA
:1085F000774FCF61774F9761774B784FD761784F3F
:108600009F61784E784FDF61784FB761784D794F31
:10861000F761794F794CAF61794FEF61794F7A48C3
:10862000A7617A4FE7617A4F7A4987617A4FC761CC
:108630007A4F7B4A8F617B4FCF617B4F7B4B97613A
:108640007B4FD7617B4F7C4E9F617C4FDF617C4FBE
:108650007C4DB7617C4FF7617C4FAF617C4C7D4FA7
:10866000EF617D4FA7617D487D4FE7617D4F876159
:108670007D497E4FC7617E4F8F617E4A7E4FCF61BD
:108680007E4F97617E4B7F4FD7617F4F9F617F4EBB
:108690007F4FDF617F4FB7617F4D804FF761804F24
:1086A000AF61804C804FEF61804FA7618048814F60
:1086B000E761814F87618149814FC761814F824A5C
:1086C0008F61824FCF61824F824B9761824FD7611A
:1086D000824F834E9F61834FDF61834F834DB7612C
:1086E000834FF761834F844CAF61844FEF61844FB8
:1086F0008448A761844FE761844F85498761854F2E
:10870000C761854F8F61854A854FCF61854F9761DE
:10871000854B864FD761864F9F61864E864FDF61BE
:10872000864F874DB761874FF761874F874CAF61A1
:10873000874F88488849EF61884F894DA761E56177
:10874000884F894D894CDFF848E2894A894B876117
:10875000C5618C61884E894F894D8A4CC1F81CE0F7
:1087600089488A499761D5619C61D861B16005B03B
:10877000F0BD00BF40420F001CA0FF1F618400003D
:10878000D08FFF1F1C8FFF1FEC91FF1F1C89FF1F45
:1087900059BE00009C8CFF1F048EFF1FF48FFF1F2B
:1087A000A16F000051840000AD6F00005572000001
:1087B000158200007D72000039820000A572000061
:1087C000BC8DFF1F5D820000C1790000088DFF1F76
:1087D000BD6F0000CD720000E08DFF1F81820000A0
:1087E000418400007C91FF1FCD6F000031840000A8
:1087F0005891FF1FDD6F0000997C0000988DFF1FCE
:10880000ED7800001D840000748DFF1F05750000C9
:108810001D750000AC8FFF1F11750000F579000079
:10882000308CFF1F0D790000297A00006090FF1F37
:10883000A5820000017D0000E48CFF1FC9820000BA
:1088400075750000F08BFF1FED6F0000F5720000E2
:10885000F090FF1FED820000697D0000C08CFF1FBB
:10886000FD6F0000D17D00004C8EFF1F0D700000D9
:10887000417E0000788CFF1F1D700000D575000040
:10888000A88BFF1F2D700000657A0000A890FF1FC5
:108890003D7000002D760000648FFF1F4D700000BA
:1088A000997A0000848BFF1F5D70000085760000C0
:1088B000288EFF1F6D700000CD7A0000CC8AFF1F4C
:1088C0007D700000DD7600002C8DFF1F8D70000094
:1088D00081800000888FFF1F9D700000057B0000D5
:1088E000AC91FF1FAD700000A97E0000F88EFF1F45
:1088F000BD700000117F0000608BFF1FCD70000075
:10890000397B00008490FF1F2D790000797F0000E3
:10891000408FFF1FDD7000009D8300003C8BFF1F18
:10892000ED700000717B0000188BFF1FFD700000D0
:10893000D97B0000848AFF1F0D7100006D83000049
:10894000508DFF1F1D71000035770000548CFF1FF4
:108950002D710000F08AFF1FCC8BFF1F8D77000068
:108960003D710000E57700004D7100003D7800008A
:108970001890FF1FA88AFF1FA091FF1F9578000085
:108980006D710000E97F00007D710000558F0000CF
:108990005D710000F0B5461C83B00D46012703232E
:1089A00036B22AB2044631468DE888002348ADB27B
:1089B00004F0A0F90C23AA1C12B20093019705231E
:1089C00021B21E4804F096F91D4A1E4B12881B68FE
:1089D000BA422AD023D3022A10D11B4CA3F6CA03D1
:1089E00084FB03241C44DB17C3EB24140A2CA8BF0C
:1089F0000A2424EAE474A2B223B202E000231A4655
:108A00001C460D35AA1A01200093019012B231467E
:108A100003230A4804F0ECF8204603B0F0BD0B4CE9
:108A2000A3F6FC0384FB0324DDE7094CA3F69803BB
:108A300084FB0324DB17C3EBA404D7E71CA0FF1FB0
:108A4000E09EFF1F449FFF1F09CB3D8D1F85EB510B
:108A5000398EE3382DE9F0438FB283B0DFF84C80D4
:108A6000BD1D461D2DB204B236B24FF001090AB247
:108A70002346314640460095CDF8049004F0EAF8CC
:108A80002A463346214640468DE8200204F0E2F8AB
:108A900007F10C020095334612B22146CDF804903E
:108AA000404604F0D7F803B0BDE8F0831CA0FF1FD8
:108AB0002DE9F043804685B0002956D10121304888
:108AC00004F05EFC2F4998F8062098F8083011F859
:108AD0000290994522DA4FEA89064D460C24D8F8CF
:108AE0000C3027489B595F6822B2002104F044FCF7
:108AF000384609F005FC39460246214804F0D6FD07
:108B00001F4804F0E9FD98F8083001350934AB42FC
:108B1000A4B206F1040601DD422CE0D1B9F1000F48
:108B200013D109F1060999450CDA3C2301213B22B6
:108B3000039102930093019239233F223A21104876
:108B400004F042F905B0BDE8F0830F2301213B2278
:108B5000039102930093019239230C223A21084891
:108B600004F032F998F80830DBE700213423009351
:108B700001913F230C22024804F03AF89EE700BF1F
:108B80001CA0FF1F14A0FF1F10B5104C0121204690
:108B900004F0FCFB2046012104F0F2FB20463422C5
:108BA000552104F0E9FB20460222094904F07EFD2C
:108BB00020460522074904F079FD204604F08CFD8B
:108BC0002046BDE8104003F0F9BD00BF1CA0FF1F08
:108BD000C03D0100C43D010070B50D46064609F0D8
:108BE0008FFB00EB40008400002D36D0284609F0B2
:108BF00087FB00EB4000400023185B1003F160018D
:108C0000091A282209B21748C3F1600404F0B4FB22
:108C10000121144804F0B4FB284609F071FB2946F1
:108C20000246104804F042FD0E4804F055FD0221B2
:108C30000C4804F0A5FB21B221220A4804F09CFB59
:108C4000304609F05DFB31460246064804F02EFD31
:108C50000448BDE8704004F03FBD6410C4F16004F6
:108C6000E5E700BF1CA0FF1F10B50D4B1B5C51F8C2
:108C70002340237884B013B1012004B010BD04AAAE
:108C800001A942F8103D2046A3699847A38A9B0793
:108C9000F2D401A80099FFF79FFF012004B010BD96
:108CA000FC9FFF1F2DE9F04F2F4DDFF8CCB0DFF810
:108CB000C4A0DFF8C8900FCD91B003AC0FC40FCDA6
:108CC0000FC40FCD0FC42B6823600025A8462F4684
:108CD0002E4600E09846BAF8003024495BF823207D
:108CE00028461123F7F77EFD00EBC00400EB84005B
:108CF00089FB00340444C017C0EB6434C4F13C0069
:108D0000C6F13C0207F14101012600B208F141031E
:108D100000901BB2019612B209B2154803F09AFFF7
:108D200008EB060305F211153C2B2646ADB247466B
:108D3000D0D134226B210E4804F01EFB00210C48D8
:108D400004F01EFB0B4B1B8810AA02EB830353F8A5
:108D5000344C204609F0D4FA02460548214611B0A9
:108D6000BDE8F04F04F0A2BC94350100402F010093
:108D70001CA0FF1F3E9DFF1FA42D010009000280C3
:108D8000234B70B5B3F9003083EAE374A4EBE374CA
:108D9000002B82B0A1B234DB68466D46012300E0AF
:108DA000134603EB830252009442F9DA194E91FB09
:108DB000F3F286FB03E403FB1211DB173032D3EB33
:108DC000A40389B205F8012BF1D119462B70FFF7E6
:108DD00003FF114B1B7813B1104B1B780BB902B07A
:108DE00070BD01210E4804F0CBFA332264210C48F7
:108DF00004F0C2FA04220B49094804F057FC02B0FF
:108E000070BD2D238DF800300DF101056846C5E7D2
:108E1000009FFF1F67666666E69EFF1FFE9EFF1FA0
:108E20001CA0FF1FCC3D010010B5424C424882B04F
:108E300003F0B8FB2378C3B906213F4804F0A0FA39
:108E40002378012B37D90A22022B11463A486BD0DE
:108E500004F092FA39490322374804F027FC3648D7
:108E600002B0BDE8104004F037BC354B1A78012140
:108E70000523002A35D10191009311462E4803F0B5
:108E800039FF304B1A78002A36D00523012201928F
:108E9000009300220A21284803F0AAFE2A4B1A78E0
:108EA000002A35D101210523019100931421224884
:108EB00003F020FFC0E7254C2388092B32D9632B10
:108EC0008CBF0A211F210A221B4804F055FA218871
:108ED000194804F051FC184802B0BDE8104004F0F5
:108EE000FBBB0022019100931146134803F080FE62
:108EF000144B1A78002AC8D105230121019100934F
:108F00000A210D4803F0F6FE0F4B1A78002AC9D04B
:108F1000012205230192009300221421064803F048
:108F200067FE89E73021CEE704F026FA03220849DC
:108F300092E700BF97A0FF1F1CA0FF1FD83D0100B4
:108F4000959FFF1F969FFF1F979FFF1F809FFF1FEB
:108F5000D43D0100F8B56D4D287840B96C4B1B68C5
:108F600099425CD36B4A012313702B70F8BD0C46F9
:108F700000266948664F03F015FB04F6AC533246F1
:108F800065483B6031212E7004F0F6F901216248FA
:108F9000624D04F0FBF931465F4804F0F1F9052217
:108FA0005F495D4804F082FB5B4804F095FB0C22AE
:108FB0001021594804F0E0F90B225A49564804F0B0
:108FC00075FB05225849544804F070FB524804F0E0
:108FD00083FB564B50481C68A4F69803C3EB03135D
:108FE00085FB03251D441021DB172022C3EB6525DB
:108FF00004F0C2F940F6CC339C4205F124054FF051
:1090000022014FF004000BDCFFF7C4FC484B1C8826
:10901000064674B3012C46D0022C41D00120F8BD85
:10902000FFF718FD092243493B4804F03FFB2A2281
:109030001021394804F0A0F93F4C374884FB05342F
:10904000EB17C3EBA404214604F096FB01223B4935
:10905000314804F02BFB04EB8401A5EB41012E48C1
:1090600004F08AFB012236492B4804F01FFB012043
:10907000F8BD34491022284804F018FB264804F0B3
:109080002BFB2A221021244804F076F9314622488D
:1090900004F072FB07222C491F4804F007FBCBE7C2
:1090A0000C222A49E7E70C2229491B4804F0FEFA62
:1090B000194804F011FB2A221021174804F05CF92A
:1090C000314615481C4E04F057FB07221E49124832
:1090D00004F0ECFA86FB0536EB17C3EBA606314627
:1090E0000D4804F049FB224614490B4804F0DEFA0F
:1090F00006EB8601A5EB4101074804F03DFB224643
:109100000F49054804F0D2FA2046F8BD148BFF1F22
:1091100010A0FF1F94A0FF1F1CA0FF1F3B773B98D0
:10912000DC3D0100E43D0100C43D0100449FFF1F00
:10913000E09EFF1FF03D010067666666DC450100AA
:109140004C450100FC3D0100103E0100283E01009D
:10915000183E01002DE9F041754C2278002A0546A1
:109160000F4614BF4FF001084FF000084ED1714E6A
:109170003368CB1AB3F5FA6F04D86B78A3B94046BD
:10918000BDE8F0816C4B6D486D49DFF8D0E11A7095
:10919000012303700988237026208EF8002000F038
:1091A00021FE6B78002BEAD03760F8F7C5FF654ADF
:1091B000654B6649127828781B78097802EB4303DF
:1091C000421E03EB81030E2AD9D801A151F822F0E7
:1091D000C19200008D9200007F910000C1920000BA
:1091E0007F9100007F9100007F9100007592000048
:1091F0007F910000279200007F9100007F91000086
:109200007F9100007F91000023920000AF21504821
:10921000484E02F077FFFFF707FE00233760237008
:10922000ABE705F033FE4A4803F0BCF90221484899
:1092300004F0A6F80F222321454804F09DF80522EA
:109240004449434804F032FA414804F045FA1E22EA
:1092500023213F4804F090F805223F493C4804F0A0
:1092600025FA3B4804F038FA394803F0A7FA00F031
:10927000D3FC84E7394D2B78012B50D9304B262075
:10928000198800F0AFFD00232B7078E7002B3FF426
:1092900076AF013B324A32F81330002B3FF46FAF08
:1092A000274C304825492D4A23804FF001080023E0
:1092B000037081F8008082F80080FFF7B5FD5EE75B
:1092C00093B1013B264A32F8131019B31C4B254DBC
:1092D0001A4C224A19800026012326202E70237062
:1092E000137000F07FFD15E0154C1E4922880B70AD
:1092F00004284FF6FF7002F1FF310CBF0122024635
:109300000A440E4E154D02F07F02013201212280E7
:1093100031702B70FFF788FD4FF001082FE70649E9
:10932000064A01230020087013702370A6E700BFCF
:10933000148BFF1F90A0FF1F94A0FF1F2C9DFF1FE9
:10934000809FFF1F959FFF1F969FFF1F979FFF1FE7
:109350001CA0FF1F383E0100403E010097A0FF1FE8
:10936000C09EFF1FA89DFF1F2DE9F04F05468BB043
:109370000F46AD480121164604F008F8AA8812F0FD
:10938000010440F0B080DFF8CC8298F80030002B68
:109390007DD1AB79A54AD15CA1B9DFF8BCA27978BF
:1093A0001AF8039041B339780139072900F2B780E0
:1093B000DFE811F0F1005401B5006C01B500B50013
:1093C000B500E9007C78002C00F0CA800139EC6817
:1093D000387854F82170FC68411EB4F800800729E1
:1093E00000F2A780DFE811F074015901A5006C01BB
:1093F000A500A500A5009F00DFF854A2DAF8002020
:10940000B21AB2F5967F75D9894A107801281ABF29
:10941000012010701170874A18BF0146D05CC0EB64
:109420000900C0B2FFF798F80124CAF80060AB88C1
:109430009B0770D57B78002B6DD0F8F77DFE7E4BB7
:109440007E4A7F481B78127839780078022515FB10
:1094500002330A2903EB800300F04E810C295AD114
:10946000002B58D003F11900764E774A013B0021BA
:10947000400080B226F813100123157088F80030E0
:1094800000F0B0FC714B032220461A702FE06648B2
:1094900003F088F80121644803F072FF6248224615
:1094A000214603F069FFAB88580725D42C68204675
:1094B00008F026FF214602465B4804F0F7F85A48B8
:1094C00004F00AF9092201238DE80C0000217F2312
:1094D000554803F0BFFB00212846FFF7E9FA0023B7
:1094E00088F8003055E7AB683146384698470BB0EE
:1094F000BDE8F08F0846FAE72B6804A8984704A84F
:1095000008F0FEFE04A90246474804F0CFF846489A
:1095100004F0E2F8D6E720460BB0BDE8F08F002457
:109520000AF8039083E70021D1543846FB69984735
:10953000FC68A4F80080002725223C238DE88400E5
:1095400041211822384803F053FBE968A879FFF756
:109550008BFB374A3E4B17701E600BB0BDE8F08F97
:109560003B490A68B21AB2F5967FD4D9304F0E60E3
:109570003E78012E00F0B480E968184601233B7064
:10958000FFF772FBB3E7304AE9791170012288F8DE
:1095900000200024C4E72A7A013A4A45BFDD09F1D8
:1095A0000104E4B2A145BAD0224E16F803B0CBEBC9
:1095B0000900C0B20021FEF7CFFF2B7A052BD94658
:1095C0001BD9CBEB0402042A40F3AE80A4F1040BB8
:1095D000BBF1000FC0F2B080063B5B45A8BF5B4605
:1095E0005FFA83F9AA791348B15C994205D000F873
:1095F000029001212846FFF75BFAC9EB0400C0B2D4
:1096000001210B4EFEF7A8FF0021342301910093A6
:109610000548317040230B223F21A14603F0E8FAB0
:109620000124AB797CE700BF1CA0FF1F84A0FF1FB3
:1096300095A0FF1F14A0FF1F959FFF1F969FFF1F60
:10964000979FFF1FC09EFF1F94A0FF1F97A0FF1FA3
:1096500080A0FF1F148BFF1FFC9FFF1F0FFA89F1D3
:10966000E868604C50F821602168049134785E49C4
:1096700004980860002C71D0012C7FF450AF5B4A35
:10968000317A88F800401170002449E7B9F1000FE1
:1096900050D009F1FF34E4B284E7B98A01F0040143
:1096A00089B200293FF440AF3B6A03929847039A7E
:1096B00000283FF43DAFAB79FC680021D15438E776
:1096C0007B8A43453CD908F101081FFA88F830E746
:1096D0003B8A43453BD208F1FF381FFA88F828E758
:1096E00025238DE8180042483C703C231822412174
:1096F00003F07EFA3046FAE6002B3FF40CAF3D4A09
:109700003D4E1188394A03F11900013B400080B2F7
:1097100026F81310012388F80030157000F062FB62
:10972000364B20461D70E2E6002A3FF755AF04F1A4
:10973000FF3B4DE74C46F3E64FF000094B4651E73F
:10974000BB8ADA077FF5F5AEB7F81080F1E6BB8A81
:10975000D9077FF5EEAEB7F81280EAE62849C85C73
:10976000C0EB090009F1010EC0B201214FF0340B2A
:1097700002F803E0FEF7F0FEB6681D4801944023AE
:109780000B223F210124CDF800B003F031FA402331
:109790000B223F211648CDF800B0019403F0AAFA3D
:1097A0002146134803F0ECFD304608F0A9FDA0EB7C
:1097B000800000F15F0109B20F220D4803F0DCFDCB
:1097C000304608F09DFD31460246094803F06EFF21
:1097D000074803F081FFE968A879FFF745FAAB79FC
:1097E0009EE600BFD4A0FF1F80A0FF1F94A0FF1F14
:1097F0001CA0FF1F809FFF1FC09EFF1F97A0FF1F81
:1098000014A0FF1F2DE9F047DFF808926D4B99F87F
:1098100000601B68DFF800A282B0003601934FF0B1
:10982000030018BF0126019F9AF8008004F00EFE85
:109830000546042004F00AFE0446052004F006FE56
:10984000800040EA4404062004F000FE2C4364B289
:109850005D4944EAC0000A7880F00F03DBB29A4207
:109860005A4A3CD01760002259480B7003788DF893
:1098700000808DF8012053B3564A12684EF66021DD
:10988000BA1A8A4219D8022B59D0012B5FD0062B65
:1098900048D0032B63D0042B69D0052B77D0072B3E
:1098A0007DD0082B00F08380092B68D016B14A4880
:1098B00002F084FF02B0BDE8F087484A484C00231C
:1098C0000121237003701360938089F800103A46D9
:1098D00069464448FFF748FD3043C6B2E6E71268E0
:1098E000BA1A1E2A6BD99AF80020934222D0394C1A
:1098F0003D488AF80030012B276082EA03020760A6
:109900009846B1D0042BAFD137480068381AB0F56B
:10991000C87FA9D9354C2068381A3228A4D92760C5
:109920001A46A1E73A4669463148FFF71DFD304324
:10993000C6B2BBE7012B4FF00002E3D1E4E73A46A1
:1099400069462C48FFF710FD3043C6B2AEE73A46F1
:1099500069462948FFF708FD3043C6B2A6E73A46F4
:1099600069462648FFF700FD3043C6B29EE73A46F7
:1099700069462348FFF7F8FC3043C6B296E73A46FB
:1099800069462048FFF7F0FC3043C6B28EE73A46FE
:1099900069461D48FFF7E8FC3043C6B286E73A4601
:1099A00069461A48FFF7E0FC3043C6B27EE73A4604
:1099B00069461748FFF7D8FC3043C6B276E7002265
:1099C00052E700BFD4A0FF1F98A0FF1F04A0FF1FF5
:1099D00094A0FF1F8CA0FF1F1CA0FF1F84A0FF1FCF
:1099E00096A0FF1F003801009CA0FF1F0CA0FF1FC6
:1099F000303C0100583701005C360100F8350100A9
:109A00009C4401004C360100B43601003C37010093
:109A1000A091FF1F148BFF1F08A0FF1F28B1102863
:109A2000044BA8BF102018607047024B012018603B
:109A3000704700BFA0A0FF1F08B5002006F010F976
:109A40000028FAD108BD00BF10B504464FF44060AD
:109A500005F01AF805F072F80A4B1B7833B96CB1AF
:109A6000102C094BA8BF10241C6010BD4FF4C0502F
:109A700004F0E0FD04F014FF002CF1D1024B0124AE
:109A80001C6010BDE69EFF1FA0A0FF1F70B50D4615
:109A90001446064605F048F8284605F045F82046E5
:109AA00005F042F8084B1B7813B1084B1B7803B93B
:109AB00070BD304604F09CFE284604F099FE204616
:109AC000BDE8704004F094BEE69EFF1FFE9EFF1F9F
:109AD00038B5164D2B78044641F6FF72A0F50050BC
:109AE000824203F1FF33A8BF02461B0202F5005277
:109AF00003F47063100443F4604343F00E0300F476
:109B0000FE005204184302F0FE42104305F0DEFF4F
:109B10002868013860F01F00C4F3C61204F07F010A
:109B2000C0B2BDE83840FFF7B1BF00BFA0A0FF1F23
:109B300070B5104E3378013B1B0203F4706304468A
:109B400043F430430806220400F0FE4043F00B03C8
:109B5000034302F4FE0018430D4605F0B7FF3068DA
:109B6000013860F04F002A462146C0B2BDE870407F
:109B7000FFF78CBFA0A0FF1F08B564210720FFF7E7
:109B8000D7FF7F210B20BDE80840FFF7D1BF00BF02
:109B900070B5104E3378013B1B0203F4706304462A
:109BA00043F410430806220400F0FE4043F009038A
:109BB000034302F4FE0018430D4605F087FF3068AA
:109BC000013860F06F002A462146C0B2BDE87040FF
:109BD000FFF75CBFA0A0FF1F38B50E4D2B78013BEF
:109BE0001B0203F47063044643F41043000443F083
:109BF000090300F4FE00184305F068FF28680138E7
:109C000060F06F002146C0B20022BDE83840FFF787
:109C10003DBF00BFA0A0FF1F10B500217B20FFF7B4
:109C200087FF0024E0B2FFF7D7FF0134022004F0E1
:109C300043FC802CF6D110BD38B50C46054604F027
:109C400073FF204604F070FF074B1B7813B1074BDE
:109C50001B7803B938BD284604F0CAFD2046BDE88C
:109C6000384004F0C5BD00BFE69EFF1FFE9EFF1FEB
:109C700038B50D4D2B78013B1B0203F4706304468D
:109C800043F45043000443F00D0300F4FE00184376
:109C900005F01CFF2868013860F02F002146C0B293
:109CA000BDE83840FFF7C8BFA0A0FF1F38B50E4D74
:109CB0002B78013B01381B02C4B203F4706320040B
:109CC00043F4404343F00C0300F4FE00184305F056
:109CD000FDFE2868013860F03F002146C0B2BDE8B3
:109CE0003840FFF7A9BF00BFA0A0FF1F38B504464A
:109CF0000D46F02004F018FF35B1254414F8010B8F
:109D000004F012FFAC42F9D1F720BDE8384004F06E
:109D10000BBF00BF00B50B4B83B002469988186893
:109D20000090032AADF8041002D903B05DF804FBDB
:109D3000684606218DF80520FFF7D8FF03B05DF8CF
:109D400004FB00BF0C45010000B50B4B024683B07D
:109D5000186899880090131F4C2BADF8041002D995
:109D600003B05DF804FB684606218DF80520FFF777
:109D7000BDFF03B05DF804FB14450100030203F4CA
:109D8000FE43C0F3C6101843704700BF0378407805
:109D9000DB0103F47E5300F07F001843704700BFDF
:109DA00082B002AA114642F8040D002012F8013BCD
:109DB00003F07F03914243EA0020F7D102B07047DD
:109DC000003210B403884FF0010404FA01F418BF04
:109DD000012202FA01F123EA04020A43028010BCC4
:109DE000704700BF70B5CEB20C46054603F0F6FED4
:109DF000864203D03146284603F00AFF0135284643
:109E000003F0ECFE240A844205D021462846BDE832
:109E1000704003F0FDBE70BD38B5054603F0DEFEB0
:109E20004FF0000460F30704681C03F0D7FE60F3F2
:109E30000F24A0B238BD00BFF8B504460020FFF7DC
:109E4000EBFF002C00F0D1854FF4AF610220FFF74B
:109E5000C9FF4FF47A610420FFF7C4FF4FF4966105
:109E60000620FFF7BFFF4FF4FA610820FFF7BAFFA3
:109E70004FF4FA610A20FFF7B5FF40F6B8310C2025
:109E8000FFF7B0FF4FF42F612220FFF7ABFF40F642
:109E9000AC512420FFF7A6FF7D212A20FFF7A2FF67
:109EA0000C210E20FFF79EFF01211020FFF79AFFE3
:109EB00002211220FFF796FF00211420FFF792FFE6
:109EC00000211620FFF78EFF02211820FFF78AFFDE
:109ED00001211A20FFF786FF01211C20FFF782FFD6
:109EE00004211E20FFF77EFF14212020FFF77AFFB8
:109EF00001212620FFF776FF03212820FFF772FFBC
:109F000004212C20FFF76EFF14212E20FFF76AFF9B
:109F100000213020FFF766FF0C213220FFF762FF9F
:109F200000213420FFF75EFF00213620FFF75AFFA3
:109F300000213820FFF756FF00213A20FFF752FF9B
:109F400000213C20FFF74EFF00213E20FFF74AFF93
:109F500000214020FFF746FF00214220FFF742FF8B
:109F60001F214420FFF73EFF13214620FFF73AFF51
:109F70000E214820FFF736FF11214A20FFF732FF5C
:109F80000A214C20FFF72EFF00214E20FFF72AFF69
:109F900006215020FFF726FF02215220FFF722FF63
:109FA0000C215420FFF71EFF00215620FFF71AFF57
:109FB00000215820FFF716FF01215A20FFF712FF5A
:109FC00008215C20FFF70EFF0A215E20FFF70AFF41
:109FD00000216020FFF706FF04216220FFF702FF47
:109FE00001216420FFF7FEFE00216620FFF7FAFE44
:109FF0000B216820FFF7F6FE7F216A20FFF7F2FEB3
:10A0000000216C20FFF7EEFE00216E20FFF7EAFE34
:10A0100000217020FFF7E6FE00217220FFF7E2FE2C
:10A0200000217420FFF7DEFE1F217620FFF7DAFE05
:10A0300013217820FFF7D6FE0E217A20FFF7D2FEFB
:10A0400011217C20FFF7CEFE0A217E20FFF7CAFEF9
:10A050001F218020FFF7C6FE13218220FFF7C2FEDA
:10A060000E218420FFF7BEFE11218620FFF7BAFEE5
:10A070000A218820FFF7B6FE00218A20FFF7B2FEF2
:10A0800000218C20FFF7AEFE00219620FFF7AAFEEC
:10A0900000219820FFF7A6FE00219A20FFF7A2FEDC
:10A0A00005219C20FFF79EFE06219E20FFF79AFEC9
:10A0B0000021A020FFF796FE7F21A220FFF792FE4D
:10A0C00040F2A461A420FFF78DFE4FF4E161A620C9
:10A0D000FFF788FE0021A820FFF784FE0021AA20B8
:10A0E000FFF780FE0221AC20FFF77CFE0121AE20AD
:10A0F000FFF778FE0121B020FFF774FE0B21B2209C
:10A10000FFF770FE6421B420FFF76CFE6421B620D7
:10A11000FFF768FE0321B820FFF764FE2C21002022
:10A12000FFF760FE0220FFF777FEB0F5805F034681
:10A1300080F03486D24A04201380FFF76DFEB0F51C
:10A14000805F034680F02186CE4A06201380FFF709
:10A1500063FEA0F52F739BB2B3F57A6F024606D962
:10A1600040F628210620FFF73DFE40F62822C64B88
:10A1700008201A80FFF750FEA0F52F739BB2B3F5AD
:10A180007A6F024606D940F6E4410820FFF72AFE1E
:10A1900040F6E442BD4B0A201A80FFF73DFEA0F5D1
:10A1A000FA739BB240F6AC518B42024606D94FF48B
:10A1B000FA610A20FFF716FE4FF4FA62B44B0C2046
:10A1C0001A80FFF729FEA0F5FA739BB240F6AC5156
:10A1D0008B42024606D940F6B8310C20FFF702FE4A
:10A1E00040F6B832AB4B0E201A80FFF715FE182848
:10A1F000034600F2C385A84A10201380FFF70CFE27
:10A20000431E9BB20F2B024604D901211020FFF7F9
:10A21000E9FD0122A14B12201A80FFF7FDFD0A285B
:10A22000034600F2A4859E4A14201380FFF7F4FD34
:10A230000128034604D900211420FFF7D3FD002391
:10A24000984A16201380FFF7E7FD7F28034600F2A7
:10A250008785954A18201380FFF7DEFD0528034601
:10A2600000F27785914A1A201380FFF7D5FD0C285C
:10A27000034600F267858E4A1C201380FFF7CCFD51
:10A280000428034600F257858A4A1E201380FFF7F0
:10A29000C3FD0928034600F24785874A2020138022
:10A2A000FFF7BAFD4628034600F23785834A22208D
:10A2B0001380FFF7B1FDA0F5FA739BB240F6AC51E5
:10A2C0008B42024606D94FF42F612220FFF78AFD08
:10A2D0004FF42F627A4B24201A80FFF79DFDA0F5E2
:10A2E000FA739BB240F6AC54A342024604D921460D
:10A2F0002420FFF777FD2246724B26201A80FFF7B5
:10A300008BFD7F28034600F201856F4A28201380C9
:10A31000FFF782FD0628034600F2F1846B4A2A20EB
:10A320001380FFF779FDA0F132039BB2B3F5967F5E
:10A33000024604D97D212A20FFF754FD7D22644B7B
:10A340002C201A80FFF768FD0C28034600F2D08409
:10A35000604A2E201380FFF75FFD1E28034600F29F
:10A36000C0845D4A30201380FFF756FD092803465C
:10A3700000F2B084594A32201380FFF74DFD1E28A9
:10A38000034600F2A084564A34201380FFF744FDB0
:10A390007F28034600F29084524C36202380FFF73A
:10A3A0003BFD7F28034600F2808438206380FFF75E
:10A3B00033FD7F28034600F271843A20A380FFF723
:10A3C0002BFD7F28034600F262843C20E380FFF7E8
:10A3D00023FD7F28034600F253843E202381FFF7AC
:10A3E0001BFD7F28034600F2448440206381FFF771
:10A3F00013FD7F28034600F235844220A381FFF736
:10A400000BFD394D28804420FFF706FD3028034618
:10A4100000F2FD83354A46201380FFF7FDFC30280B
:10A42000034600F2EE83324C48202380FFF7F4FC11
:10A430003028034600F2DF834A206380FFF7ECFCFC
:10A440003028034600F2D1834C20A380FFF7E4FCC0
:10A450003028034600F2C3834E20E380FFF7DCFC84
:10A460000128034604D900214E20FFF7BBFC00233E
:10A47000204A50201380FFF7CFFC431E3CE000BF72
:10A48000E89DFF1FB29FFF1F8E9DFF1F7C9FFF1F38
:10A49000489FFF1F549DFF1F1E9DFF1F009FFF1F12
:10A4A000349FFF1FDA9DFF1F249DFF1FEE9DFF1F9E
:10A4B000769DFF1F6C9DFF1F5C9DFF1F8E9FFF1FE2
:10A4C000FC9EFF1FF89EFF1F809FFF1F569FFF1FD0
:10A4D000AC9FFF1F3E9DFF1FD09DFF1FC09FFF1F12
:10A4E0007E9FFF1FC09EFF1FB49FFF1F929FFF1FF5
:10A4F000589FFF1F6A9DFF1F9BB20B2B024604D97A
:10A5000006215020FFF76EFC0622CF4B52201A8006
:10A51000FFF782FC0428034600F25B83CB4A5420F9
:10A520001380FFF779FC431E9BB21D2B024604D912
:10A530000C215420FFF756FC0C22C54B56201A80E4
:10A54000FFF76AFC0128034604D900215620FFF7D3
:10A5500049FC0023BF4A58201380FFF75DFC7F2889
:10A56000034600F23083BC4A5A201380FFF754FCA4
:10A57000431E9BB2092B024604D901215A20FFF742
:10A5800031FC0122B54B5C201A80FFF745FC431ECD
:10A590009BB2102B024604D908215C20FFF722FC55
:10A5A0000822AF4B5E201A80FFF736FC431E9BB299
:10A5B0001D2B024604D90A215E20FFF713FC0A2254
:10A5C000A84B60201A80FFF727FC0228034600F200
:10A5D000F482A54A64201380FFF71EFC012803467D
:10A5E00004D901216420FFF7FDFB01239F4A62206B
:10A5F0001380FFF711FCC31E9BB2012B024604D946
:10A6000004216220FFF7EEFB0422994B66201A809A
:10A61000FFF702FC7F28034600F2C982954A6820B2
:10A620001380FFF7F9FB7F28034600F2BA82924AB3
:10A630006A201380FFF7F0FB7F28034600F2AB820D
:10A640008E4A6C201380FFF7E7FB0428034600F2D4
:10A650009C828B4A6E201380FFF7DEFB192803468D
:10A6600000F28D82874A70201380FFF7D5FB022805
:10A67000034600F27E82844A72201380FFF7CCFBEF
:10A680000628034600F26F82804A74201380FFF789
:10A69000C3FB0528034600F260827D4A8A201380AE
:10A6A000FFF7BAFB0A28034600F25182794A8C2050
:10A6B0001380FFF7B1FB0428034600F24282764A7A
:10A6C00098201380FFF7A8FB0128034604D9002136
:10A6D0009820FFF787FB0023704A9A201380FFF72A
:10A6E0009BFB0128034604D900219A20FFF77AFB3F
:10A6F00000236B4A96201380FFF78EFB0B2803463E
:10A7000000F21982674A9C201380FFF785FB831EA5
:10A710009BB2032B024604D905219C20FFF762FB64
:10A720000522614B76201A80FFF776FB302803461E
:10A7300000F2FB815D4A78201380FFF76DFB302823
:10A74000034600F2EC815A4C7A202380FFF764FB29
:10A750003028034600F2DD817C206380FFF75CFB3C
:10A760003028034600F2CF817E20A380FFF754FB00
:10A770003028034600F2C1818020E380FFF74CFBC4
:10A780003028034600F2B3814A4A82201380FFF743
:10A7900043FB3028034600F2A481474C84202380E9
:10A7A000FFF73AFB3028034600F29581862063804C
:10A7B000FFF732FB3028034600F287818820A38010
:10A7C000FFF72AFB3028034600F27981A020E380BE
:10A7D000FFF722FB0128034604D90021A020FFF740
:10A7E00001FB0023354A9E201380FFF715FBC31E93
:10A7F0009BB20C2B024604D906219E20FFF7F2FAE9
:10A8000006222F4BA2201A80FFF706FB431E9BB2A5
:10A810007E2B024604D97F21A220FFF7E3FA7F2294
:10A82000284BA4201A80FFF7F7FAA0F5AF639BB27C
:10A83000B3F5167F024647D940F2A461A420FFF782
:10A84000D1FA40F2A4623FE02089FF1F5E89FF1F1A
:10A85000188AFF1FBE9DFF1F429FFF1F189DFF1FED
:10A86000648AFF1F5C89FF1FF49EFF1F509FFF1F1C
:10A870007C9DFF1F909FFF1FB09DFF1F609DFF1FCE
:10A880000C9DFF1FEE9FFF1FE09EFF1FBC9FFF1F41
:10A89000749FFF1F029FFF1FEE9EFF1F5E9DFF1F05
:10A8A000C89DFF1F3C9FFF1F429DFF1F569DFF1F1E
:10A8B000D09EFF1F589DFF1FD89EFF1F609FFF1F48
:10A8C000C489FF1F869FFF1FD44BA6201A80FFF765
:10A8D000A3FAA0F5AF639BB2B3F5167F024606D983
:10A8E0004FF4E161A620FFF77DFA4FF4E162CC4B13
:10A8F000A8201A80FFF790FA0628034600F2D980B4
:10A90000C84AAA201380FFF787FA0328034600F2FB
:10A91000CA80C54AAC201380FFF77EFA032803469D
:10A9200000F2BB80C14AB0201380FFF775FA0328FC
:10A93000034600F2AC80BE4AAE201380FFF76CFAEB
:10A940007F28034600F29D80BA4AB2201380FFF7A9
:10A9500063FA7F28034600F28E80B74AB420138042
:10A96000FFF75AFA431E9BB2C62B024604D9642154
:10A97000B420FFF737FA6422B04BB6201A80FFF7F5
:10A980004BFA431E9BB2C62B024604D96421B62063
:10A99000FFF728FA6422AA4BB8201A80FFF73CFA86
:10A9A000082862D82B88DFF8B8E2A64FA64AA74D40
:10A9B000A74EA84CA84903F0010CAEF800C0C3F3A1
:10A9C000400EA7F800E0C3F380071780C3F3C00769
:10A9D000A24A2F70C3F30017C3F34015C3F38013CB
:10A9E000378025800B801080F8BD4FF6FF739842AA
:10A9F0003FF42AAA2C283FF495AB17287FF624AA07
:10AA000019287FF68DAA1B287FF6AAAA1C283FF4D6
:10AA1000BFAA1E287FF6C4AA1F283FF4C9AA20286F
:10AA20003FF4E2AA21283FF4EBAA22283FF4F0AA3F
:10AA300023283FF4F9AA24283FF42AAB25283FF421
:10AA40002FAB26283FF430AB27283FF435AB28281E
:10AA50003FF440AB29283FF445AB2A283FF452ABE2
:10AA60002B287FF45BABFFF755BBB8200321FFF722
:10AA7000B9F9032096E70B21B220FFF7B3F90B23B6
:10AA80006BE70121AE20FFF7ADF901235CE701215F
:10AA9000B020FFF7A7F901234DE70221AC20FFF713
:10AAA000A1F902233EE70021AA20FFF79BF900232A
:10AAB0002FE70021A820FFF795F9002320E70A21BE
:10AAC0008820FFF78FF90A2380E611218620FFF7FF
:10AAD00089F9112372E60E218420FFF783F90E23F2
:10AAE00064E613218220FFF77DF9132355E61F2129
:10AAF0008020FFF777F91F2346E60A217E20FFF723
:10AB000071F90A2338E611217C20FFF76BF9112334
:10AB10002AE60E217A20FFF765F90E231CE61321A1
:10AB20007820FFF75FF913230DE61F217620FFF74A
:10AB300059F91F23FEE500219620FFF753F9002362
:10AB4000E0E500218C20FFF74DF90023B7E5002157
:10AB50008A20FFF747F90023A8E500217420FFF7BA
:10AB600041F9002399E500217220FFF73BF900230A
:10AB70008AE500217020FFF735F900237BE50021ED
:10AB80006E20FFF72FF900236CE500216C20FFF702
:10AB900029F900235DE57F216A20FFF723F97F2350
:10ABA0004EE50B216820FFF71DF90B233FE500213F
:10ABB0006620FFF717F9002330E500216020FFF73A
:10ABC00011F9002305E500215820FFF70BF90023B8
:10ABD000C9E402215220FFF705F902239EE40A216D
:10ABE0004C20FFF7FFF80A2336E411214A20FFF733
:10ABF000F9F8112328E40E214820FFF7F3F80E237B
:10AC00001AE413214620FFF7EDF813230BE41F216C
:10AC10004420FFF7E7F81F23FFF7FCBBEC9DFF1F65
:10AC2000689FFF1F1A9DFF1F949DFF1F529FFF1FCC
:10AC3000E49EFF1F689DFF1F869DFF1FA89FFF1FAB
:10AC4000D89FFF1F8C9DFF1FD29DFF1FFE9EFF1FE1
:10AC5000F69EFF1F549FFF1F069FFF1F209DFF1F93
:10AC60003E9FFF1F00214020FFF7BCF80023FFF7A5
:10AC7000C4BB00213E20FFF7B5F80023FFF7B5BBAA
:10AC800000213C20FFF7AEF80023FFF7A6BB002110
:10AC90003A20FFF7A7F80023FFF797BB00213820E1
:10ACA000FFF7A0F80023FFF788BB00213620FFF74D
:10ACB00099F80023FFF779BB00213420FFF792F8C1
:10ACC0000023FFF769BB0C213220FFF78BF80C2320
:10ACD000FFF759BB00213020FFF784F80023FFF76E
:10ACE00049BB14212E20FFF77DF81423FFF739BB51
:10ACF00004212C20FFF776F80423FFF729BB03215A
:10AD00002820FFF76FF80323FFF708BB0121262057
:10AD1000FFF768F80123FFF7F8BA14212020FFF7A6
:10AD200061F81423FFF7C2BA04211E20FFF75AF876
:10AD30000423FFF7B2BA01211C20FFF753F80123C7
:10AD4000FFF7A2BA01211A20FFF74CF80123FFF701
:10AD500092BA02211820FFF745F80223FFF782BAC2
:10AD600000211620FFF73EF80023FFF772BA0221F8
:10AD70001220FFF737F80223FFF755BA0C210E20F7
:10AD8000FFF730F80C23FFF736BA4FF47A6104204E
:10AD9000FFF728F84FF47A63FFF7D6B94FF4AF61A5
:10ADA0000220FFF71FF84FF4AF63FFF7C3B900BFEE
:10ADB000F8B5CB2006F008FD204B214A054603CB11
:10ADC0001368C5F803001A0CBA20C5F807102B80C9
:10ADD000AA70FEF7D3FF2E46002426F80B0FA0B270
:10ADE000FFF71AF8FEF7CAFF0234BA2C26F8020F52
:10ADF000F5D16C1E05F1C6064FF0FF3014F8013F87
:10AE0000082758400F4B40F300017A1E0B4012F008
:10AE1000FF0783EA5000F5D1B442EFD1C043FEF7FB
:10AE2000BFFF3A46C5F8C700CB21284604F09CFE78
:10AE30002846BDE8F84006F0CFBC00BF2045010021
:10AE40001C4501002083B8EDF0B50E4B0E4C0546B5
:10AE500093E8070085B024682E88AD7801AB83E8BD
:10AE60000700270C184600220B21ADF804408DF88E
:10AE70000670ADF80C608DF80E5004F075FE05B04C
:10AE8000F0BD00BF2C4501001C450100F0B5124B80
:10AE9000124D1E68124F0FCD87B06C460FC495E857
:10AEA000030044F8040B38683B79CDF80D00320CF0
:10AEB0002C2021808DF802208DF81130ADF8006033
:10AEC000FEF75CFF0022ADF80B001221684604F08B
:10AED0004BFE07B0F0BD00BF1C4501003845010026
:10AEE000C43D0100002004F0BBBE00BF02F02EBE36
:10AEF00070B5124C82B000254023064629462046F4
:10AF0000009301958023202201F072FE2022294621
:10AF1000204602F031FA2046012102F037FA30468D
:10AF200007F0EEF931460246204602F0BFFB20460C
:10AF300002B0BDE8704001F041BC00BF1CA0FF1F83
:10AF4000F0B5CA2983B075D90546441E00F1C6067E
:10AF50004FF0FF3014F8012F08275040404A40F3CB
:10AF600000017B1E0A4013F0FF0782EA5000F5D172
:10AF7000B442EFD1C043FEF713FF0146D5F8C70036
:10AF80000190019A914202D0B2F17F2F0BD105F1CD
:10AF90000B00FEF7FBFEBA280BD03248FFF7A8FFE4
:10AFA000002003B0F0BD3048FFF7A2FF384603B0E1
:10AFB000F0BD05F10D00FEF7E9FE2C2840D100247C
:10AFC00040F6AC5613E004281AD0062821D00828F1
:10AFD0001FD00A2828D00C2822D1A1F5FA7292B2EB
:10AFE000B24201D8FEF7FEFE0234BA2C0ED004F1B4
:10AFF0000D002844FEF7CAFE022C0146A0B2E2D1A1
:10B00000B1F5805FEED30234BA2CF0D1012003B049
:10B01000F0BDA1F52F7292B2B2F57A6FE4D8E1E7F4
:10B02000222801D0242811D1A1F5FA7292B2B2429D
:10B03000DAD8D7E70D48FFF75BFF002003B0F0BD7B
:10B040000B48FFF755FF002003B0F0BD2A28C9D1F7
:10B05000A1F1320292B2B2F5967FC5D8C2E700BF25
:10B060002083B8ED7C450100684501005045010092
:10B070009045010003290CD970B5461C82B00546E5
:10B080000C46304603222A4907F0A8F910B102B055
:10B0900070BD70470B2C05D905222649281D07F0E5
:10B0A0009DF940B12448FFF723FF244802B0BDE8D2
:10B0B0007040FFF7C9BE05F10901032201A807F09E
:10B0C000DDF901A803221E4907F088F9D8B103224F
:10B0D0001C4901A807F082F908B301A803221A4904
:10B0E00007F07CF9B0B91948FFF702FFA11E89B239
:10B0F0003046FFF725FF0028C9D0154802B0BDE84B
:10B100007040FFF7F5BE1348FFF7F2FEFFF750FE61
:10B110001148F3E71148FFF7EBFE1148C6E7114865
:10B12000FFF7E6FE02B0BDE87040FFF7AFBE00BF1C
:10B130001C450100A8450100B0450100C4450100BF
:10B14000C8450100F0450100084601000C46010019
:10B1500020460100CC450100E045010034460100D5
:10B1600048460100F44501002DE9F043174D2B68D6
:10B1700083B081460F469046F3B1154E34880A19C4
:10B1800092B218461146328006F09CFE28603A467C
:10B190004946204402F06CFDB8F1000F09D0318817
:10B1A0002868FFF767FF286806F016FB00232B606E
:10B1B000338003B0BDE8F083054E0193084631802B
:10B1C00006F002FB019B28601C46E0E7A8A0FF1FD9
:10B1D000A4A0FF1F10B51F4C4FF4FA70FBF762FDDF
:10B1E000204601F0DFF900221146204602F0C4F8A3
:10B1F0002046012102F0CAF82046002102F0C0F8E2
:10B200000B221549204602F051FA204602F064FA5A
:10B210000F221249204602F049FA204602F05CFA59
:10B220000F490722204602F041FA204602F054FA64
:10B23000204601F0C3FA0B4B0B4A1A604FF4FA7028
:10B24000FBF730FDFFF722FE0848BDE81040FFF78E
:10B250004FBE00BF1CA0FF1F4C4601005846010016
:10B2600068460100DCA2FF1F69B1000070460100C2
:10B270000020704790F8392090F83800101A704775
:10B2800090F8383090F839209A4205D95A1C034476
:10B2900080F83820187E70474FF0FF30704700BFAD
:10B2A00090F8383090F839209A4286BF1B18187EE3
:10B2B0004FF0FF30704700BF704700BF38B50546FC
:10B2C000B0F85E0090B195F85D301446C3F12102EC
:10B2D00094420CD805F13B001844224602F0C8FC09
:10B2E00095F85D30234485F85D30204638BD012057
:10B2F00014462871EEE700BFB0F85E306BB190F8ED
:10B300005D30202B07D8C218013380F85D30012052
:10B3100082F83B107047012303710020704700BF83
:10B320000023426980F8383080F8393080F85C308A
:10B3300080F85D3080F85E3080F85F3006CA30B447
:10B340000D68046943662A4383660A60A3704269F4
:10B3500090F861301649146813441D7A5B7B01EB49
:10B36000C5051B026D6803F4E06343F064032B60C2
:10B3700090F8623013449D7CDB7D01EBC5011B021C
:10B38000496803F4E06343F064030B602168536889
:10B39000194205D0036927225A70036904229A7161
:10B3A000036920225A71036980229A7030BC704769
:10B3B000A451010043690CCB12681A420CD0094B0E
:10B3C00099420AD9084B9942036994BF1A220D2267
:10B3D0005A70036904229A717047036927225A70D0
:10B3E000F7E700BF7F1A06003F420F0010B5026961
:10B3F000D378DBB2D90604463DD510215806D1706A
:10B4000038D503F0040303F0FF02002B51D03D496F
:10B41000626E00230B7084F85D30002A5BD0904789
:10B4200094F85D30002B56D02369D0229A7023699E
:10B4300094F83B201A712369012284F85C200222CF
:10B44000DA7010BD304B84F860009C424AD02F4B1C
:10B450009C4252D094F8391013791F29DBB207D8D7
:10B460002848007820B16018013184F8391003763B
:10B470000223D37010BD5906C3D4917801F0100196
:10B4800001F0FF000029DDD013F001031ED194F874
:10B490005C1094F85D00884281BF4B1C091984F848
:10B4A0005C3091F83B3013712369D0229A70226985
:10B4B000DEE7236984F83920C0229A702369114A93
:10B4C0001979012111700222DA7010BDC023937026
:10B4D00022691379CCE70122002384F85D2084F8E7
:10B4E0003B30A1E7626994F86130094913440322B3
:10B4F000187A02F043FD2269ACE7626994F8613082
:10B500000449F3E7ACA0FF1FEC91FF1F5892FF1F07
:10B5100075B5000081B500000369DB7803F02003F6
:10B5200073B190F860300133DBB2012B80F86030EA
:10B530001AD9426990F861301344187A02F09ABD22
:10B5400070B5426903F0FF0590F86130134404467A
:10B55000187A02F08FFDA36E5BB184F8385094F82E
:10B560003900BDE87040184790F85F30002BE0D0FC
:10B57000704770BD0148FFF7CFBF00BFEC91FF1FC0
:10B580000148FFF7C9BF00BF5892FF1F2DE9F047E0
:10B59000374FDFF8E0903B68026982B006460093BF
:10B5A000DDF800800021A025D3789B065BD53B68A1
:10B5B0000193019BC8EB03030F2BF5D949B1102B65
:10B5C000F2D000209070336980229A7002B0BDE8FA
:10B5D000F087726996F8613013440521187A02F0F9
:10B5E00043FF726996F861301344012193F812A069
:10B5F000504602F039FF09240021504602F020FF96
:10B600002B46013BFDD10121504602F019FF2B468C
:10B61000013BFDD1013CEFD1706996F86110014406
:10B620004FF4A0720C7A4B7B09EBC4011B024968F2
:10B6300003F4E06343F064030B6096F86230034464
:10B64000997CDB7D09EBC1011B02496803F4E063CF
:10B6500043F064030B60013AFDD13269D3789B0655
:10B660004FF00101A3D4012002B0BDE8F08700BF74
:10B67000D4A0FF1FA4510100F0B503691222DA70B3
:10B680000269937803F0200385B004460D46002B31
:10B690005ED0B42393703C4922690B680093009EEE
:10B6A00005E00B680193019B9B1B042B42D8D378C8
:10B6B00003F0200303F0FF00002BF2D094F85D307C
:10B6C000002B31D04FF0000E4FF0020C04EB0E03B4
:10B6D00093F83B3013710B680393039F206907E0D5
:10B6E0009B060DD50B680293029BDB1B052B28D80C
:10B6F000C378DBB203F0020202F0FF06002AEFD0AB
:10B7000080F803C02669F378DBB2DF0632462DD419
:10B710009F062BD5DB0731D40EF1010E94F85D3076
:10B720005FFA8EFE7345D1D800201DBB002384F83C
:10B730005E3004E09070236980229A70042005B086
:10B74000F0BD86702369802204209A7005B0F0BD98
:10B7500003F0FF06FFF71AFF10B9042005B0F0BD93
:10B76000236984F85F60B0229A7094E78023B370F5
:10B770000420DAE726698023B370D7E7BEF1000F13
:10B780000CBF02200320F6E7D4A0FF1F2DE9F041F3
:10B7900006690025122780F8385080F83950F77074
:10B7A000D0F810C09CF802E00EF0200E88B00446DD
:10B7B000884615461E46BEF1000F49D0B4238CF8CA
:10B7C0000230784B21691A680092DDF800E006E04B
:10B7D0001A6801920198CEEB0000042830D8C8788E
:10B7E00000F0200000F0FF070028F1D04FEA4802E7
:10B7F00042F00102D2B20A711A680292DDF808E042
:10B80000206906E01A6803920399CEEB010105292D
:10B810002AD8C17801F0020101F0FF070029F1D018
:10B820004FF0020C80F803C02269D17811F01107A3
:10B8300022D12DBB002E0CBFA0238023937003E0E8
:10B840008F70236980229A70384608B0BDE8F08175
:10B850000EF0FF07FFF79AFE0028F5D0236984F861
:10B860005F70B0229A70ACE78770236980223846F7
:10B870009A7008B0BDE8F081802393700027E3E759
:10B88000012D75D0A021917021690A79BE466746C5
:10B890004FF0A80C1A680492049805E01A68059203
:10B8A000059A121A052A4AD8CA7802F0020202F052
:10B8B000FF08002AF2D0CF702169CA78D2B212F004
:10B8C000100F08465AD1920658D5013DEDB2012D10
:10B8D00049D0BEF11F0F3BD90A79012DDAD11A6880
:10B8E0000692069D05E01A680792079A521B052AE0
:10B8F00046D8C27802F0020202F0FF01002AF2D01C
:10B900000223C3702269D378DBB2D9063AD49B06EE
:10B9100034D5B023BEF11F0F93703FD8226904EBDA
:10B920000E0312791A760EF1010E5FFA8EFE16B131
:10B93000236980229A7084F839E0774684E781F899
:10B940000280236980229A70774684F839E07BE789
:10B9500004EB0E0291F8048082F818800EF1010EBB
:10B960005FFA8EFEB9E781F802C021690846B0E7A8
:10B97000A82191702069BE460279B0E7774663E757
:10B980008170DEE71021A023D170013BFDD1226937
:10B99000937803F0F7037746937055E723691B7993
:10B9A000C5E700BFD4A0FF1F0148FFF71FBD00BFC0
:10B9B000EC91FF1F0148FFF719BD00BF5892FF1F10
:10B9C000704700BF38B5144C037801225B00054670
:10B9D000204684F83B3084F85E2084F85D20FFF731
:10B9E0008BFC20460021FFF747FE0B4C29780123F2
:10B9F00020461A46FFF7CAFE0128F6D194F83830DF
:10BA000094F839209A4205D9E218013384F8383085
:10BA1000107E38BDFF2038BDEC91FF1F38B51B4CA0
:10BA2000037801225B000546204684F83B3084F809
:10BA30005E2084F85D20FFF75FFC20460021FFF7C1
:10BA40001BFE124C2978204601230222FFF79EFE9E
:10BA50000228F6D194F8382094F839108A420FD28F
:10BA6000531CDBB2A018994284F83830007E0AD902
:10BA7000234402321B7E84F8382040EA032038BD7C
:10BA80004FF6FF7038BD40F47F4038BDEC91FF1F8A
:10BA90000C2901D9002070470231490001F0FE0154
:10BAA000FFF7BCBF70B50C4C0378164601255B0050
:10BAB000204684F83B3084F85E5084F85D50FFF7F0
:10BAC0001BFC31462046FFF717FC29462046BDE8FF
:10BAD0007040FFF7D1BD00BFEC91FF1FF8B50546E0
:10BAE0000F461646412421463A462846FFF7DAFF1C
:10BAF000611C0234C9B232462846E4B2FFF7D2FFD5
:10BB0000592CF0D1F8BD00BF38B504460D46354874
:10BB1000FFF706FC6322802120462570FFF7C2FF55
:10BB2000012002F0C9FC204600225E21FFF7BAFF87
:10BB300020465D21FFF746FF242801D0002038BDB4
:10BB4000204606220C21FFF7C9FF204601222B21A7
:10BB5000FFF7A8FF204601222C21FFF7A3FF204674
:10BB60000E222D21FFF79EFF204600222E21FFF7F7
:10BB700099FF204601222F21FFF794FF204605223E
:10BB80003021FFF78FFF204601223121FFF78AFF86
:10BB9000204600223221FFF785FF20460022332174
:10BBA000FFF780FF204600223421FFF77BFF20466D
:10BBB00000223521FFF776FF204600225B21FFF7A8
:10BBC00071FF204610225C21FFF76CFF20462022E7
:10BBD0005D21FFF767FF20468F225E21FFF762FF9E
:10BBE000012038BDEC91FF1F10B4047F4160022C8E
:10BBF000C26002D010BC01F0D7BB836810BC1847EC
:10BC000090E80C00F0B41C6859682568164F174E70
:10BC100029432160164D17491760D66015611160E0
:10BC2000417A154A5C180A3194F8244053F821509F
:10BC300002EBC40149680D60017A5C1803EB8101D5
:10BC4000247ECD6902EBC40149680D60817A5818E1
:10BC500003EB810390F83000596B02EBC002F0BC9B
:10BC600053681960704700BF01401F000110003881
:10BC70000110007800001F80A4510100704700BF30
:10BC8000F0B50C1EBDF8146034DBB0F9067019195C
:10BC9000B942C4BF3B1B1BB2002BA6461CDD002AC9
:10BCA0001146B8BFD11D02F00705CC10826A0120F1
:10BCB00007FB04E1A840012E0A44C0B21ED00CD3F9
:10BCC000022E09D1013B12FA83F3013A12F8011F47
:10BCD00041409A421170F9D1F0BDC043013B12FAC4
:10BCE00083F3C0B2013A12F8011F01409342117070
:10BCF000F9D1F0BD23441BB20024C6E7013B12FA80
:10BD000083F3013A12F8011F01439A421170F9D1ED
:10BD1000F0BD00BFF8B50D1E0EDB14461F460646EB
:10BD200001F03AFBA84207DD002C05DB304601F0AC
:10BD300037FBA04201DCF8BDF8BD304601F02AFB1C
:10BD4000022853D003284BD0012806D16540F38840
:10BD50006C406540013B5D1B2DB2012F03D02AD3FF
:10BD6000022F14D0F8BD002C2246B6F90630B06A76
:10BD7000B8BFE21D42F3CF0202FB035504F00704F3
:10BD8000435D012101FA04F41C434455F8BD002C25
:10BD90002246B6F90630B06AB8BFE21D42F3CF02C0
:10BDA00002FB035504F00704435D012101FA04F48A
:10BDB0005C404455F8BD002C2246B6F90630B06A06
:10BDC000B8BFE21D42F3CF0202FB035504F00704A3
:10BDD000435D012101FA04F423EA04044455F8BD4B
:10BDE0003389013B591B25460CB2B6E7F1883289ED
:10BDF0000139013A4D1B141B2DB224B2ADE700BF2F
:10BE00002DE9F041079E9DF91880089D04461F46C4
:10BE100000F0C0FF0D4B0E480E4984F83380FF221E
:10BE2000002F08BF1F4684F82F20002384F83020FD
:10BE300084F8312084F832202060A665E5656762C9
:10BE400061652362A3622046BDE8F081EC91FF1F8B
:10BE5000FC4601000110013810B50446806A034B0E
:10BE6000236008B105F0B8FC204610BDFC46010077
:10BE7000F8B5436ADBB190F82C200125AA4083F87D
:10BE80003B2083F85E5083F85D500446406A0368A7
:10BE90000E461B6800219847606A036831461B689C
:10BEA00098472946606ABDE8F840FFF7E5BBC26BDA
:10BEB000C56C1368046A23EA050313604CB1226859
:10BEC0004FF00043D3625163D36A002BFCDA936BCB
:10BED000F8BD836B466B0825802410E03768426C00
:10BEE0003A4332601F68826C3A431A601A68876C62
:10BEF000013D22EA07024FEA54041A6007D02142AA
:10BF0000ECD13268476C22EA07023260EAE7F8BDFA
:10BF100070B50446406A0D4600282BD0A16DFFF78E
:10BF200049FA002D20460CBFA621A721FFF7A0FF4C
:10BF3000606A20B1E16DBDE87040FFF73BBA216C4B
:10BF4000226D0868236A02430A6093B1DA7A82B1EB
:10BF5000D00703D5224A99691160DA7A910703D58F
:10BF6000204AD9691160DA7A520702D51E4A1B6A43
:10BF7000136070BD236A002B2BD0D97A626DE1B1BA
:10BF800072B6D97ACE0706D51848D9680668314006
:10BF900099610160D97A880706D51548196906683C
:10BFA0003140D9610160D97A4E0705D511485969E8
:10BFB000066831401962016062B61B68D968914217
:10BFC00007D00D4818600D49DA6042F080401861D2
:10BFD0001960226C216D136823EA01031360A0E746
:10BFE00000E100E004E100E008E100E080E100E0C1
:10BFF00084E100E088E100E001403F0000003F8074
:10C00000436A2DE9F04105460E469046002B3ED08E
:10C0100090F82C100124A14083F83B1083F85E4077
:10C0200083F85D40406A036800211B6808F1FF3710
:10C030009847FFB2B8F1000F23D03744A046013E25
:10C04000686A16F8011F03681B6898470134B742F5
:10C05000E4B216D0202CF3D10121686AFFF70CFB63
:10C0600095F82C206B6A520083F83B2083F85E80A1
:10C0700083F85D80686A036800211B689847012483
:10C08000DEE7686A0121BDE8F041FFF7F5BAC26B4F
:10C09000C16C136823EA010306EB080413604FF038
:10C0A0000048A6420ED02B6A16F801EB63B11A685D
:10C0B000C2F82C80C2F834E0D36A002BFCDAA64226
:10C0C000936BF0D1BDE8F081AB6BD5F834C008209C
:10C0D0008021DCF800206F6C1EEA010F14BF3A4388
:10C0E000BA43CCF800201A68AF6C3A431A601A6859
:10C0F000AF6C013822EA07024FEA51011A60E8D119
:10C10000CFE700BF70B50446406A0D46002828D02E
:10C11000A16DFFF74FF920462946FFF7A9FE606A97
:10C1200020B1E16DBDE87040FFF744B9216C226D8C
:10C130000868236A02430A6093B1DA7A82B1D007B1
:10C1400003D5234A99691160DA7A910703D5214A08
:10C15000D9691160DA7A520702D51F4A1B6A136047
:10C1600070BD236A002B2BD0D97A626DE1B172B613
:10C17000D97ACE0706D51948D96806683140996141
:10C180000160D97A880706D51548196906683140D3
:10C19000D9610160D97A4E0705D5124859690668F8
:10C1A00031401962016062B61B68D968914207D0BC
:10C1B0000D4818600D49DA6042F08040186119603E
:10C1C000226C216D136823EA01031360A3E700BF0B
:10C1D00000E100E004E100E008E100E080E100E0CF
:10C1E00084E100E088E100E001403F0000003F8082
:10C1F0002DE9F041044686B0806A9DF830801E46E5
:10C200000F461546B4F90830002800F04281DA1DC7
:10C2100048BF03F10E02B4F90630D21003FB02F25C
:10C22000002105F0FDFDB4F90820202A00F39280DA
:10C23000B4F90610A34B0120203A733902EBD272F5
:10C2400001EBD1714FF0200E029073208DE8014078
:10C2500042F34F0241F34F01204600F051FE606A65
:10C2600084F82D70002800F04D81002D40F08A8068
:10C27000B4F90830202B14BF3D253C2584F82C5000
:10C28000B8F1000F40F0858006B394F93300002820
:10C2900018DBC0B2012102F0E7F8012194F8330065
:10C2A00002F0CEF8012002F007F9002194F83300E3
:10C2B00002F0C6F80A2002F0FFF8012194F83300DA
:10C2C00002F0BEF8606A002800F08280A16DFFF7DE
:10C2D00071F804227C492046FFF792FE217A013949
:10C2E000C9B22046FFF7C4FD784904222046FFF773
:10C2F00087FE94F92D30012B14BF14211021204604
:10C30000FFF7B6FD042272492046FFF779FEB4F923
:10C310000630802B00F09280602B00F0A680D9219F
:10C320002046FFF7A5FD94F92D30012B14BFF12114
:10C3300022212046FFF79CFD204606226549FFF793
:10C340005FFE606A50B3E16DFFF734F8012006B07C
:10C35000BDE8F081B4F906105F4B0120403A523934
:10C360004FF0400E029002EBD272522001EBD171DD
:10C370008DE8014042F34F0241F34F01204600F0A7
:10C38000BFFD6CE76DB284F82C50B8F1000F3FF49C
:10C390007BAFFEF7C5FF002E94D076E7216C226DAF
:10C3A0000868236A02430A6073B1DA7A62B1D0077F
:10C3B00003D54A4A99691160DA7A91077CD4520709
:10C3C00002D5474A1B6A1360012006B0BDE8F08120
:10C3D000236A002B2BD0D97A626DE1B172B6D97A7B
:10C3E000CF0706D53F48D9680568294099610160A3
:10C3F000D97A8E0706D53C48196905682940D96164
:10C400000160D97A4D0705D5384859690568294032
:10C410001962016062B61B68D968914207D034483E
:10C4200018603449DA6042F0804018611960226C6B
:10C43000216D136823EA010313604AE7B4F9083059
:10C44000202B00F08680402B7FF469AF2A492046DC
:10C450000322FFF7D5FD94F92D30012B14BFCF2116
:10C460009F212046FFF704FD59E7B4F90830102B4F
:10C470007FF455AF214920460322FFF7C1FD94F90F
:10C480002D30012B14BFAF2110212046FFF7F0FC07
:10C4900045E7DA1D48BF03F10E02B4F90630D210A9
:10C4A00003FB02F21046059205F08EF9A062002807
:10C4B0003FF44DAF059AB3E6114AD9691160DA7AB3
:10C4C0007DE700BF544701003449010038490100AD
:10C4D0003C490100404901004849010000E100E0F9
:10C4E00008E100E080E100E084E100E088E100E0B4
:10C4F00001403F0000003F8050470100084C010010
:10C5000004E100E0012194F83100244F01F0ACFF78
:10C5100094F83200012101F0A7FF94F9312094F939
:10C52000323057F83220E26357F83330206A236400
:10C530000125E56425651A682A431A6078B1B8F1C7
:10C54000000F3FF428AFFFF75BFB002E3FF4BAAEBD
:10C550009BE6042212492046FFF752FDDFE62946FA
:10C5600094F82F0001F080FF294694F8300001F084
:10C570007BFF94F92F2094F9303057F83220626312
:10C5800057F833306564A5641A68A36322F001028A
:10C590001A60002E3FF496AE77E600BFA45101006A
:10C5A0004C470100B0F90820D31D48BF02F10E032B
:10C5B000B0F90620806ADB1002FB03F2002105F0CF
:10C5C0002FBC00BFF0B50029BDF814502EDBB0F928
:10C5D0000660B1422ADA002A59DBB0F90870144625
:10C5E0001C44BC42C4BFBB1A1BB2002B1EDDD2B21E
:10C5F000D408D0F828E016FB041112F00702DBB2D1
:10C600000EEB010421D0C2F10807FAB2374F934272
:10C61000BF5C0CD2C3EB020CFF2646FA0CF6012DD0
:10C6200007EA06073FD005D3022D36D0F0BD012D15
:10C6300039D030D21EF8016026EA07070EF80170E3
:10C640009342F3D3B0F906100C449A1AD2B2072AD7
:10C6500010D9022D36D0002D14BFFF260026134618
:10C660002670083BB0F90610DBB2072B0C44F7D854
:10C6700002F00702002AD9D01D4B012D9B5C1DD072
:10C6800017D3022DD2D1227853402370F0BD13442A
:10C690001BB20022A1E7022D25D11EF801607740D0
:10C6A0000EF80170CCE71EF8016037430EF80170F8
:10C6B000C6E7227822EA03032370F0BD22781343F1
:10C6C0002370F0BD11462378DB4323700839B0F99D
:10C6D0000630C9B207291C44F5D812F00702A5D0CC
:10C6E000034B9B5CCFE73444AFE700BFEC4601004F
:10C6F000DC46010070B4C47DBDF80C50022C18D08B
:10C70000032C1FD0012C0BD0002A03DBB0F908400A
:10C71000944201DC70BC7047039570BCFFF7B0BA5F
:10C72000C4880395013CA41A0A4621B270BCFFF7E5
:10C7300049BF0689C488013E641AB21AE41A12B2CB
:10C7400021B2E1E704890395E41A641A114622B282
:10C7500070BCFFF737BF00BF70B4C57DBDF80C607B
:10C76000022D1AD0032D12D0012D03D0039670BCD8
:10C77000FFF728BFC488E41AA41A0A4621B2002A87
:10C7800003DBB0F90840944213DC70BC70470489A5
:10C79000013C641A114622B2F1E7C4880589039668
:10C7A000013CAD1AED1A621A11B22AB270BCFFF741
:10C7B00009BF039670BCFFF763BA00BF2DE9F843C9
:10C7C0000446406A002863D0A16DFEF7F3FD052200
:10C7D00074492046FFF714FCA1790139C9B22046FB
:10C7E000FFF746FBB4F90820E588A66AD31D48BFC9
:10C7F00002F10E03DB10626A15FB03F51FFA85F8E0
:10C80000002A7BD094F82C300125AB4082F83B30D5
:10C8100082F85E5082F85D50606A036840211B68B0
:10C8200008F1FF379847BFB2B8F1000F23D0374463
:10C83000A846013E606A16F8011F03681B68984706
:10C840000135B742EDB216D0202DF3D10121606A37
:10C85000FEF712FF94F82C20636A520083F83B2005
:10C8600083F85E8083F85D80606A036840211B68FE
:10C8700098470125DEE70121606AFEF7FDFE606A48
:10C88000002800F08D80E16DBDE8F843FEF792BD11
:10C89000236A002B2BD0D97A626DE1B172B6D97AB6
:10C8A000CE0706D54048D9680568294099610160DE
:10C8B000D97A8D0706D53D48196905682940D9619F
:10C8C0000160D97A480705D5394859690568294072
:10C8D0001962016062B61B68D968914207D0354879
:10C8E00018603549DA6042F0804018611960226CA6
:10C8F000216D136823EA0103136068E7E26BE36CC0
:10C900001168276A0B4306EB080913604FF0004ECD
:10C910004E450DD016F801CB2FB33A68C2F82CE083
:10C92000C2F834C0D36A002BFCDA4E45936BF1D1C8
:10C93000226C236D11680B43136097B1FB7A83B1AE
:10C94000D90703D51D4BBA691A60FB7A9A0703D53C
:10C950001B4BFA691A60FB7A5B0702D5194B3A6ADE
:10C960001A60BDE8F883A36BD4F8348008208021D6
:10C97000D8F80020656C1CEA010F14BF2A43AA43B3
:10C98000C8F800201A68A56C2A431A601A68A56CBA
:10C99000013822EA05024FEA51011A60E8D1B7E7EF
:10C9A000276AC5E7E446010080E100E084E100E099
:10C9B00088E100E001403F0000003F8000E100E02E
:10C9C00004E100E008E100E02DE9F04F85B0994670
:10C9D000BDF93870BDF83CA0BB1AC1EB090B002BA8
:10C9E000B8BF5B42BBF1000FB8BFCBF1000B5B459A
:10C9F0000D4616460093804648DC4D453A46334680
:10CA00004CDC194613460A46C5EB09019B1A89B24C
:10CA1000002B0CB2B8BF5B4204EBD474BE42ACBF77
:10CA20004FF0FF3201224D45039102924FEA640418
:10CA300029DC9BB201930DE0D8F80070BF69B847BC
:10CA4000019BE41AA3B21CB20135002C2DB211DBFC
:10CA5000A94518DB009B5B452A46534631464046B4
:10CA6000EADCD8F80020534697692946324640460A
:10CA7000B847E5E7029A1644039AA94502EB030476
:10CA800036B224B2E6DA05B0BDE8F08F4A462B464E
:10CA9000B94635464D4517461E46B2DD3046294655
:10CAA0003E464D4607468946AEE700BF10B40468CF
:10CAB0002469A44610BC604730B40468BDF808502F
:10CAC0000295A46BA44630BC604700BF30B4046834
:10CAD000BDF808500295E46BA44630BC604700BF27
:10CAE00070B40468BDF90C60BDF81050039604954D
:10CAF000246CA44670BC6047704700BF10B582B07C
:10CB0000B0F90C2001910168009200220C6CB0F980
:10CB10000A301146A04702B010BD00BF704700BFE9
:10CB200001F003010129C17506D0032904D0C28890
:10CB300003894281838170470289C388428183814E
:10CB4000704700BF2DE9F0410568134E6F6986B04C
:10CB5000B7420446BDF8308010D1013B13441BB2EC
:10CB60000093CDF804800B46AD6A2046A8472368A1
:10CB7000DB6AB3420AD106B0BDE8F08105930492A6
:10CB80000391B84703A925680EC9E6E7204606B019
:10CB9000BDE8F041184700BFF9CA00002DE9F04197
:10CBA0000568124E6F6986B0B7420446BDF8308002
:10CBB0000FD1013BCDF804800B4400921BB2AD6A4B
:10CBC0002046A8472368DB6AB3420AD106B0BDE815
:10CBD000F081059304920391B84703A925680EC913
:10CBE000E7E7204606B0BDE8F0411847F9CA000063
:10CBF0002DE9F04F0568DFF858B06F6985B05F45E3
:10CC00000646BDF93890BDF83CA00C46904615D1BB
:10CC10001F19BC420CDACDF800A0214601342D6A60
:10CC20004B464246304624B2A847BC423568F2DB48
:10CC3000EB6A5B4507D105B0BDE8F08F0393B847B9
:10CC40003568039BE4E7304605B0BDE8F04F184770
:10CC5000F9CA00002DE9F04387B099420546BDF9B5
:10CC60003840BDF83C6025D0A24212D00768DFF8FA
:10CC70008080D7F81490C14532D18DE85000284605
:10CC8000BC6AA0472B68DB6A434524D107B0BDE8E6
:10CC9000F083994202DD08461946034628680E963D
:10CCA000C46B01335B1A1BB22846A44607B0BDE82B
:10CCB000F0436047A24202DD134622461C46286824
:10CCC0000E96631C846B9B1A1BB22846A44607B0C1
:10CCD000BDE8F0436047284607B0BDE8F043184779
:10CCE000059304920391C84703A92F680EC9C4E7AE
:10CCF000F9CA00002DE9F04FD0F800E0DFF890907D
:10CD0000DEF814B083B0CB450446BDF93080BDF8E1
:10CD100034A00D4617461E4631D1CDF800A0DEF8EE
:10CD200024B0294633463A462046D8472368CDF8F2
:10CD300000A008F1FF323A44D3F824B0294612B2D9
:10CD400033462046D8472368CDF800A02946D3F8BB
:10CD500020B03A4643462046D8472068CDF800A088
:10CD6000711E29444346056A09B23A462046A8473F
:10CD70002368DB6A4B4506D103B0BDE8F08FD84786
:10CD8000D4F800E0C9E7204603B0BDE8F04F1847EB
:10CD9000F9CA0000F0B4002401264FF6FF75094FD0
:10CDA00007600471C475C48104824476C4618675C9
:10CDB000067685824582C180028141818281F0BCF4
:10CDC000704700BF144C01002DE9F04F85B0066894
:10CDD000BDF84450BDF93880CDF800800446019577
:10CDE000D6F848B00392BDF93C60BDF94070894661
:10CDF0009A46D84723680195009742465146D3F892
:10CE0000488020463346C0472068039B0E930F9509
:10CE1000856C4B463A4631462046AC4605B0BDE8E7
:10CE2000F04F60472DE9F04F87B01746BDF94040FD
:10CE300000912546E91D059344BF2B4603F10E01E1
:10CE40000268BDF8486053690294C91003912B49E8
:10CE5000BDF9444001968B42824645D1002C3CDD11
:10CE6000029B3C445E1EB6B24FF0000923B204930D
:10CE700001364D46029B002B28DD059B002403EB69
:10CE8000090806E0EDB22B0604F1010411D4A64214
:10CE90001CD0A1B211F0070F23B24FEA4505F1D122
:10CEA000002BB8BF0733DB10013418F803502B06F2
:10CEB000EDD5009BD2F818B019443A4609B2019B4F
:10CEC0005046D847A642DAF80020E2D1039B01374A
:10CED0009944049B3FB2BB42CCD1D36A074A9342E8
:10CEE00006D107B0BDE8F08F9847DAF80020B5E723
:10CEF000504607B0BDE8F04F184700BFF9CA000020
:10CF000070B4BDF90C60BDF91050BDF81440039623
:10CF10000495059470BCFFF785BF00BF2DE9F04F65
:10CF200093B090460591C1691090BDF870000790CC
:10CF3000BDF874909DF878A00493002900F0CD808E
:10CF40000A7A0AC9894604998A1AD2B203EBC20343
:10CF5000BAF1010FDA780B9293F905201E8893F845
:10CF600002B00F9293F9064079D913B2099323B214
:10CF70000C93109B1A68A94B1193194653698B4265
:10CF800040F0A6800B9B002B55D01FFA88F30021A0
:10CF90000D93C8462344DDF8409006910E930F464A
:10CFA0000C46BBF1000F3FD0BDF818100C9B039747
:10CFB0001FFA8AF0CB1813FB00F304900E9801447B
:10CFC0000D98034409B21BB20A910893002505E0AD
:10CFD0000135EBB264009B45E4B222D9039B2B449C
:10CFE000590703D1731C18F806409EB22306EFD5EB
:10CFF000099BBDF81000E91811FB00F10598BAF182
:10D00000010F0FFA8AF301441CD007980190009396
:10D01000D26909B217464846089AB847D9F800209D
:10D02000D6E7039F5F44FFB2069B0B99013306933B
:10D03000DBB29942B5D8D36A119A934243D113B067
:10D04000BDE8F08F0F9B191893690A9A29441F466F
:10D0500009B2079B4846B847D9F80020B8E7002333
:10D060000C93099385E70A9A0D9B0132013B52B25A
:10D0700013F0FF030A920D936FD1DDF81890079B10
:10D08000DDF83C80DDF820A04B4517D0BAF1010F48
:10D0900000F0C8800B9A109DCDF804900BEB8B012B
:10D0A0004FEACB030A4400931146DEF81C40534676
:10D0B000424609B22846A047D5F800E0DEF82C30F9
:10D0C000119A9342BBD0109813B0BDE8F04F1847A7
:10D0D000109D284698472A6854E7109A0598B2F997
:10D0E0000A308342ABDDB2F90C304345A7DD06239D
:10D0F00013FB0A03002BA2DD08EBCA03002B9EDD05
:10D10000537E2BB9049BAF2B02D90133DBB20493BE
:10D11000109BD3F800E0414B11931A46DEF814300F
:10D12000934240F08E801FFA88F30E9308339BB22F
:10D13000BDF81420059305230D9300230A93CDF821
:10D140003C800FFA8AF3DDF84080CDF818900B92FE
:10D150001FFA8AFBCDF820A099460A9ABDF8100064
:10D160000B9C0E9D0523194611FB00232C481146EC
:10D17000C75C039702FB0B4214FA81F312B21BB295
:10D1800009920C932C462E461CE0089B0999012B12
:10D190002AB24B4640462DD0079F0197CDF800900C
:10D1A000DEF81CA0D047D8F800E0039B5B080134F0
:10D1B0000393059BA4B25D445E44A342ADB2B6B2F4
:10D1C0003FF451AF039BD807DFD4079B069A9342E5
:10D1D000EBD0089B012B16D0069B0193CDF8009055
:10D1E000DEF81CA009994B4632B24046D047D8F829
:10D1F00000E0DAE7DEF818A0079B0C9922B2D047CE
:10D20000D8F800E0D1E7DEF818A00C9913464046A4
:10D2100022B2D047D8F800E0C7E700BFF9CA000043
:10D22000644C01000B99109DCDF800900531DEF89B
:10D23000204009B2424608232846A047D5F800E01E
:10D240003CE7109C20469847D4F800E06BE700BF0D
:10D25000F0B5C36985B004462BB30A2968D00D29FF
:10D260004AD01A7A914247D3587A884244D35D68AB
:10D270008A1A05EBC205AA78002A50D0E87800285F
:10D280004DD0207E00283AD095F905E0B4F90E0083
:10D29000A67DB4F90A70724406FB0202BA4262DC4F
:10D2A000B4F9102030E00A2956D00D2924D0027E8E
:10D2B000002A4BD0B0F90E00A57DB4F90A60062211
:10D2C00012FB0502B2423EDD228AE38102EBC50277
:10D2D00012B218462282A78A668A02950B468DE80A
:10D2E000C00001462046FFF719FEA37DE28903EB4B
:10D2F000430302EB4303E381012005B0F0BDA67DAB
:10D30000B4F90E00B4F91020B4F814E0678A02965C
:10D310000B468DE8804001462046FFF7FFFD297946
:10D32000E389A27D012001FB0233E38105B0F0BD5A
:10D330000022C2819A7A817D038A01FB0233038233
:10D34000012005B0F0BDB4F91020C4E7857DB4F923
:10D350001020B0F90E00BEE7028A817DC38102EB86
:10D36000C1030382C8E70020E0819B7A228A03FB85
:10D37000062212B22282C7E7C1810282704700BF33
:10D38000002908BF01218175704700BF8182418259
:10D39000704700BFC07D7047B0F90A00704700BFFA
:10D3A000B0F90C00704700BF10B4EFF3108272B6F2
:10D3B000437F33B9017F012907D003290FD001230F
:10D3C000437702B962B610BC7047124C2168A1B114
:10D3D000114943610B68836108605861EFE70F4CA6
:10D3E000216881B10E4943610B688361086058610F
:10D3F0000C4B4FF080511960E1E7074B41618161AF
:10D4000020601860DBE7064B416181612060186095
:10D41000EEE700BFC0A0FF1FBCA0FF1FB0A0FF1F12
:10D42000B4A0FF1F04ED00E070B5EFF3108272B6F8
:10D430000C4C206880B10C4E00254369236073B109
:10D440009D6102B962B6457783689847EFF3108211
:10D4500072B620680028F0D102B962B670BD3360A0
:10D46000EFE700BFB0A0FF1FB4A0FF1FFFF7DCBFB6
:10D47000184A30B41468002C27D0036821688B4206
:10D480000ED2CB1A00218460C1602360E06010607E
:10D490000223037530BC704711688B42144608D3D1
:10D4A000A2685B1A0360002AF6D18260C460A060A3
:10D4B000EEE7D268C2608460E060C568CB1A0222E1
:10D4C000A8602360027530BC70478460C46010603F
:10D4D000DEE700BFB8A0FF1FF8B5224E34682CB3BA
:10D4E0002368002B3AD1204F1D4604E03468ECB18C
:10D4F0002368002B32D1A36803B1DD60206933605B
:10D50000036825751B68BB4221D1037F4560022B50
:10D51000C46020D0FFF748FF6368002BE6D023608B
:10D520002046FFF7A5FF3468002CE1D1EFF310830C
:10D5300072B60E4A00211068116003B962B628B1B4
:10D540008468FFF795FF20460028F9D1F8BD2246F0
:10D5500000219847E0E783689847DDE7013B2360B7
:10D56000E4E700BFB8A0FF1FE9BB0000C8A0FF1F91
:10D57000024A136801331360FFF7AEBFD4A0FF1F48
:10D58000704700BF0368F0B4FBB1002501249D6023
:10D59000DC601B4C1A601C44241104F144056A1120
:10D5A000032692009E60174F0679174B47F8241008
:10D5B00002F1604202F5614205F01F05012000FA08
:10D5C00005F5E6541560F0BC7047104C236843F431
:10D5D0000003236000BF0E4B0E4DA4F58734A4F565
:10D5E0009E7401261E60234604609C68002CD0D0E7
:10D5F0001033AB420360F8D1002303601846E2E722
:10D60000008FFCBFC492FF1F44E400E03C80044054
:10D6100000700340407103400168A9B10B4BF0B4A6
:10D620000B441B110A4E0B4F0B4D46F8237003F1B0
:10D63000440202F01F0401235211A340002445F8C4
:10D6400022308C600460F0BC704700BF008FFCBFCC
:10D65000C492FF1F81D5000080E100E0024A034B25
:10D66000012111601B6818470C710340C492FF1F11
:10D67000024A034B012111605B6818471C7103408B
:10D68000C492FF1F024A034B012111609B68184797
:10D690002C710340C492FF1F024A034B0121116009
:10D6A000DB6818473C710340C492FF1FF8B50E4673
:10D6B00071B17AB10746144600253B6816F8011B84
:10D6C0001B6838469847013C0544F6D12846F8BD0A
:10D6D0000846F8BD1046F8BD00B5064A0368128832
:10D6E0005B6883B001A9ADF804200222984703B01B
:10D6F0005DF804FB64510100F0B507468BB0002AC9
:10D7000033D0012A08BF0A2251B3212400E0F4B229
:10D71000B1FBF2F502FB1511C8B2092900F1300185
:10D7200098BFC8B20AA988BF3730214488BFC0B2A9
:10D7300001F8240C661E2946002DE8D133B1013CC6
:10D74000E4B20AAB23442D2203F8242C3B6801AA3F
:10D7500011195B683846C4F1220298470BB0F0BD3E
:10D7600030228DF825202124E8E70368C9B21B6820
:10D7700098470BB0F0BD00BF0029BABF49422D2326
:10D7800000230A22FFF7B8BF374A384913681B063F
:10D79000FCD40B6813F08003F8D172B634490A78D0
:10D7A000002A5FD0334A3448F0B4344C1768066816
:10D7B0002568D4680C303E44143200681268304F3B
:10D7C00035442C4420440244C2F34E022D4E2E48D0
:10D7D0002E4D2F4C42F400423A60376806682D689F
:10D7E0002C4A24680C303E44006812682A4F3544A5
:10D7F0002C4420440244C2F34E02284E2848294DAE
:10D80000294C42F400423A60376806682D68274A7E
:10D8100024680C303E4400681268254F35442C447F
:10D8200020440244C2F34E02224E2348234D244C8E
:10D8300042F400423A60376806682D68214A24683D
:10D840000C303E440068126835442C4420440244A5
:10D85000C2F34E021C4842F4004202600B7062B6F2
:10D86000F0BC704762B6704724B0034024B00B4050
:10D87000CDA0FF1F38B003403CB0034040B0034090
:10D880002CB0034058B003405CB0034060B003408C
:10D8900064B003406CB0034030B0034038B00B407C
:10D8A0003CB00B4040B00B4044B00B404CB00B4080
:10D8B0002CB00B4058B00B405CB00B4060B00B403C
:10D8C00064B00B406CB00B4030B00B4030B4294812
:10D8D000294A2A4B2A4D6024E121047011701B78DB
:10D8E000284C082B30D00A2B2748284937D00C2B3E
:10D8F0000CBF35223D2212232A60236002600B6098
:10D90000234B24491B78244ABBB101230B601360CD
:10D91000224B23491B78234A012B26D9042B0FD9EC
:10D92000082B1ED9102B94BF862387230B6013600E
:10D930001D4B01221A7030BC70470B601360E7E783
:10D9400084230B601360F3E700F58E200F49083045
:10D95000012213232A60236002600B60D0E7392282
:10D96000F7E785230B601360E2E780230B60136009
:10D97000DEE700BF0040074001400740D492FF1F90
:10D9800008B003400CB0034008B00B400CB00B4093
:10D99000D0A0FF1F20B0034020B00B40D592FF1F46
:10D9A00024B0034024B00B40CDA0FF1F0C2830B49E
:10D9B00017D91023984228BF18461C46104A114D0B
:10D9C0001178181A8C42287018D00F4913700B78F0
:10D9D00023B10E490E4A00230B60136030BCFFF7E1
:10D9E00075BF0A2802D90C231C46E7E7082802D98C
:10D9F0000A231C46E2E708231C46DFE730BC7047D9
:10DA0000D492FF1FCCA0FF1FCDA0FF1F24B0034066
:10DA100024B00B4028282FD8334B2DE9F0411E5C51
:10DA2000FF2E2BD0314B1B78002B2AD132062CD461
:10DA300072B62F4D2F4C2F46012326602B7062B6F5
:10DA400072B623681B060CD43B781BB9F4E72B781D
:10DA5000002BF1D062B602F073FB72B62368180691
:10DA6000F5D5254B1B6800222A7062B6234A107830
:10DA700043FA00F0BDE8F081002070470020BDE8C7
:10DA8000F081FFF781FE3206D2D572B61C4DDFF869
:10DA90007C801C4C06F04007FFB206F03F06D8F829
:10DAA0000030DFB123F01003C8F8003001232660F6
:10DAB000134A2B7062B672B6236819060CD4137819
:10DAC0001BB9ECE72B78002BE9D062B602F038FBEB
:10DAD00072B623681B06F5D50B4BC3E743F0100362
:10DAE000C8F80030E2E700BF68510100CDA0FF1F79
:10DAF000CFA0FF1F00B0034010B00340CCA0FF1F19
:10DB0000CEA0FF1F00B00B4010B00B400CB00B407C
:10DB10000A4A0B49136843F4805313600B7843B9E6
:10DB2000084BC0221A70084B80F30C0000B218801A
:10DB30007047044B80221A70F5E700BF2C80044028
:10DB4000D0A0FF1F21C00C4000C00C40F0B51B4B03
:10DB50001B4E596818689A68DB6885B06C460FC41C
:10DB6000337899071DD5174A174C1378174913F0C6
:10DB7000700318BF1370164A164B802717700026C3
:10DB80003320032226706D4608701A7072B6043C6A
:10DB900045F001052046A84762B6237813F07003CC
:10DBA00009D10D4B064901E0013B02D00A78D207AA
:10DBB000FAD505B0F0BD237005B0F0BD9451010059
:10DBC0000100024000000240040002400B0002403D
:10DBD000070002400A000240410D0300B0F5006F4B
:10DBE0000AD210B5094B1B78DB07044606D504F1B1
:10DBF000A0500078C0B210BD00207047FFF7A6FF0C
:10DC000004F1A0500078C0B210BD00BF0100024076
:10DC1000B0F5006F17D238B50F4B1B78DA070D46F9
:10DC2000044611D504F1A0500378AB420AD00B4A48
:10DC3000137813F0700318BF1370074A0570137838
:10DC4000DB07FCD538BD7047FFF780FF04F1A0501B
:10DC50000378AB42EBD1F5E701000240000002403F
:10DC600008B5F4F713F8F4F759FF02F069FAFAE788
:10DC7000844641EA000313F003036DD1403A41D3D7
:10DC800051F8043B40F8043B51F8043B40F8043B96
:10DC900051F8043B40F8043B51F8043B40F8043B86
:10DCA00051F8043B40F8043B51F8043B40F8043B76
:10DCB00051F8043B40F8043B51F8043B40F8043B66
:10DCC00051F8043B40F8043B51F8043B40F8043B56
:10DCD00051F8043B40F8043B51F8043B40F8043B46
:10DCE00051F8043B40F8043B51F8043B40F8043B36
:10DCF00051F8043B40F8043B51F8043B40F8043B26
:10DD0000403ABDD2303211D351F8043B40F8043BC5
:10DD100051F8043B40F8043B51F8043B40F8043B05
:10DD200051F8043B40F8043B103AEDD20C3205D3D5
:10DD300051F8043B40F8043B043AF9D2043208D0CD
:10DD4000D2071CBF11F8013B00F8013B01D30B883F
:10DD500003806046704700BF082A13D38B078DD01D
:10DD600010F003038AD0C3F10403D21ADB071CBFEF
:10DD700011F8013B00F8013B80D331F8023B20F859
:10DD8000023B7BE7043AD9D3013A11F8013B00F892
:10DD9000013BF9D20B7803704B7843708B7883701A
:10DDA0006046704708B5104C08E0236859050DD44B
:10DDB00023681A050FD42368DB0411D423685803A1
:10DDC000F3D501F065F823685905F1D502F01CFA86
:10DDD00023681A05EFD500F07FFD2368DB04EDD53D
:10DDE00000F0C8FEEAE700BF3480044008B5FFF742
:10DDF000D9FF00BF014B10221A8070470020054058
:10DE0000704700BF094908B50B6830B16A4618442D
:10DE1000A2F58052904202D20860184608BD03F075
:10DE2000A5FC0C2303604FF0FF3008BDD892FF1F04
:10DE3000FEE700BFEFF3138070B9EFF310836BB907
:10DE4000EFF305825AB94FF48070EFF311832BB1D1
:10DE5000984228BF184670474FF0FF3070470F2A8E
:10DE600001D81846F1E7014BD05CEEE7F0E300E0A3
:10DE7000F0B44D1E2E46002400E00134B0FBF2F356
:10DE800002FB1300092800F130078ABF3730F8B2CF
:10DE9000C0B206F8010F1846002BEED10A195370D4
:10DEA0004CB1107815F8016F28700133E01A8342E5
:10DEB00002F80169F5DB0846F0BC7047704700BF07
:10DEC00010B40F4B53F8302092F880422CB101234C
:10DED00069B182F8803010BC704703EBC0035B6807
:10DEE0001A6841B922F002021A6010BC704782F829
:10DEF000003110BC704742F003021A6010BC70473A
:10DF0000A45101001C4A02EBC00301295B6811D037
:10DF100004291BD052F83000002280F8802229B159
:10DF2000022920D0032922D01A6070474FF4807252
:10DF30001A60704752F830004FF4A27280F88012D5
:10DF40001A601A6822F020021A60704752F83010E6
:10DF50004FF4A272012081F880021A601A6842F020
:10DF600020021A60704740F203121A6070474FF4A3
:10DF700081721A60704700BFA4510100212848D85F
:10DF8000F8B5042A44D8DFE802F0484B4E034500B8
:10DF90004FF410262B4B03EBC0030D465C68216841
:10DFA00011F4E06148D0284B284A2949C3F89C2144
:10DFB00004F140422748C3F8A411A2F59221264F4C
:10DFC000C3F8A0017C292548C3F8A871C3F8AC01A7
:10DFD0002CD9A2F594237C2B2AD9A2F596237C2B4D
:10DFE00028D9A2F598237C2B29D9A2F59A227C2A3C
:10DFF00027D81B4872B6236823F4702343F080723D
:10E00000C4F384011643236040F82150266062B6B1
:10E01000F8BD70474FF43026BCE74FF40026B9E74F
:10E020004FF44026B6E74FF42026B3E70D48E1E76A
:10E030000D48DFE70D48DDE7FFF764FFB3E70C4865
:10E04000D8E7F8BDA45101000082FF1FF188FF1F2F
:10E050009988FF1FC588FF1F6D88FF1F4188FF1F1C
:10E06000B493FF1FDC92FF1F1493FF1F6493FF1FE5
:10E070009493FF1F1A4B03EBC00010B4426802F1E7
:10E080004043A3F592217C2923D9A3F594217C292F
:10E090000DD9A3F596217C291FD9A3F598217C29B8
:10E0A00019D9A3F59A237C2B11D80E4C00E00E4C05
:10E0B00072B613680D4823F08773C2F3840123F40A
:10E0C000803343F08073136044F8210062B610BCC3
:10E0D0007047074CECE7074CEAE7074CE8E700BF5E
:10E0E000A4510100B493FF1F1493FF1FBDDE000075
:10E0F000DC92FF1F9493FF1F6493FF1F30B4054B06
:10E10000054D064C002210211A602A60206019601B
:10E1100030BC704714D0034004D0034000D003400B
:10E12000282838B52ED0002904464FDD5F4B1B78D8
:10E13000012505FA03F28A4202D8212837D938BDD1
:10E140000338C2B2012A3AD9202C4AD0192C48D01F
:10E15000574A126802FB011222FA03F31D2800F24B
:10E160009B80DFE800F0928B847D9999766F999976
:10E170009999999999999968615A53994C9999994A
:10E1800099999945494B1B780B2B08D90C2B1CBF2F
:10E190000C3B19410846BDE83840FFF7B9BCC3F154
:10E1A0000C0399400846BDE83840FFF7B1BC29464A
:10E1B000FFF786FE2946BDE83840FFF7A3BE3D4A7B
:10E1C000126802FB011222FA03F3C7E72128B6D82E
:10E1D0000021FFF775FE20460121BDE83840FFF71A
:10E1E00091BE354A126802FB011222FA03F3B5E729
:10E1F0003249334A0B604FF45173136038BD3149D3
:10E20000314A0B604FF45173136038BD2F49304AC7
:10E210000B6040F24443136038BD2E492E4A0B6018
:10E2200040F24443136038BD2C492D4A0B6040F244
:10E230004443136038BD2B492B4A0B6040F24443E2
:10E24000136038BD29492A4A0B6040F244431360E9
:10E2500038BD2849284A0B6040F24443136038BD5A
:10E260002649274A0B6040F24443136038BD2549D4
:10E27000254A0B6040F24443136038BD2349244AC9
:10E280000B604FF45173136038BD2249224A0B6072
:10E290004FF45173136038BD212C3FF650AF7F29E6
:10E2A000D4BF00210121204693E700BFBC93FF1F8C
:10E2B000088003400890034008800B4010800B400A
:10E2C00048A0044018800B404CA004401880034034
:10E2D00008B004401080034004B004404080034074
:10E2E00018C004403880034014C004402880034014
:10E2F00010B00440208003400CB004403080034044
:10E3000010C00440488003401CC0044018900340E3
:10E3100034900440109003403090044038B11028ED
:10E3200028BF1020044AC3B2107813707047024A05
:10E330000123107813707047BC93FF1F2DE9F84339
:10E340000E4680463249334D304603F095F947F684
:10E35000122300281ABF1D464FF002094FF0010991
:10E36000002425FA04F002F091FF4FF05E510746B9
:10E3700002F0E4FF0146304603F092F930B901346F
:10E38000072CEED1E80902F081FF074631463846F6
:10E3900003F088F84FF07C5102F0C6FE03F0BAF9A2
:10E3A0004FF6FF729042A8F1030328BF1046012BDD
:10E3B00029D9B8F1170F17D8174B23FA08F303F030
:10E3C000010383F0010223B9B8F1190F0FD0BDE8A2
:10E3D000F883124B124D13491A6044EAC9042A60AB
:10E3E00008601C60BDE8F883B8F1200FECD10E4B3B
:10E3F0000E4D0F49002244EAC9041A602A600860E1
:10E400001C60BDE8F8830B4B0B4D0C49F2E700BFD5
:10E41000001BB740006CDC026006F0000080034087
:10E42000048003400880034000800B4004800B40C0
:10E4300008800B4000900340049003400890034084
:10E44000212801D8FFF73CBD704700BF212806D81E
:10E45000044B53F8303093F80002C0B270470020EC
:10E46000704700BFA4510100212801D8FFF74ABD21
:10E47000704700BF72B60C490C4B0D4A1B68086808
:10E48000126862B6520102D5322B88BF01300949A9
:10E49000C3F5BB334FF47A72FF33A1FB031302FBC6
:10E4A00000F000EB93107047D4A0FF1F18E000E0CD
:10E4B00004ED00E0ABAAAAAA2DE9F843054672B61E
:10E4C000204F214B214A1B683C68126862B65201FA
:10E4D00002D5322B88BF013495B3C3F5BB331C4E34
:10E4E000DFF86490DFF86480FF334FF47A72A6FBA4
:10E4F000031302FB04F404EB931472B6D9F8001072
:10E500003A68D8F800E062B6C1F5BB33FF33A6FB2A
:10E5100003031EF0806FC4EB93134FF47A7002D0A4
:10E52000322988BF013200FB0233B3F57A7F04D36E
:10E53000013D05D004F57A74DFE701F001FEDCE768
:10E54000BDE8F883D4A0FF1F18E000E004ED00E070
:10E55000ABAAAAAAF8B52D4B2D49DFF8D0E0DFF819
:10E56000D0C02C4E2C4D2D4C2D4A2E4F4FF4000078
:10E5700018604FF0807018604FF0007018604FF016
:10E58000806018604FF00060186000200860282349
:10E590004BF6FF71CCF80010CEF8003033601360FA
:10E5A0002B6023603B60B3629362092245F8242C00
:10E5B000C4F8D80F05F57F65C7F8D41F07F5FF2706
:10E5C00007F5FA67C6F8F83F2B6006F5FF26C4F892
:10E5D000D42F05F5FD2504F5FF24386006F2F47606
:10E5E0001148316005F5FF6504F5FD642B6023607B
:10E5F0000260FFF76BF91920FFF75EFF01F08EF95B
:10E6000040F21310BDE8F840FFF756BF08E100E004
:10E610000480034014800340248003402C80034086
:10E620001C8003403480034000800B400C8003407A
:10E63000088003402B4A2C491368F0B543F400636B
:10E6400013600A78294F2A4E2A4D2B4C2B49002360
:10E65000092A3B7033702B7023700B703DD01A2A3F
:10E6600021D0274B1B780A2B25D01F2B30D01F28F9
:10E6700027D8002002460125224B234C1A7023493B
:10E680005D7004224FF0020E88273C2640259872C8
:10E690009A704FF4004083F813E05A751F74DE70CF
:10E6A00025700860F0BD1A4B40F213321A60144B0B
:10E6B0001B780A2BD9D1174B4FF451721F281A60BF
:10E6C000D7D9C0F34432C0F3471500F01F00D3E799
:10E6D000114B4FF451721A60C9E7104B40F21332DC
:10E6E0001A60BEE734800440BD93FF1F48A1FF1F9E
:10E6F000DDA0FF1F50A1FF1F49A1FF1FDCA0FF1FCE
:10E70000BE93FF1F00B006402FE400E004E100E0EC
:10E7100004D0044010B0044000D004400CB00440C9
:10E7200009B140F08000174A1378984216D010B40F
:10E73000154C246824050FD503F07F030A2B1CD049
:10E740001F2B11D0002900F07F0114BF6023442348
:10E750000A290DD01F2902D0107010BC70470B4938
:10E7600043F440730B60F7E7084B00241C60E9E7B3
:10E77000074943F440730B60EEE7054B00241C602F
:10E78000E0E700BFBE93FF1F3480044000D0044088
:10E7900010B00440124B1A7882420CD0114909681B
:10E7A000090507D5092A16D01A2A0AD009280DD03A
:10E7B0001A2801D0187070470B4A40F213311160CB
:10E7C000F8E7094A002109281160F1D1074A40F20F
:10E7D00013311160EEE7054A00211160E6E700BF42
:10E7E000BD93FF1F3480044004D004400CB00440AB
:10E7F0002DE9F84F234B1B681A053BD5224B1B68AC
:10E800000BB101221A70DFF89090204D99F800406A
:10E81000DFF888801E4E0134272C8ABF4FF0000A93
:10E820005FFA84FA54460746AB462B789C4216D1D1
:10E83000FFF700FB40281FDC33791B06F5D59BF85A
:10E8400000300133272B86BF00221346DAB218F8B6
:10E850000330DBB2F3712A702B789C42E8D00D496B
:10E860000B4BFFB20120BC2208F80470087089F835
:10E8700000A0DA70BDE8F88FFF28D6DD01F060FC5B
:10E88000D3E700BF348004404CA1FF1F49A1FF1F04
:10E8900000B00640DCA0FF1F50A1FF1FE0A0FF1F3B
:10E8A00010B5044C237823B101F04AFC2378002BE7
:10E8B000FAD110BDDCA0FF1F054A064B10781B786B
:10E8C000C0B2DBB2984238BF4030C01A704700BFB8
:10E8D00048A1FF1FDDA0FF1FF0B4384B1A7912F0DA
:10E8E000300F2CD072B6997D01F0FF0200293DD087
:10E8F00062B6334F334938780D78334E1C46C0B278
:10E90000EDB2431C402BE17928BF0023AB4202F15A
:10E91000FF32C9B21CBFF154184612F0FF02F0D109
:10E920002A4B1B68C2B23A704BB1A84236BFC5F140
:10E930004005401B40192728C4BF01221A701F49F7
:10E94000CA78D2B2150616D452060DD51B4B1B79C8
:10E950005B0609D51E4B1F491B6800220A7003B1D4
:10E960001A70164B3C22DA70F0BC70474022D979FD
:10E970005A7462B6E3E70B791C06E5D5164B174EC1
:10E980001C783378E4B2DBB29C420ED0144D01E027
:10E99000A3420AD00133282B28BF00230879E85C62
:10E9A000C0B2C871087D0728F2D9DBB203493370C1
:10E9B0000B79180644BF7C23CB70C5E700B0064036
:10E9C00048A1FF1FDDA0FF1F08A1FF1FD8A0FF1F48
:10E9D0004CA1FF1FDCA0FF1F50A1FF1F49A1FF1F7B
:10E9E000E0A0FF1F2DE9F84F214B1B6807460BB134
:10E9F00001221A70DFF888901E4D99F80040DFF868
:10EA000084801D4E0134272C8ABF4FF0000A5FFA24
:10EA100084FA5446AB462B78A34216D1FFF70AFA84
:10EA200040281FDC33791B06F5D59BF800300133F5
:10EA3000272B86BF00221346DAB218F80330DBB268
:10EA4000F3712A702B78A342E8D00C490A4BFFB22D
:10EA500008F804700120AC22087089F800A0DA7070
:10EA6000BDE8F88FFF28D6DD01F06AFBD3E700BFD1
:10EA7000C8A1FF1FC5A1FF1F00C00640C4A1FF1F02
:10EA8000CCA1FF1F5CA1FF1F1C4BDFF894C01A68CC
:10EA90001B49F0B542F480521A4D1A60DFF884E049
:10EAA000194F1A4E1A4C00238CF800304FF4517253
:10EAB0002B701F2840F213358EF800303B703370F6
:10EAC00025600A6012D819460124124A124D1170AD
:10EAD0001248547000212C27402693724FF40034C2
:10EAE00091701174D7702E700460F0BDC0F3443182
:10EAF000C0F3471400F01F03E7E700BF3480044071
:10EB00000CC0044059A1FF1FC5A1FF1FC4A1FF1FD6
:10EB100008C0044000C0064031E400E004E100E029
:10EB200058A1FF1FCCA1FF1F034B1B68DB0401D5BD
:10EB3000FFF758BF704700BF3480044010B5044C45
:10EB4000237823B101F0FCFA2378002BFAD110BD11
:10EB5000C4A1FF1F054A064B10781B78C0B2DBB278
:10EB6000984238BF4030C01A704700BF58A1FF1FFD
:10EB700059A1FF1F30B42B4B1A7994061FD52A4890
:10EB8000DA790378294901333F2B0978C8BF00237C
:10EB90008B42D2B203D0264CD9B2E2540170254A3E
:10EBA000116861B1244A1278D2B2934236BFC2F1E1
:10EBB00040029B1A9B18272BC4BF01230B70194AD4
:10EBC000D378DBB2180611D45A060DD5154B1B7934
:10EBD0005B0609D5194B1A491B6800220A7003B15C
:10EBE0001A70104B2C22DA7030BC7047117909066C
:10EBF000EAD5144910480C780178C9B28C420DD07E
:10EC00004A1C272A84BF00210A460F4D054C98BF95
:10EC1000D1B2AA5CD2B2E2710170D5E76C21D17099
:10EC2000D2E700BF00C0064058A1FF1F59A1FF1F37
:10EC300084A1FF1F54A1FF1FC5A1FF1FC8A1FF1F73
:10EC4000C4A1FF1FCCA1FF1F5CA1FF1F21282FD84B
:10EC5000184B195CFF292BD0174B184ADFF870C0EE
:10EC600003EBC000F0B54368DFF868E0144F154DC2
:10EC7000154E00241C60DEF80030012043F0200314
:10EC80008840CEF8003014604FF4A07338602E60D6
:10EC9000C2F800C0013BFDD113689B05FCD42023C2
:10ECA000013BFDD1094B09B233F8110080B2F0BD30
:10ECB00000207047B4520100A451010000500440EC
:10ECC0000850044004500440000002030051044076
:10ECD00080014A0038800440431E032B14D872B6CA
:10ECE0000A4951F8230068B170B4094C058834F81A
:10ECF0001320466841F82360521B24F8132062B6A3
:10ED000070BC704762B670470020704728A2FF1F92
:10ED1000F0A3FF1F013803280BD872B6074B53F836
:10ED2000203043B100205B680130002BFBD162B67C
:10ED30007047002070471846F9E700BF7CA2FF1F0C
:10ED400030B472B62B4A13781D0706D52A4B196AC0
:10ED5000002936D0996A002941D053781C0706D57E
:10ED6000254B196C00293ED0996C002939D0937835
:10ED7000190705D5204B196E002936D0996E89B137
:10ED8000D3781B0707D51C4BD3F880207AB3D3F870
:10ED9000882011213AB162B6184B00221A7030BC9B
:10EDA00000F04ABE0D21154C154D227843F8315024
:10EDB00003EBC1030830013A5860227062B630BCE0
:10EDC000704704220D4C0F4D217843F8325003EB6D
:10EDD000C20308304A1E5860227062B6EFE7052170
:10EDE000E1E70921DFE70822ECE70C22EAE710223D
:10EDF000E8E700BFD85201000080FF1FA5A2FF1F57
:10EE0000C800400088004000431E032B1DD81B4A49
:10EE1000400140F0100030B4104472B6184CE25C6F
:10EE2000032A1BD8DFE802F00212151703220D880F
:10EE3000E25410F0080F14BFC823882343EA0543A7
:10EE400008310360416062B630BC7047083002226E
:10EE5000EDE70522EBE708300422E8E7094A52F81B
:10EE6000230038B1084A52F82300416042F82310C9
:10EE700062B6E9E742F82310034AF7E70080FF1F74
:10EE8000B4A2FF1F7CA2FF1F8CA2FF1F00BE704711
:10EE90002DE9F04FDFF818B3DFF818A387B044E08E
:10EEA000AD4F4FEA930807EBC809013ED9F804209B
:10EEB00003F00803F6B2A2F1080003F0FF04002BF0
:10EEC00040F0018157F838301B0C99B222F8081C29
:10EED000002B00F0EF80A14B22F8064C42F8044CC6
:10EEE00053F82620002A00F0CF819D4D55F826309A
:10EEF00058609C4C45F8260034F81630194424F824
:10EF0000161000F079FD002800F0C281964A974B58
:10EF100019F0080F00F1080018BF1346C9F80400E3
:10EF200047F8383008238BF800309BF80040E4B2F3
:10EF300065071CD58E4B1B78B3B18E490A7802F059
:10EF4000FF0322B1013BDBB20B7003B900BE8A495B
:10EF50000A7802F0FF032AB1013BDBB20B70002BF1
:10EF600000F0688100F066FE04238BF8003004F0A6
:10EF7000080303F0FF02002B00F0C9809AF800306C
:10EF8000DBB21E098CD19A08DFF8CC9159F8321007
:10EF900009EBC200C1F38301013940680C2900F27A
:10EFA0008580DFE801F07A7A8383838383834683D5
:10EFB000838307000168714D4068714F714E68602E
:10EFC000296088B240F281610024674B49F83230F1
:10EFD0004FF0010E88423C60C9F81040C9F8184053
:10EFE00086F800E05C4A00F2E780B0F5D06F80F070
:10EFF0001B82B0F5817F00F0D98100F26981802801
:10F0000000F02A82822840F0D781A98801F07F0190
:10F01000042900F2D1815C485C4A890008441470DC
:10F02000547001788C0740F1608382F800E002217F
:10F0300073E1534F3A682AB3554B524E55481988DD
:10F040003478057840298E4645F0020828BF4FF0F5
:10F05000400E002C84F001043470CEEB01010CBF93
:10F060008824C82409EBC80689B285F0010544EA62
:10F070000E447260198049F83840724405700029C6
:10F0800065D03A603D4B1A88B2F5A06F0ED10021D1
:10F090009A785970404B1A7008E038493F4C0D6817
:10F0A000A54200F09880304949F832103C4A0123CB
:10F0B000137037E72C4A2D4B19F0080F18BF134671
:10F0C00047F838302EE700F0B7FC364A364952F898
:10F0D0002630002B00F0E38058688C5D42F8260053
:10F0E00003F10802C9F80420032C05D8DFE804F076
:10F0F0002C02292602228A551A8819F0080F0CBF03
:10F100008823C82343EA024347F838300AE7E00778
:10F1100000F19380210600F1D180A20706D5234A91
:10F12000234913780220DBB213700870E30602D57E
:10F130001F4B10221A7007B0BDE8F08F04228A55C9
:10F14000DAE705228A55D7E703228A55D4E7BEF1CC
:10F15000400F18BF002294E70080FF1F28A2FF1F66
:10F16000D4A1FF1FF0A3FF1FC8004000880040008B
:10F17000B0A2FF1F39A2FF1F24A3FF1F9CA2FF1FE5
:10F18000D0A1FF1F38A2FF1FC0200740A8A2FF1F69
:10F19000E4A1FF1FA4A2FF1F98200740210900033C
:10F1A000942007407CA2FF1FB4A2FF1F88200740C5
:10F1B0008020074090200740B0F5106F00F07C8160
:10F1C00040F2A38040F62112904240F07B82A54A93
:10F1D000012313706AE74C68A3498C427FF463AF44
:10F1E0000178A9297FF45FAF417845297FF45BAFAF
:10F1F0008178C2297FF457AFC1786B297FF453AF70
:10F200009A489B4E0178347881F00105002C41F03A
:10F21000020105700CBF8820C82084F0010449F861
:10F22000310009EBC10193483470002505244D607D
:10F23000047038E700F064FF94E68F4B89488B49EF
:10F240001A614FF0020E80F800E08C4F0A708C4972
:10F25000196099608B4E8C4D8C4C9A610D213970E0
:10F26000FF213170DFF84CE229702270884D894A05
:10F270008EF800109F27012406F8047C5D6004705E
:10F28000DA6007B0BDE8F08F43F82600824D30E623
:10F29000824A47F8380013780133137042E68B5DD9
:10F2A000032B00F2BA8001A252F823F025EF0000F0
:10F2B00025EF000005F30000FFF200006F49724BDC
:10F2C00080220D2008701A70A2077FF52FAF26E765
:10F2D00040F20232904240F0ED81AA8802F07F02B3
:10F2E000042A69D86D88002D66D16449CDF804E000
:10F2F000920011440A7842F002020A70C1E101232F
:10F300008B550FE600238B550CE6B0F5086F53D1F3
:10F310006349644A097811707146ED888D4280F026
:10F32000E88252480478402DAE4644F0020C28BFD3
:10F330004FF0400E02EB0E0309EBCC0102930123C8
:10F340004A604FEA0E48CEEB050101930025C82222
:10F3500042EA080384F0010249F83C30357002703B
:10F36000DFF814C1424BDFF8048149BBBEF1400F06
:10F370007FF42DAF42F0020C09EBCC03029ADFF8C8
:10F38000F8E05A608DBB0D0445F088059DF8043007
:10F390004EF83C500A4433700470134640297FF401
:10F3A00016AF0021404A3B60118010E7AA8802F0A6
:10F3B0007F02042A40F28B81304A0F23137006E744
:10F3C0004029D7D942F002020CEBC200029E4660EF
:10F3D000BDB19DF8045035481D703346403988F85A
:10F3E000004040334CF83200DCE79DF804303370C5
:10F3F0000D04029B047045F0C8050B444EF83C50C8
:10F40000CCE79DF804501D70029B1D4888F8004011
:10F41000403940334CF83200C4E719F0080F0CBFF4
:10F42000022303238B557DE521494A68002AC3D076
:10F430006C88B5F804E003E00C314A68002ABBD0C0
:10F440000B88A342F8D14B887345F5D1240A032CCD
:10F450000CBF1178098960E7124A022114705470B8
:10F460005BE700BF9420074001000400A4A2FF1F37
:10F4700038A2FF1F39A2FF1F0080FF1FC0200740D6
:10F4800088004000882007408020074098200740DF
:10F49000E8A1FF1F3CA2FF1FD4A1FF1FA5A2FF1FD1
:10F4A000B0A2FF1FA8A2FF1FE4A1FF1FC8004000D9
:10F4B000DC5201008C200740B248116AAC7804701D
:10F4C0000C0600F19881D9F82820AF49100600F108
:10F4D000DB81D9F83020AC49120600F1D081D9F88F
:10F4E0003820A949130600F1C581D9F84020A64962
:10F4F000150600F1BA81D9F84820A349140600F195
:10F50000AF81D9F85020A049100600F1A481D9F8A4
:10F5100058209D49120600F19981D9F860209A4936
:10F52000130600F18E81D9F868209749150600F17D
:10F530008381D9F870209449140600F17881D9F8B4
:10F5400078209149100600F16D81D9F880208E490C
:10F55000120600F16181D9F888208B49130600F169
:10F560005581D9F890208849150600F14981D9F8CC
:10F5700098208549140600F1FF808448844A854913
:10F5800001908548854D864C049700230596029589
:10F5900080460F4616461D460394306828B14468DD
:10F5A00000F04AFA2046002CF9D100233360029B78
:10F5B00038681A46002342F8253028B1446800F024
:10F5C0003BFA2046002CF9D100223A60019A98F8C3
:10F5D00000301146002241F8042B039A0191023BAE
:10F5E0004FF0000122F81510032B07D8DFE803F0D5
:10F5F0005D025D024FF0010388F800300135042DF3
:10F6000006F1040607F1040708F10108C5D1654CAD
:10F61000654D2278654B049F059E002110072970D7
:10F620001A7000F19280624962780A700021C9F86C
:10F630003010C9F838101107DFF84C816ED4A27869
:10F640005C49DFF844810A7000211207C9F85010A4
:10F65000C9F858104BD4E27857494B4C0A7013073D
:10F660004FF00001C9F87010C9F8781000F1AE80B1
:10F6700033780193002283F00105C9F89020C9F87E
:10F6800098200021029188468E460A464B4804780D
:10F6900044F0020C09EBCC030393019B002B039B6A
:10F6A0005A600CBF8822C82252E64FF0000388F847
:10F6B0000030A3E7B0F5A06F7FF47EAE01230025F4
:10F6C0000193DEE740F621229042F7D074E66D8880
:10F6D000002D7FF471AE3A49CDF804E09200114458
:10F6E0000A7822F002020A70CBE7022115E600F048
:10F6F00083F9002800F0EB800830324AC8F8640033
:10F70000C8F8602000F078F9002800F0DA800830AE
:10F710002D4AC9F86C00C9F868209CE700F06CF924
:10F72000002800F0E0800830264AC8F84400C8F8F5
:10F73000402000F061F9002800F0CF800830224A14
:10F74000C9F84C00C9F8482079E700F055F90028BD
:10F7500000F0A58008301B4AC9F82400C9F8202011
:10F7600000F04AF9002800F094800830164AC9F8E1
:10F770002C00C9F8282056E7D1F89C00083800F082
:10F780005BF9FAE6B0A2FF1F0080FF1F8CA2FF1FEB
:10F7900028A2FF1F7CA2FF1FB4A2FF1FD4A1FF1F3E
:10F7A000F0A3FF1FD8520100A5A2FF1FC4200740ED
:10F7B000C8200740CC200740D0200740A4A2FF1F4C
:10F7C000C020074088004000C800400000F014F945
:10F7D000002870D008304F4AC4F88400C4F8802054
:10F7E00000F00AF9002860D008304B4AC9F88C00B4
:10F7F000C9F888203CE7506A083800F01DF962E635
:10F80000D1F89400083800F017F9B0E6D1F88C0070
:10F81000083800F011F9A4E6D1F88400083800F0A7
:10F820000BF998E6C86F083800F006F98DE6486FC6
:10F83000083800F001F982E6C86E083800F0FCF8DC
:10F8400077E6486E083800F0F7F86CE6C86D0838BF
:10F8500000F0F2F861E6486D083800F0EDF856E681
:10F86000C86C083800F0E8F84BE6486C083800F03F
:10F87000E3F840E6C86B083800F0DEF835E6486B80
:10F88000083800F0D9F82AE6C86A083800F0D4F839
:10F890001FE62A78C9F8280001322A70C3E62A78C0
:10F8A000C9F8200001322A705AE72A78C9F888007E
:10F8B00001322A70DCE62A78C4F8800001322A700E
:10F8C0008EE72A78C9F8680001322A70C3E62A78E0
:10F8D000C8F8600001322A7014E72A78C9F8480095
:10F8E00001322A70ABE62A78C8F8400001322A704B
:10F8F0001FE740298E4628BF4FF0400E02EB0E0353
:10F9000002930123CEEB01014FEA0E48002501933B
:10F91000BCE600BF88004000C8004000F8B500F019
:10F92000F9FC294B29482A4C2A4F2B4DDFF8BCC043
:10F93000DFF8BCE0294E00221A605A609A60DA6053
:10F940001A615A619A61DA611A625A629A62DA62DB
:10F950001A635A639A63DA631A645A649A64DA64BB
:10F960001A655A659A65DA651A665A669A66DA669B
:10F970001A675A679A67DA67C3F880200168C3F884
:10F98000842041F480210160C3F307212170C3F377
:10F990000740134938701B0E2B70FF238CF8003082
:10F9A000104D8EF8003010480B700123337084F82E
:10F9B000642070264FF40074102207F82C3C2E703F
:10F9C000046081F8F820F8BD0080FF1F34800440F7
:10F9D0009C200740B0200740B420074094200740F7
:10F9E0001020074049E400E008E100E080200740E3
:10F9F00088200740704700BF72B60D480268B2FA0F
:10FA000082F30F2B10DC4FF00041D94022EA0102B3
:10FA1000026062B6074803EBC303DB00C218002193
:10FA2000C15010465160704762B60020704700BF59
:10FA3000C093FF1FBC83FF1F0D4B0E4AC31AA2FBCE
:10FA400003231B090F2B0CD80B4A127852B972B63C
:10FA50000A484FF00041026821FA03F31A4302609A
:10FA600062B67047064A1278002AF0D0FFF768B9EC
:10FA7000BC83FF1F398EE338A5A2FF1FC093FF1F71
:10FA8000B0A2FF1F38B50E4B0E4C1B6821880546EF
:10FA90008BB1B1F5917F05D20B4A4B1C55549BB2EB
:10FAA000238038BD0022084898470021064A555453
:10FAB0000123238038BDB1F5917FEDD338BD00BF60
:10FAC000DCA2FF1FFAA3FF1F00A4FF1F2DE9F843CC
:10FAD000214E224F3168012380463B70B1B1204D49
:10FAE0004B8801EB8302013300240F2BC2F80880FE
:10FAF0002C7004D84B8000233B70BDE8F883402372
:10FB00000B800320FFF780F93460F4E7DFF85490AE
:10FB100099F80030002BF0D0114D45F6215408E043
:10FB2000013C12D02B7883B900F00AFB99F8003021
:10FB30007BB10320FFF7EEF80528F1D8FFF75CFF53
:10FB4000014630600028EBD0CAE701232B70BDE8E6
:10FB5000F883BDE8F88300BFF8A2FF1FCCA2FF1F07
:10FB6000FCA2FF1FB0A2FF1F1201F8B5D5B2A1B3CE
:10FB7000012943D04378044600781B0643EA00403D
:10FB800040F4704045F004068F1E3043FFF79EFF9F
:10FB9000022F04F1020314D9053414F8023C14F8BE
:10FBA000032C14F8010C1B0443EA0223334343EAF9
:10FBB0000060033FFFF78AFF022F234604F103048E
:10FBC000EBD8022F23D0012F0DD045F4774040F021
:10FBD0000500BDE8F840FFF779BF14482843BDE8A9
:10FBE000F840FFF773BF187845F4770545F0060530
:10FBF00045EA0020BDE8F840FFF768BF03780C48ED
:10FC000045EA03452843BDE8F840FFF75FBF1A788F
:10FC1000587845F0774545F0070545EA022545EA5D
:10FC20000040BDE8F840FFF751BF00BF06F0F70005
:10FC300007F000F738B5084B1C7824B9074D296840
:10FC400009B14B8803B938BD9B000B800320FFF737
:10FC5000DBF82C6038BD00BFCCA2FF1FF8A2FF1F4D
:10FC60002DE9F041AD4E33680746002B00F092803D
:10FC70001D885A88910803EB81010432AA428C68DE
:10FC800042D25A8004F00F064FEA1428A449A6F184
:10FC9000080208F00F00C4F30313062A00F101055F
:10FCA0000B701AD9B31E012B5FFA88F04ED9052EBE
:10FCB00048D0042E00F0A481731F022B7FD90F2E91
:10FCC0000ED1F72842D8F02802D0964B1B883BB1C2
:10FCD000FFF7D8FE0020BDE8F08127B1BD4202D079
:10FCE0000020BDE8F081082EC4F3033300F08780C4
:10FCF000092E11D00A2E40F094800A2BF0D18A4BA5
:10FD00008A4A1B68A02181E01846FFF795FE04206F
:10FD1000FEF7E2FF3060B5E7092BE1D1270E00F0D6
:10FD20007B81834B814A1B689021C4F30746117085
:10FD3000EDB2FCB2002B00F09D80224631462846F1
:10FD4000984797E0F02843D9F72841D0F1380E289A
:10FD5000C6D801A353F820F00FFF0000F3FE000007
:10FD6000E1FE0000E1FC0000E1FC0000D3FE000029
:10FD7000E1FC0000B3FF0000E1FC00007DFF00009B
:10FD800097FF0000BBFE0000E1FC0000A3FE0000A6
:10FD900087FE0000674B1B78002BA1D00420FEF7E4
:10FDA0009BFF0346306000289AD00588002D7FF421
:10FDB00060AFFFF741FE35602846BDE8F081FFF7F0
:10FDC00061FEC4F30740FFF75DFE072E02D1200E4F
:10FDD000FFF758FE534B584A198858481468584D35
:10FDE000524A017000270E0AF0201F802E701070FA
:10FDF0000CB301225348A0470120BDE8F081082B35
:10FE00007FF46EAF504B494A1B688021C4F307460C
:10FE10001170EDB2240E6BB3284622463146984746
:10FE200028E00B2E11D10B2B7FF45AAF474B3F4AE2
:10FE30001B68B021EAE7464B1B68002B00F0FB80F3
:10FE4000404898470120BDE8F0810C2E40F0008129
:10FE50000C2B7FF445AF3F4B344A1B68C021117017
:10FE6000EDB2C4F30746002B00F0C88028463146A7
:10FE7000240E98473849314A314B0D7016701C706A
:10FE80000120BDE8F081354B1B68002B00F0D680C7
:10FE90009847C4F30746254BEDB2240E83F8008043
:10FEA000E8E72F4B1B68002BF2D12E4B1B68A3B148
:10FEB000FE209847C4F30746EDE72B4B1B68002B49
:10FEC000E6D1284B1B6843B1FC209847C4F3074692
:10FED000E1E7264B1B68002BDAD1C4F30746DAE7CB
:10FEE000234B1B68C4F30746002BD4D030469847F9
:10FEF000D1E7204B1A68002AEFD0260C630C06F0DD
:10FF00007F0003F47E531843F6B29047C3E71A4BC1
:10FF10001B68C4F30746002BE8D1BCE704A3FF1F0E
:10FF2000FEA3FF1FFAA3FF1FE0A2FF1FF8A3FF1FFE
:10FF300014A3FF1FB0A2FF1FDCA2FF1FFCA3FF1F23
:10FF4000FDA3FF1F00A4FF1F0CA3FF1F10A3FF1F93
:10FF5000F4A2FF1FD0A2FF1FFFA3FF1FBCA2FF1F21
:10FF6000C0A2FF1FC4A2FF1F00A3FF1FF0A2FF1F1C
:10FF700008A3FF1FD8A2FF1FECA2FF1F3F4B1B6867
:10FF8000002B85D13E4B1B68002BA6D0FA2098474A
:10FF9000C4F307467FE73B4B1B68002B7FF478AF29
:10FFA000374B1B68002B98D0FB209847C4F30746BB
:10FFB00071E7354B1B68002B7FF46AAF304B1B6831
:10FFC000002B8AD0F8209847C4F3074663E70E2B2E
:10FFD0007FF486AE2D4A2E4B1268E0211970002A5C
:10FFE00047D0260C610C06F07F0301F47E511943C3
:10FFF000EDB2A1F5005128469047F6B2240E39E73C
:020000021000EC
:10000000FFF740FDC4F30740FFF73CFD200EFFF76C
:1000100039FD0020BDE8F0811E4B1D4A1B68802180
:100020001170EDB2C4F3074683B1314628463A4613
:1000300098473C461EE70120BDE8F081104B1B6845
:10004000002B3FF44AAFFF20984746E71C4611E7D4
:100050000D2EBCD10D2B7FF443AE0F4B0C4A1B6809
:10006000D0211170EDB2C4F30746002B7FF4FEAE31
:10007000C4E7C4F30746EDB2240EFBE6E8A2FF1F77
:10008000C4A2FF1FC8A2FF1FB8A2FF1FD4A2FF1F58
:10009000F8A3FF1F0CA3FF1FE4A2FF1F38B5164DE6
:1000A0002868E0B101884488A14213DD03191B7A56
:1000B00083B104F10803C2180C1B002302E012F8FC
:1000C000011F21B10133A342F9D1204638BD1C469E
:1000D000204638BDFFF7B0FC0020286038BD074B34
:1000E0001B780BB9002038BD0220FEF7F5FD286013
:1000F0000028D7D1F6E700BF20A3FF1FB0A2FF1F43
:100100000D4B1B78BBB910B50C4C216803F0FF02F6
:100110004B883F2B07DC07330B4401F1470003F802
:10012000012F8342FBD140230B800120FEF76CFEA0
:100130000023236010BD704718A3FF1F1CA3FF1FDF
:1001400038B5224C237803B138BD01232370FFF763
:10015000A5FF70BB00F048F840BBFEF7ADFB10BB3D
:10016000FEF7F8FCE0B900232370EFF30583002BC2
:10017000EAD1EFF3108172B6154B1868E0B1154C57
:100180002278CAB945691D6001232370C5B1AA61EF
:1001900001B962B600254577836898472570D3E793
:1001A00000F020F8DFE700F01BF8D9E700F016F8C0
:1001B000D3E7FFF71FFCCDE70029C5D162B638BDF4
:1001C000054B1D600029E5D1E3E700BF25A3FF1F14
:1001D000C0A0FF1FC4A0FF1FBCA0FF1F704700BF2F
:1001E000704700BF704700BF054A064B10781B7868
:1001F000C0B2DBB2984238BF4030C01A704700BF6F
:100200002CA3FF1F2DA3FF1FF0B4384B1A7912F057
:10021000300F2CD072B6997D01F0FF0200293DD03D
:1002200062B6334F334938780D78334E1C46C0B22E
:10023000EDB2431C402BE17928BF0023AB4202F111
:10024000FF32C9B21CBFF154184612F0FF02F0D1C0
:100250002A4B1B68C2B23A704BB1A84236BFC5F1F7
:100260004005401B40192728C4BF01221A701F49AE
:10027000CA78D2B2150616D452060DD51B4B1B797F
:100280005B0609D51E4B1F491B6800220A7003B18B
:100290001A70164B3C22DA70F0BC70474022D979B4
:1002A0005A7462B6E3E70B791C06E5D5164B174E78
:1002B0001C783378E4B2DBB29C420ED0144D01E0DE
:1002C000A3420AD00133402B28BF00230879E85C01
:1002D000C0B2C871087D0728F2D9DBB20349337078
:1002E0000B79180644BF7C23CB70C5E700A00640FD
:1002F0002CA3FF1F2DA3FF1F70A3FF1F28A3FF1F09
:10030000B4A3FF1FB0A3FF1FB8A3FF1FB1A3FF1F1C
:1003100030A3FF1F70B584B072B6194B194D1A483F
:10032000702241260F2480211A702E701A46047004
:10033000197013781B06FCD5144B186862B6144B61
:10034000144C984298BF00EB800001A998BF400070
:100350000A22FDF78DFD01A92046002311F8012B8B
:1003600001333AB10A2B20F8022FF7D1162323705C
:1003700004B070BD5B00DBB2237004B070BD00BF81
:100380000000024007000240060002400800024050
:100390007F9698008C94FF1F2DE9F043DFF8EC80E6
:1003A0008BB006460F4600F073F898F90030013321
:1003B00004460D4637D03046394600F0DFF90028B4
:1003C00031D02BA3D3E900233046394600F026FE76
:1003D000814668BB28A3D3E900233046394600F0A4
:1003E000FFFD00B398F90030254ACDF82090042491
:1003F00000200021022BCDE90467CDE902670094BB
:100400000192CDE906012CD0684600F0BDF940B359
:10041000089B1BB101F0AAF9089B0360DDE9060106
:100420000BB0BDE8F083204629460BB0BDE8F08351
:10043000134A98F90030019203210022CDE90467A4
:10044000CDE90267009108922BB90E4B4FF0604244
:10045000CDE90623D8E70C490020022BCDE906019F
:10046000D2D101F083F922230360D1E7AFF30080FA
:10047000EF39FAFE422E864051302DD5104987C003
:1004800048530100FFFFEF470000F07FA294FF1FD9
:100490002DE9F04FB04F21F00042BA4283B00C4634
:1004A0004FEAD17605460DD9AC4FBA4225D9C1F3F2
:1004B0001303034340F0EF800EB10020014603B068
:1004C000BDE8F08FA64B9A4200F2CC80A54B9A4231
:1004D00000F2DE808AA3D3E9002300F05DF9002258
:1004E000A14B00F09BFD002800F005812846214625
:1004F00000229D4B00F050F9E1E783A3D3E90023EC
:1005000000F08CFD002840F0CB802846214680A3D7
:10051000D3E9002300F064FD0028CED1934B284698
:1005200003EBC60821467CA3D3E9002300F0E6FADA
:10053000D8E9002300F030F900F07AFD804600F0A1
:1005400077FA77A3D3E9002306460F4600F0D6FAE0
:1005500002460B462846214600F01CF972A3D3E957
:100560000023CDE900013046394600F0C7FA824643
:100570008B4652465B46DDE9000100F00BF905466B
:100580000C462A4623462846214600F0B7FA68A3BF
:10059000D3E9002306460F4600F0B0FA66A3D3E97C
:1005A000002300F0F7F832463B4600F0A7FA64A3B8
:1005B000D3E9002300F0F0F832463B4600F09EFA03
:1005C00061A3D3E9002300F0E5F832463B4600F092
:1005D00095FA5FA3D3E9002300F0DEF832463B46EC
:1005E00000F08CFA02460B462846214600F0D2F86D
:1005F00006460F462846214632463B46B8F1000FD4
:1006000056D000F07BFA324604460D463B460020A9
:100610004FF0804100F0BEF802460B4620462946C6
:1006200000F096FB02460B465046594600F0B2F8E1
:10063000DDE9002300F0AEF80B4602464A490020EF
:1006400000F0A8F86FF47F7398454FDA08F57A78D0
:1006500001EB085100224FF0B87300F04FFA03B0DD
:10066000BDE8F08F424B9A423FF658AF414BF40041
:100670002344D3E9002300F08DF83F4BC6F1010875
:100680001C44CDE90001D4E900ABC6EB080870E7D3
:100690004FF0000875E702460B4600F07DF80EE7C4
:1006A00017A3D3E900231046194600F027FA06E7FE
:1006B00000F024FA0022804689464FF080433046FD
:1006C000394600F067F802460B464046494600F0BE
:1006D0003FFB2A46234600F05DF802460B46002009
:1006E000214900F057F803B0BDE8F08F01EB085145
:1006F00003B0BDE8F08F804643E700BFAFF3008052
:100700009C7500883CE4377EEF39FAFE422E864025
:1007100051302DD5104987C0FE822B654715F73F14
:100720000000E0FE422EE63F763C7935EF39EA3DA7
:10073000D0A4BE726937663EF16BD2C541BDBB3EE7
:100740002CDE25AF6A56113F93BDBE166CC1663FC5
:100750003E5555555555C53F412E8640FFFFEF7F0D
:10076000422ED63FFFFF2F3E0000F03F50530100C6
:10077000B1A2F03F705301006053010041F000410D
:1007800001F58010C00F70470020704781F00041D4
:1007900002E000BF83F0004330B54FEA41044FEA66
:1007A000430594EA050F08BF90EA020F1FBF54EA01
:1007B000000C55EA020C7FEA645C7FEA655C00F09D
:1007C000E2804FEA5454D4EB5555B8BF6D420CDD6E
:1007D0002C4480EA020281EA030382EA000083EAF1
:1007E000010180EA020281EA0303362D88BF30BD91
:1007F00011F0004F4FEA01314FF4801C4CEA1131E7
:1008000002D0404261EB410113F0004F4FEA033345
:100810004CEA133302D0524263EB430394EA050FD0
:1008200000F0A780A4F10104D5F1200E0DDB02FA3F
:100830000EFC22FA05F2801841F1000103FA0EF2D3
:10084000801843FA05F359410EE0A5F120050EF199
:10085000200E012A03FA0EFC28BF4CF0020C43FACA
:1008600005F3C01851EBE37101F0004507D54FF0D7
:10087000000EDCF1000C7EEB00006EEB0101B1F527
:10088000801F1BD3B1F5001F0CD349085FEA30006D
:100890004FEA3C0C04F101044FEA445212F5800F78
:1008A00080F09A80BCF1004F08BF5FEA500C50F115
:1008B000000041EB045141EA050130BD5FEA4C0CF8
:1008C000404141EB010111F4801FA4F10104E9D181
:1008D00091F0000F04BF01460020B1FA81F308BF78
:1008E0002033A3F10B03B3F120020CDA0C3208DD44
:1008F00002F1140CC2F10C0201FA0CF021FA02F11F
:100900000CE002F11402D8BFC2F1200C01FA02F18E
:1009100020FA0CFCDCBF41EA0C019040E41AA2BFB3
:1009200001EB0451294330BD6FEA04041F3C1CDA7B
:100930000C340EDC04F11404C4F1200220FA04F09B
:1009400001FA02F340EA030021FA04F345EA030145
:1009500030BDC4F10C04C4F1200220FA02F001FA07
:1009600004F340EA0300294630BD21FA04F0294689
:1009700030BD94F0000F83F4801306BF81F4801122
:100980000134013D4EE77FEA645C18BF7FEA655C95
:1009900029D094EA050F08BF90EA020F05D054EA67
:1009A000000C04BF1946104630BD91EA030F1EBF6C
:1009B0000021002030BD5FEA545C05D14000494170
:1009C00028BF41F0004130BD14F580043CBF01F563
:1009D000801130BD01F0004545F0FE4141F4700149
:1009E0004FF0000030BD7FEA645C1ABF1946104624
:1009F0007FEA655C1CBF0B46024650EA013406BF25
:100A000052EA033591EA030F41F4002130BD00BFE3
:100A100090F0000F04BF0021704730B54FF48064A0
:100A200004F132044FF000054FF0000150E700BF21
:100A300090F0000F04BF0021704730B54FF4806480
:100A400004F1320410F0004548BF40424FF000016D
:100A50003EE700BF42004FEAE2014FEA31014FEAB0
:100A600002701FBF12F07F4393F07F4F81F06051FF
:100A7000704792F0000F14BF93F07F4F704730B56E
:100A80004FF4607401F0004521F0004120E700BF01
:100A900050EA010208BF704730B54FF000050AE088
:100AA00050EA010208BF704730B511F0004502D589
:100AB000404261EB41014FF4806404F132045FEA8B
:100AC000915C3FF4DCAE4FF003025FEADC0C18BF30
:100AD00003325FEADC0C18BF033202EBDC02C2F126
:100AE000200300FA03FC20FA02F001FA03FE40EAB8
:100AF0000E0021FA02F11444C1E600BF70B54FF0B8
:100B0000FF0C4CF4E06C1CEA11541DBF1CEA135599
:100B100094EA0C0F95EA0C0F00F0DEF82C4481EA01
:100B2000030621EA4C5123EA4C5350EA013518BF21
:100B300052EA033541F4801143F4801338D0A0FB0E
:100B400002CE4FF00005E1FB02E506F00042E0FBBB
:100B500003E54FF00006E1FB03569CF0000F18BFC1
:100B60004EF0010EA4F1FF04B6F5007F64F5407469
:100B700004D25FEA4E0E6D4146EB060642EAC621FC
:100B800041EA55514FEAC52040EA5E504FEACE2E69
:100B9000B4F1FD0C88BFBCF5E06F1ED8BEF1004F6C
:100BA00008BF5FEA500E50F1000041EB045170BDE8
:100BB00006F0004646EA010140EA020081EA03012C
:100BC000B4EB5C04C2BFD4EB0C0541EA045170BD28
:100BD00041F480114FF0000E013C00F3AB8014F1A2
:100BE000360FDEBF002001F0004170BDC4F10004EB
:100BF000203C35DA0C341BDC04F11404C4F120056C
:100C000000FA05F320FA04F001FA05F240EA0200C6
:100C100001F0004221F0004110EBD37021FA04F6FC
:100C200042EB06015EEA430E08BF20EAD37070BDB6
:100C3000C4F10C04C4F1200500FA04F320FA05F015
:100C400001FA04F240EA020001F0004110EBD37017
:100C500041F100015EEA430E08BF20EAD37070BD87
:100C6000C4F1200500FA05F24EEA020E20FA04F360
:100C700001FA05F243EA020321FA04F001F000410F
:100C800021FA04F220EA020000EBD3705EEA430E80
:100C900008BF20EAD37070BD94F0000F0FD101F0AF
:100CA0000046400041EB010111F4801F08BF013CE8
:100CB000F7D041EA060195F0000F18BF704703F026
:100CC0000046520043EB030313F4801F08BF013DAD
:100CD000F7D043EA0603704794EA0C0F0CEA135569
:100CE00018BF95EA0C0F0CD050EA410618BF52EA23
:100CF0004306D1D181EA030101F000414FF0000029
:100D000070BD50EA410606BF1046194652EA430636
:100D100019D094EA0C0F02D150EA013613D195EAAA
:100D20000C0F05D152EA03361CBF104619460AD1F2
:100D300081EA030101F0004141F0FE4141F47001FC
:100D40004FF0000070BD41F0FE4141F4780170BDEC
:100D500070B54FF0FF0C4CF4E06C1CEA11541DBF51
:100D60001CEA135594EA0C0F95EA0C0F00F0A7F853
:100D7000A4EB050481EA030E52EA03354FEA013180
:100D800000F088804FEA03334FF0805545EA131393
:100D900043EA12634FEA022245EA111545EA10655B
:100DA0004FEA00260EF000419D4208BF964244F1F2
:100DB000FD0404F5407402D25B084FEA3202B61A11
:100DC00065EB03055B084FEA32024FF480104FF4E5
:100DD000002CB6EB020E75EB030E22BFB61A754659
:100DE00040EA0C005B084FEA3202B6EB020E75EBEC
:100DF000030E22BFB61A754640EA5C005B084FEA54
:100E00003202B6EB020E75EB030E22BFB61A754620
:100E100040EA9C005B084FEA3202B6EB020E75EB2B
:100E2000030E22BFB61A754640EADC0055EA060EEC
:100E300018D04FEA051545EA16754FEA06164FEA2F
:100E4000C30343EA52734FEAC2025FEA1C1CC0D1DB
:100E500011F4801F0BD141EA00014FF000004FF068
:100E6000004CB6E711F4801F04BF01430020B4F129
:100E7000FD0C88BFBCF5E06F3FF6AFAEB5EB030CE1
:100E800004BFB6EB020C5FEA500C50F1000041EBDE
:100E9000045170BD0EF0004E4EEA113114EB5C04AB
:100EA000C2BFD4EB0C0541EA045170BD41F480117E
:100EB0004FF0000E013C90E645EA060E8DE60CEA86
:100EC000135594EA0C0F08BF95EA0C0F3FF43BAFA3
:100ED00094EA0C0F0AD150EA01347FF434AF95EA5A
:100EE0000C0F7FF425AF104619462CE795EA0C0F3E
:100EF00006D152EA03353FF4FDAE1046194622E70B
:100F000050EA410618BF52EA43067FF4C5AE50EAE4
:100F100041047FF40DAF52EA43057FF4EBAE12E7D4
:100F20004FF0FF3C06E000BF4FF0010C02E000BFB5
:100F30004FF0010C4DF804CD4FEA410C7FEA6C5C98
:100F40004FEA430C18BF7FEA6C5C1BD001B050EA3B
:100F5000410C0CBF52EA430C91EA030F02BF90EA26
:100F6000020F0020704710F1000F91EA030F58BFE5
:100F7000994208BF90422CBFD8176FEAE37040F047
:100F8000010070474FEA410C7FEA6C5C02D150EAE5
:100F9000013C07D14FEA430C7FEA6C5CD6D152EAA0
:100FA000033CD3D05DF8040B704700BF8446104665
:100FB00062468C461946634600E000BF01B5FFF764
:100FC000B7FF002848BF10F1000F01BD4DF808ED34
:100FD000FFF7F4FF0CBF012000205DF808FB00BF05
:100FE0004DF808EDFFF7EAFF34BF012000205DF85F
:100FF00008FB00BF4DF808EDFFF7E0FF94BF0120AC
:1010000000205DF808FB00BF4DF808EDFFF7CEFFAC
:1010100094BF012000205DF808FB00BF4DF808EDEB
:10102000FFF7C4FF34BF012000205DF808FB00BFBC
:101030004FEA410212F5001215D211D56FF4787300
:10104000B3EB625212D94FEAC12343F0004343EAA3
:10105000505311F0004F23FA02F018BF404270477E
:101060004FF00000704750EA013005D111F0004008
:1010700008BF6FF0004070474FF00000704700BF9E
:101080004FEA4102B2F1E04324BFB3F5001CDCF1AA
:10109000FE5C0DD901F0004C4FEAC0024CEA5070E2
:1010A000B2F1004F40EB830008BF20F00100704711
:1010B00011F0804F21D113F13872BCBF01F0004014
:1010C000704741F480114FEA5252C2F11802C2F146
:1010D000200C10FA0CF320FA02F018BF40F00100C7
:1010E0004FEAC1234FEAD32303FA0CFC40EA0C0079
:1010F00023FA02F34FEA4303CCE77FEA625307D1B6
:1011000050EA01331EBF4FF0FE4040F440007047EC
:1011100001F0004040F0FE4040F40000704700BF86
:1011200080F0004002E000BF81F0004142001FBF9C
:101130005FEA410392EA030F7FEA226C7FEA236CA5
:101140006AD04FEA1262D2EB1363C1BFD21841409A
:1011500048404140B8BF5B42192B88BF704710F030
:10116000004F40F4000020F07F4018BF404211F0D3
:10117000004F41F4000121F07F4118BF494292EA3B
:10118000030F3FD0A2F1010241FA03FC10EB0C0067
:10119000C3F1200301FA03F100F0004302D54942F4
:1011A00060EB4000B0F5000F13D3B0F1807F06D3A1
:1011B00040084FEA310102F10102FE2A51D2B1F199
:1011C000004F40EBC25008BF20F0010040EA03008E
:1011D0007047490040EB000010F4000FA2F101023B
:1011E000EDD1B0FA80FCACF1080CB2EB0C0200FAC5
:1011F0000CF0AABF00EBC25052421843BCBFD04013
:101200001843704792F0000F81F4000106BF80F48C
:1012100000000132013BB5E74FEA41037FEA226C4F
:1012200018BF7FEA236C21D092EA030F04D092F01A
:10123000000F08BF0846704790EA010F1CBF00204E
:10124000704712F07F4F04D1400028BF40F00040AB
:10125000704712F100723CBF00F50000704700F0CB
:10126000004343F0FE4040F4000070477FEA2262F2
:1012700016BF08467FEA23630146420206BF5FEAC3
:10128000412390EA010F40F4800070474FF00003C3
:1012900004E000BF10F0004348BF40425FEA000C8A
:1012A00008BF704743F0964301464FF000001CE032
:1012B00050EA010208BF70474FF000030AE000BF88
:1012C00050EA010208BF704711F0004302D54042C6
:1012D00061EB41015FEA010C02BF84460146002038
:1012E00043F0B64308BFA3F18053A3F50003BCFA53
:1012F0008CF2083AA3EBC25310DB01FA02FC634400
:1013000000FA02FCC2F12002BCF1004F20FA02F206
:1013100043EB020008BF20F00100704702F12002F9
:1013200001FA02FCC2F1200250EA4C0021FA02F25A
:1013300043EB020008BF20EADC7070474FF0FF0C5F
:101340001CEAD0521EBF1CEAD15392EA0C0F93EA5A
:101350000C0F6FD01A4480EA010C400218BF5FEAFC
:1013600041211ED04FF0006343EA501043EA51116F
:10137000A0FB01310CF00040B1F5000F3EBF490069
:1013800041EAD3715B0040EA010062F17F02FD2A6D
:101390001DD8B3F1004F40EBC25008BF20F0010050
:1013A000704790F0000F0CF0004C08BF49024CEA67
:1013B000502040EA51207F3AC2BFD2F1FF0340EAF9
:1013C000C250704740F400004FF00003013A5DDC6A
:1013D00012F1190FDCBF00F000407047C2F10002AB
:1013E000410021FA02F1C2F1200200FA02FC5FEA98
:1013F000310040F1000053EA4C0308BF20EADC70E2
:10140000704792F0000F00F0004C02BF400010F453
:10141000000F013AF9D040EA0C0093F0000F01F000
:10142000004C02BF490011F4000F013BF9D041EA22
:101430000C018FE70CEAD15392EA0C0F18BF93EA24
:101440000C0F0AD030F0004C18BF31F0004CD8D14E
:1014500080EA010000F00040704790F0000F17BFD5
:1014600090F0004F084691F0000F91F0004F14D01B
:1014700092EA0C0F01D142020FD193EA0C0F03D173
:101480004B0218BF084608D180EA010000F0004076
:1014900040F0FE4040F40000704740F0FE4040F451
:1014A000400070474FF0FF0C1CEAD0521EBF1CEAF0
:1014B000D15392EA0C0F93EA0C0F69D0A2EB03020E
:1014C00080EA010C49024FEA402037D04FF08053A8
:1014D00043EA111143EA10130CF000408B4238BF6D
:1014E0005B0042F17D024FF4000C8B4224BF5B1A7B
:1014F00040EA0C00B3EB510F24BFA3EB510340EAC9
:101500005C00B3EB910F24BFA3EB910340EA9C0076
:10151000B3EBD10F24BFA3EBD10340EADC001B01E6
:1015200018BF5FEA1C1CE0D1FD2A3FF650AF8B428A
:1015300040EBC25008BF20F0010070470CF0004C97
:101540004CEA50207F32C2BFD2F1FF0340EAC250C2
:10155000704740F400004FF00003013A37E792F083
:10156000000F00F0004C02BF400010F4000F013AE1
:10157000F9D040EA0C0093F0000F01F0004C02BFDC
:10158000490011F4000F013BF9D041EA0C0195E745
:101590000CEAD15392EA0C0F08D142027FF47DAFDE
:1015A00093EA0C0F7FF470AF084676E793EA0C0FCE
:1015B00004D14B023FF44CAF08466EE730F0004CCC
:1015C00018BF31F0004CCAD130F000427FF45CAF5C
:1015D00031F000437FF43CAF5FE700BF4FF0FF3CCA
:1015E00006E000BF4FF0010C02E000BF4FF0010C1D
:1015F0004DF804CD4FEA40024FEA41037FEA226CE6
:1016000018BF7FEA236C11D001B052EA530C18BF07
:1016100090EA010F58BFB2EB030088BFC81738BF6C
:101620006FEAE17018BF40F0010070477FEA226C5A
:1016300002D15FEA402C05D17FEA236CE4D15FEA56
:10164000412CE1D05DF8040B704700BF844608468A
:101650006146FFE70FB5FFF7C9FF002848BF10F14B
:10166000000F0FBD4DF808EDFFF7F4FF0CBF012090
:1016700000205DF808FB00BF4DF808EDFFF7EAFF1A
:1016800034BF012000205DF808FB00BF4DF808EDD5
:10169000FFF7E0FF94BF012000205DF808FB00BFCA
:1016A0004DF808EDFFF7D2FF94BF012000205DF850
:1016B00008FB00BF4DF808EDFFF7C8FF34BF01205D
:1016C00000205DF808FB00BF4FEA4002B2F1FE4F78
:1016D0000FD34FF09E03B3EB12620DD94FEA0023F4
:1016E00043F0004310F0004F23FA02F018BF4042CD
:1016F00070474FF00000704712F1610F01D14202B4
:1017000005D110F0004008BF6FF0004070474FF067
:101710000000704742000ED2B2F1FE4F0BD34FF0E3
:101720009E03B3EB126209D44FEA002343F0004357
:1017300023FA02F070474FF00000704712F1610F7A
:1017400001D1420202D14FF0FF3070474FF000004C
:10175000704700BF0B460146184600F001B800BFB5
:1017600013460A460146022000F0BCBE014B186831
:10177000704700BFD098FF1F70B50F4E0F4D761BFE
:10178000B61018BF002405D0013455F8043B984723
:10179000A642F9D10A4E0B4D761B03F0F3FDB610AD
:1017A00018BF002406D0013455F8043B9847A642E0
:1017B000F9D170BD70BD00BF90530100905301007E
:1017C000A453010090530100024B0146186800F039
:1017D0000BB800BFD098FF1F024B0146186800F0FD
:1017E00045BF00BFD098FF1F2DE9F04F01F10B0559
:1017F000162D83B0064640F29F8035F0070500F1B4
:10180000BF80A94200F2BC8000F058FBB5F5FC7F18
:10181000C0F09C826B0A00F0BA80042B00F2838136
:10182000A80900F1390E4FEA4E033830C44F07EBD8
:101830008303A3F108015C68A14207D1ACE0002A50
:1018400080F2AC80E468A14200F0A680636823F0D7
:1018500003035A1B0F2AF2DDB9493C6901F1080E56
:10186000744500F0B381636823F003035A1B0F2A09
:1018700000F39981002AC1F814E0C1F810E080F269
:101880009E80B3F5007F80F06781DB0803F1010CD7
:1018900001229B1002FA03F34A6851F83C80C4F815
:1018A000088001EBCC091A43A9F10803E3604A6000
:1018B00041F83C40C8F80C40831001249C409442FD
:1018C00000F28A80144206D120F003006400144222
:1018D00000F10400FAD007EBC009CC468046DCF8E2
:1018E0000C108C4507D173E1002A80F28181C96810
:1018F0008C4500F06D814B6823F003035A1B0F2ABF
:10190000F2DD0C46D1F80CC054F8088F4B1945F0A5
:1019100001054D6042F00101C8F80CC03046CCF81A
:1019200008807B613B61C3F80CE0C3F808E05960B4
:101930009A5000F0C5FA1FE0102921D800F0BEFA35
:101940001025062302207E4F07EB8303A3F1080234
:101950005C68944200F045816368E168A56823F003
:101960000303234430465A68E96042F001028D6067
:101970005A6000F0A5FA0834204603B0BDE8F08FA5
:1019800000240C232046336003B0BDE8F08F802391
:101990004FF0400E3F2049E770465DE72344E16881
:1019A0005A68A56842F00102E96030468D605A60CD
:1019B00000F086FA0834204603B0BDE8F08F2344D7
:1019C00030465A6842F001025A6000F079FA083451
:1019D000204603B0BDE8F08FBC68636823F00308BD
:1019E000A84504D3C5EB08030F2B00F38C80554B9F
:1019F000DFF860911A68D9F8003001332A4404EB0B
:101A0000080A00F0608102F580520F3222F47F62F2
:101A100022F00F0211463046019200F04BFCB0F16B
:101A2000FF3F8346019A00F05881824500F2FC8016
:101A3000454B1968DA451144196000F05381D9F813
:101A40000000DFF810E101301BBFCAEB0B0A514464
:101A5000CEF800B019601BF0070100F01781C1F14A
:101A60000800C1F58051834408315A44C2F30B0287
:101A7000C2EB010949463046019300F01BFC431CB0
:101A8000019B00F03F81CBEB00024A4442F001028F
:101A90001968C7F808B04944BC42CBF80420196063
:101AA000DFF8A49016D0B8F10F0F40F2FD80626805
:101AB000A8F10C0323F00703E01802F001024FF035
:101AC000050E1A430F2B6260C0F804E0C0F808E06E
:101AD00000F21C811D4BBC681A68914288BF1960D6
:101AE0001B4B1A689142626888BF196022F003029A
:101AF0009542A2EB050301D80F2B04DC304600F021
:101B0000DFF9002438E7621943F0010345F00105CD
:101B100065603046BA60536000F0D2F90834204660
:101B200003B0BDE8F08F142B71D9542B00F2A480C0
:101B3000280B00F16F0E4FEA4E036E3076E600BFC1
:101B4000D498FF1FC4A3FF1FC8A3FF1FC0A3FF1F7C
:101B5000BCA3FF1FE09CFF1F5A0A042A5ED9142A67
:101B600000F2B38002F15C0149005B3207EB810CAB
:101B700057F82110DFF8DC81ACF1080C8C4500F03F
:101B800088804A6822F00302934202D289688C4519
:101B9000F7D1D1F80CC07A68C4F80CC0A160CCF8B9
:101BA0000840CC6088E6631942F0010745F0010562
:101BB000656030464B610B61C3F80CE0C3F808E088
:101BC0005F609A50083400F07BF9D5E64A6873E606
:101BD00008F1010818F0030F0CF1080C7FF47FAE38
:101BE00030E0DC68A34208BF02303FF435AEB3E614
:101BF0000B440C465A68C96854F8085F42F0010269
:101C00005A603046E9608D6000F05AF9B4E603F19D
